:100000005446495300010000E4D901006E91CB45EC
:10001000051001251605201748524F5405100152AE
:100020001605201748524F540510010716052017D2
:1000300048524F5403000000000000000000000080
:100040005446435300200000A4C9010000000000F2
:10005000004001200121000025210000272100008F
:10006000292100002B2100002D2100003D2100004E
:100070003D2100003D2100003D2100002F21000016
:10008000312100003D210000332100007B5700009A
:100090007B580000372100003D210000BD07001003
:1000A000372100007D390000D13900003D210000DA
:1000B0003D2100004F54000037210000372100008F
:1000C00043510000372100003D2100003D21000088
:1000D0000000000000000000000000000000000020
:1000E0000000000000000000000000000000000010
:1000F0000000000000000000000000000000000000
:1001000000000000000000000000000000000000EF
:1001100000000000000000000000000000000000DF
:1001200000000000000000000000000000000000CF
:1001300000000000000000000000000000000000BF
:1001400000000000000000000000000000000000AF
:1001500000F003F800F020F8FEE70D48016821F0F8
:100160000301002001C101C101C101C170470000AC
:10017000940D0010FEE7FEE7FEE7FEE7FEE7FEE770
:10018000FEE7FEE7FEE703480047FEE7FEE7000064
:10019000202100003D21000000F002F800F068F886
:1001A0000AA090E8000C82448344AAF10107DA45D2
:1001B00001D100F05DF8AFF2090EBAE80F0013F0BC
:1001C000010F18BFFB1A43F001031847E0B9010003
:1001D00010BA01000A444FF0000C10F8013B13F074
:1001E000070408BF10F8014B1D1108BF10F8015B90
:1001F000641E05D010F8016B641E01F8016BF9D183
:1002000013F0080F1EBF10F8014BAD1C0C1B09D1D9
:100210006D1E58BF01F801CBFAD505E014F8016B4B
:1002200001F8016B6D1EF9D59142D6D370470000DD
:10023000103A24BF78C878C1FAD8520724BF30C812
:1002400030C144BF04680C607047000000230024E4
:1002500000250026103A28BF78C1FBD8520728BFD6
:1002600030C148BF0B6070471FB51FBD10B510BD32
:10027000DFF80CD0FFF7F8FF04F076FF19F05DFB14
:100280000040012003B4FFF7F1FF03BC19F05CFB51
:1002900008B5002103200B460A46009118F0E2FC45
:1002A00008BD38B5AF4D0024AC80EC8018F0B7FC29
:1002B000E860FF206870AC48234622460460446032
:1002C00004720120A87003202146009418F0CAFC93
:1002D000012038BD38B5A34D02286C7822460DD0D8
:1002E000052814D0A24208BF38BD002003460246AC
:1002F0002146009018F0B6FC6C7038BD022908BF8A
:100300000224EFD00D2914BF01240024EAE70229BA
:1003100014BF64246524E5E738B5944B944C0A4631
:100320001B7824784FF0010C6343002401465B00E6
:100330006046009418F096FC38BD38B54FF0010CBB
:10034000062400250B46024621466046009518F01B
:1003500089FC38BD2DE9F04104460127002503F052
:100360000700804E8846012804BF0020F08046D058
:10037000022844D1F08804280BD2002818BFB068A6
:1003800002D118F090FCB06010F8011B2170B06031
:100390002EE0062808D218F088FCF188C1F105018A
:1003A000C900C840207023E0082808D218F081FC5A
:1003B000F188C1F10701C900C840207018E00C287D
:1003C00008D218F02CFCF188C1F10B01C900C8401B
:1003D00020700DE00E2808D218F023FCF188C1F13E
:1003E0000D01C900C840207002E0FF2020700027E6
:1003F000F088401C80B2F0800E2828BF012588F8C4
:1004000000503846BDE8F08130B403F00700002406
:10041000DFF850C1012804BFACF80440ACF8064036
:1004200014D05048BCF806308088022B05D2120246
:1004300042EA1020ACF8040005E0DCF80C50184447
:10044000284400F8022C581CACF806000C7030BC94
:100450000020704770B40546002003F0070C414CA3
:100460000646BCF1010F08BFE68008D03D4BBCF149
:10047000020F9B8806D0120242EA1322A2800E705D
:1004800070BC7047E0881A18E368401C9A5C2A70B8
:10049000E0800120F3E738B503F0070000240D46A3
:1004A000012809D12F4821460B46C48084800220B0
:1004B0000A46009418F0D6FB2C70002038BD2A4A5A
:1004C0001154704700225A2101200BF05EBC00221B
:1004D0005B2101200BF059BC00284FF0000001D037
:1004E0000BF08FBF0BF099BF1E49002008707047BA
:1004F0001C48007870471B49012008707047194953
:10050000002818BF01208870704708B5B9B10023D2
:100510000221012808BF8DF8001017D0022808BF5B
:100520008DF8001015D00522642808BF8DF8002032
:100530000CD0652808BF8DF800200AD00BE0012000
:100540000BF036FF012008F069FF08BD8DF801307F
:1005500001E08DF80110684607F0F3FF08BD01487F
:100560008078704700400020C04200208E4000206C
:100570008F4000207047002818BF0120FE490968FD
:1005800008627047FC480068006A002818BF012014
:100590007047F94A126802EBC00041637047F649A0
:1005A000096801EBC000006B00F480707047F24AEC
:1005B0001021126802EBC00041637047EE490A68DF
:1005C000D2F8402160F30D220868C0F8402170473E
:1005D000E9480068D0F84001C0F305207047E64ABA
:1005E00000F00F03C0F303101268002902EBC312DE
:1005F00002EB4010D0F8401114BF41F0010121F08E
:100600000101C0F840117047DB4A00F00F01C0F350
:100610000310126802EBC11101EB4010D0F8400149
:1006200000F001007047D44900230A681362026891
:10063000D1F800C0CCF800204268D1F800C0CCF856
:1006400004208268D1F800C0CCF80820C268D1F834
:1006500000C0CCF80C20426AD1F800C0CCF8402091
:10066000826AD1F800C0CCF844200269D1F800C0F9
:10067000CCF818204269D1F800C0CCF81C20826B5D
:10068000D1F800C0CCF86020C26BD1F800C0CCF823
:100690007020026CD1F800C0CCF87420426CD1F804
:1006A00000C0CCF87820826CD1F800C0CCF8802053
:1006B000C26CD1F800C0CCF88420026DD1F800C023
:1006C000CCF88820426DD1F800C0CCF88C20426E66
:1006D000D1F800C0CCF89C20826ED1F800C0CCF8D4
:1006E000A020C26ED1F800C0CCF8A420026FD1F8CF
:1006F00000C0CCF8A820826FD1F800C0CCF8C02090
:10070000C26FD1F800C0CCF8C420D0F88020D1F856
:1007100000C0CCF8C820D0F88420D1F800C0CCF8B4
:10072000CC20D0F88820D1F800C0CCF8D020D0F868
:100730008C20D1F800C0CCF8D420D0F89420D1F887
:1007400000C0CCF8DC20D0F89C20D1F800C0CCF858
:10075000F020D0F8A020D1F800C0CCF8F420D0F8D8
:10076000A420D1F800C0CCF8F820D0F8A820D1F807
:1007700000C0CCF8FC20D0F8AC20D1F800C0CCF8F8
:100780000021D0F8B020D1F800C0CCF80421D0F876
:10079000B420D1F800C0CCF80821D0F8B820D1F8A6
:1007A00000C0CCF80C21D0F8BC20D1F800C0CCF8A7
:1007B0001021D0F8C020D1F800C0CCF81421D0F816
:1007C000C420D1F800C0CCF81821D0F8C820D1F846
:1007D00000C0CCF81C21D0F8CC20D1F800C0CCF857
:1007E0002021D0F8D020D1F800C0CCF82421D0F8B6
:1007F000D420D1F800C0CCF83021D0F8D820D1F8DE
:1008000000C0CCF84021D0F8DC20D1F800C0CCF8F2
:100810004421D0F8E020D1F800C0CCF84821D0F82D
:10082000E420D1F800C0CCF84C21D0F8E820D1F871
:1008300000C0CCF85021D0F8EC20D1F800C0CCF8A2
:100840005421D0F8F020D1F800C0CCF85821D0F8CD
:10085000F420D1F800C0CCF85C21D0F81821D1F8F0
:1008600000C0CCF88021D0F81C21D1F800C0CCF811
:100870008421D0F82021D1F800C0CCF88821D0F80C
:100880002421D1F800C0CCF88C21D0F82821D1F84F
:1008900000C0CCF89021D0F82C21D1F800C0CCF8C1
:1008A0009421D0F83021D1F800C0CCF89821D0F8AC
:1008B0003421D1F800C0CCF89C21D0F83821D1F8EF
:1008C00000C0CCF8A021D0F83C21D1F800C0CCF871
:1008D000A421D0F84021D1F800C0CCF8B021D0F844
:1008E0004421D1F800C0CCF8C021D0F84821D1F87B
:1008F00000C0CCF8C421D0F84C21D1F800C0CCF80D
:10090000C821D0F85021D1F800C0CCF8CC21D0F8C3
:100910005421D1F800C0CCF8D021D0F85821D1F81A
:1009200000C0CCF8D421D0F85C21D1F800C0CCF8BC
:10093000D821D0F86021D1F800C0CCF8DC21D0F863
:100940006421D1F800C0CCF8E021D0F86821D1F8BA
:1009500000C0CCF8E421D0F86C21D1F800C0CCF86C
:10096000E821D0F87021D1F800C0CCF8EC21D0F803
:100970007421D1F800C001E0D0D40100CCF8F021FE
:10098000D0F87821D1F800C0CCF8F421D0F87C213F
:10099000D1F800C0CCF8F821D0F88021D1F800C0FF
:1009A000CCF8FC21D1F800C02122CCF83420D1F8B9
:1009B00000C0CCF83C20C269D1F800C0CCF824209B
:1009C000C26AD1F800C0CCF84820026BD1F800C050
:1009D000CCF84C20426FD1F800C0CCF8AC20D0F855
:1009E0009820D1F800C0CCF8E020D0F88421D1F8CC
:1009F00000C0CCF80022D0F88821D1F800C0CCF893
:100A00000422D0F88C21D1F800C0CCF80822D0F80C
:100A10009021D1F800C0CCF80C22D0F89421D1F864
:100A200000C0CCF81022D0F89821D1F800C0CCF842
:100A30001422D0F89C21D1F800C0CCF81822D0F8AC
:100A4000A021D1F800C0CCF81C22D0F8A421D1F804
:100A500000C0CCF82022D0F8A821D1F800C0CCF8F2
:100A60002422D0F8AC21D1F800C0CCF83022D0F844
:100A7000B021D1F800C0CCF84022D0F8B421D1F890
:100A800000C0CCF84422D0F8B821D1F800C0CCF88E
:100A90004822D0F8BC21D1F800C0CCF84C22D0F8C4
:100AA000C021D1F800C0CCF85022D0F8C421D1F830
:100AB00000C0CCF85422D0F8C821D1F800C0CCF83E
:100AC0005822D0F8CC21D1F800C0CCF85C22D0F864
:100AD000D021D1F800C0CCF86022D0F8D421D1F8D0
:100AE00000C0CCF86422D0F8D821D1F800C0CCF8EE
:100AF0006822D0F8DC21D1F800C0CCF86C22D0F804
:100B0000E021D1F800C0CCF87022D0F8E421D1F86F
:100B100000C0CCF87422D0F8E821D1F800C0CCF89D
:100B20007822D0F8EC21D1F800C0CCF87C22FA4A27
:100B3000126832F0FF0C08D1D1F800C0DCF890C088
:100B400062F3030C0A68C2F890C0F44A1370836F12
:100B500013F0010F1CBF02231370D0F8880010F0AF
:100B6000010F03D0107840F0010010700868D0F831
:100B7000C0000A6820F00100C2F8C0000868D0F880
:100B8000D000096820F00100C1F8D0007047E349A7
:100B900008707047E2480068D0F8C00000F001001B
:100BA0007047DF480068C068704770B5DC4D044688
:100BB0002868D0F8400114F0020F20F00D0118BF92
:100BC00041F0010114F0080F18BF41F0040114F0C6
:100BD000040F18BF41F008012868C0F8401114F054
:100BE000010F70D001F075F8064601F075F8014666
:100BF0002868C06800280EBF3046084631460028E5
:100C00002868D0F8C00114BF40F0010020F00100B6
:100C10002A68C2F8C00128680029D0F8E00114BF92
:100C200040F0010020F001002968C1F8E001BB4854
:100C300090F800C01CF0010F5DD0BA480168496C03
:100C4000026841F4803151640168896CC1F3090282
:100C500040F2E73103689B6CC3F30903934202D16E
:100C6000491EF7D117E0B1B11CF0010F07D0286879
:100C7000D0F8D000296840F00100C1F8D0001CF085
:100C8000020F38D02868D0F8C000296840F0010071
:100C9000C1F8C0002FE02968D1F8D0102A6821F0EF
:100CA0000101C2F8D0102968D1F8C0102A6821F0DB
:100CB0000101C2F8C0100168496C006821F480315C
:100CC000416418E0FFE72868D0F8C001296820F0E7
:100CD0000100C1F8C0012868D0F8E001296820F0BF
:100CE0000100C1F8E0012868D0F8C000296820F0B0
:100CF0000100C1F8C00014F0200F18BF002413D069
:100D0000204600F0F0FF0028286800EB4410D0F8DF
:100D1000401214BF41F0010121F00101C0F840125E
:100D2000641C022CECD370BD2868D0F840022968FE
:100D300020F00100C1F840022868D0F8600229685C
:100D400020F00100C1F8600270BD2DE9F003744984
:100D5000024602F00F03D1F800C000200CEBC315CF
:100D6000C2F3031305EB4313D3F8403113F0010F23
:100D70000DD142F01003C3F3031305EB4313D3F873
:100D8000403113F0010F04BFBDE8F00370470CEBD6
:100D9000C214D4F81C31DCF81C10C3F3080901F0AC
:100DA0000807D4F80011C1F30A08002142EA011330
:100DB000C3F3031305EB4313D3F8403113F0010FD2
:100DC00014D004EB4113D3F844C1CCF3080617F157
:100DD000000C1CBFD3F844C1CCF3023CD3F8403123
:100DE00006FA0CFCC3F3054360441844491C02296D
:100DF000DCD300FB08F0C9EB0911BDE8F00300EB00
:100E00004100704770B5464801680968006801F004
:100E10001F064068C0F30C050120FFF796FF04464B
:100E20000220FFF792FF044400F078FB211805FB35
:100E300006F0C0EB001001EB40004FF47A7148431C
:100E400047F23051B0FBF1F070BD2DE9F041344F65
:100E500005463868006810F01F0408BF012401200F
:100E6000FFF773FF06460220FFF76FFF064400F00E
:100E700055FB2D4A3118B5B1B2FBF5F0884298BF49
:100E800000200AD9C4EB0413401A5B00B0FBF3F056
:100E9000B0F5005F88BF41F6FF703B685B6860F3A8
:100EA0000C033868436038684068C0F30C00604346
:100EB000C0EB001001EB4000B2FBF0F0BDE8F081A8
:100EC00070B5174801680968006801F01F0540689F
:100ED000C0F30C060120FFF738FF04460220FFF79D
:100EE00034FF044400F01AFB06FB05F1C1EB0111CD
:100EF00004EB410108440C49B1FBF0F070BD084916
:100F00000A6852680B68C2F30C025B6860F30C035A
:100F10000868436010467047E0FE03001040002060
:100F2000D0D40100CCD4010000389C1CFB480068E0
:100F30004068C0F30C007047F849096801EBC01025
:100F4000D0F800014EF66021C0F30A00B1FBF0F0CA
:100F5000401C400870474EF66022B2FBF1F1491C7C
:100F60004908B2FBF1F2F0B4EC4D521C56082A6865
:100F70004FEA510C02EBC01238B1D2F804318C1F89
:100F800024F00104012806D019E0ACF10603981FF3
:100F900020F0010413E02868D0F8D00010F0010F11
:100FA0000DD04800B0F5006F88BF40F2FF702F6889
:100FB000D7F8E07060F30A072868C0F8E07041EAEB
:100FC0000C40C2F80001C2F80431C2F810413046AA
:100FD000F0BC7047D14A00F00F01C0F30310126853
:100FE00002EBC11101EB4010D0F84401C0F308003E
:100FF0007047CA4A00F00F03126802EBC312D2F81E
:101000001431C0F3031002EB4010CB1AD0F8442186
:1010100061F30802C0F84421D0F844119B1E63F329
:101020001841C0F844117047BC490A68D269096880
:1010300012F0100F00F00F0201EBC211D1F82021C5
:10104000C0F3031001EB4010D2B2D0F84401C0F35A
:10105000080008BF0022801A0004000C08BF01200D
:1010600070474FEA101C0007C00EAD4B02FA00F0AB
:101070001B6803EBCC1303EB810101F5C0410B6846
:10108000184308607047A64B020900071B68C00E92
:1010900003EBC21202EB810101F5C041096821FA9C
:1010A00000F000F0030070479C480068006D704736
:1010B0009A4910200968C8657047984B00F00F02E4
:1010C000C0F303101B6803EBC21202EB4010C0F820
:1010D0004C117047914A00F00F01C0F303101268E1
:1010E00002EBC11101EB4010D0F84C0170478B4B63
:1010F00000211A68D26912F0080F0CD000F00F011D
:101100001A68C0F3031002EBC11101EB4010D0F8D4
:101110004401C0F3023108467047804A1368DB6916
:10112000D2F800C043F00803CCF81C3000F00F03E5
:101130001268C0F3031002EBC31202EB4010D0F8A8
:10114000442161F30E32C0F844217047734B0021F3
:101150001A68D26912F0080F0CD000F00F011A685B
:10116000C0F3031002EBC11101EB4010D0F84801AD
:10117000C0F3024108467047684A00F00F03C0F30D
:101180000310126802EBC31202EB4010D0F84821A2
:1011900061F31242C0F848217047042988BF7047A4
:1011A00030B400235D4C2268D269254612F0080F46
:1011B00000F00F022D68C0F3031005EBC21202EB22
:1011C00040121CBFD2F84401C0F302330020D4F80F
:1011D00000C0DCF81CC01CF0080F1CBFD2F848018E
:1011E000C0F30240C91A0844042803DD081A011D8F
:1011F000042003E00028BCBF0144002019442368F8
:10120000DB69D4F800C043F00803CCF81C30D2F8F6
:10121000443161F30E33C2F84431D2F8481160F31F
:101220001241C2F8481130BC70473C490028086898
:10123000806904D0096840F0080088617047096837
:1012400020F0080088617047344800688069C0F366
:10125000C0007047314A00F00F01C0F3031012685C
:1012600002EBC11101EB4010D0F8480180B2704789
:101270002A4B00211A68D26912F0080F0CD000F036
:101280000F011A68C0F3031002EBC11101EB40100B
:10129000D0F84801C0F30051084670471F490200CA
:1012A000086880690A6800F00100926904D0096842
:1012B00042F001028A617047096822F001028A61E6
:1012C000704730B4022ADDF808C026BF921E5208CB
:1012D0000022022B26BF9B1E5B080023114C00F04E
:1012E0000F05A4FB0C4C4FEA1C14DFF830C0C0F310
:1012F0000310DCF800C00CEBC51C0CEB4010D0F860
:1013000054C161F3196C62F3134C63F30B2C64F357
:10131000070CC0F854C130BC70470000D0D40100A5
:10132000E8D40100CDCCCCCC70B49B4D00F00F04C0
:10133000C0F303102D68DDF80CC005EBC41404EBFA
:101340004010D0F854010029C0F30166C0F30345F2
:10135000C0F30324C0B218BF0E6012B16900891C2B
:10136000116013B16100891C1960BCF1000F04BF4A
:1013700070BC704700EB80008000CCF8000070BCAF
:10138000704770B491B000224FF480456C10EC4669
:1013900001E0082A05D2531C03EB8303B5FBF3F3EA
:1013A00004E0D31F03EB8303B4FBF3F35B1A48BFE2
:1013B0005B424CF82230521C102AEAD30026009BD4
:1013C00001215CF821209A42BCBF13460E46491CFD
:1013D0001029F6D3704900F00F02C0F3031009681A
:1013E00001EBC21101EB4011D1F85801C1F858616D
:1013F000082807D2401C00EB8000B5FBF0F011B0CC
:1014000070BC7047C01F00EB8000B4FBF0F011B05F
:1014100070BC7047604A00F00F01C0F303101268FF
:1014200002EBC11101EB4010D0F85801082834BF7D
:10143000401CC01F00EB800034BF4FF480414FF4CC
:101440000051B1FBF0F0704710F00F0F08BF70476C
:10145000514A00F00F000029126802EBC010D0F8CA
:1014600024110CBF21F4803141F48031C0F82411E3
:101470007047002110F00F0F0BD0474A00F00F000B
:10148000126802EBC010D0F8240110F4803F18BF9E
:10149000012108467047404902460868D0F8AC0070
:1014A00012F0010F0A68C0F3C000D2F8AC2005D0DA
:1014B000096842F00802C1F8AC207047096822F0C0
:1014C0000802C1F8AC207047334A136858671068A7
:1014D00081677047304900280868D0F8AC0005D013
:1014E000096840F00200C1F8AC007047096820F0BC
:1014F0000200C1F8AC007047274900280868D0F8FE
:10150000AC0005D0096840F00100C1F8AC0070479C
:10151000096820F00100C1F8AC00704770B41E4E9D
:1015200000203168D1F8401111F0010F04BF70BCE8
:10153000704711F0040F336801F00805D3F81C312F
:10154000D6F800C0C3F30803DCF800C1CCF30804EC
:10155000D6F800C0DCF844C1CCF3080C18BFC1F3C6
:1015600007403268D269C1F3052112F0080204D0A5
:101570003268D2F84421C2F30232002D18BF491C50
:101580000CFA02F201FB0200604370BCC3EB0311D2
:1015900000EB410070470000D0D40100FEF7F2BF1D
:1015A00010B5FEF7EFFF012818BF10BD0020FEF7B1
:1015B000E2FF21210020FEF7ECFF2121BDE81040D1
:1015C0000120FEF7E6BF10B5FEF7D4FFFEF7DAFF05
:1015D00001280AD10020FEF7CEFF21210020FEF7CE
:1015E000D8FF21210120FEF7D4FF0121052001F0C1
:1015F000A4FC0121052001F0A0FCFF490020487057
:1016000010BD10B5602001F0EEFCBDE81040602078
:1016100001F0DCBCF84A0146507A002818BF0120CE
:10162000002918BF012151727047F34A91699061F6
:1016300008467047F04800210172C1717047EE48BA
:1016400000210172C17170472DE9F34F00F00F05C1
:101650006800861E9DB0002445EA0410FEF7D4FF02
:10166000002845D01E9AC4EBC400002102EB0017ED
:10167000EC46C1EBC10307EBC30200200CEBC30334
:1016800052F8208043F82080401C0E28F8D3491CD3
:101690000229EED3D9490022301909684FF0020817
:1016A000C0EBC000434601EB001723FA02F101F042
:1016B0000101C2EBC200C1EBC1010CEBC10107EBA0
:1016C000C000B1E8004E00F5E76000F58040521C14
:1016D000A0E8004EB1E8004EA0E8004EB1E8004E90
:1016E000A0E8004ED1E90091C0E900914245DCD369
:1016F000641C022CB0D31FB0BDE8F08F70B5054656
:10170000FEF766FF29460446BC4DC0EBC400C2008C
:10171000286800F5804018F01DF92968C4EBC40062
:1017200001EBC00000F58040002101604160816054
:10173000C160016141618161C16101624162816297
:10174000C1620163416370BDAB494861FFF72DBAC7
:10175000AB4801688968AB4A11430268916001682F
:101760000968A94A00681143016000F0BBBE2DE979
:10177000F047A34A06460D4610688068A149014318
:1017800010688160106800689F490843116808600C
:1017900000F0A8FE0024984F002D63D00020FEF733
:1017A000EAFE286820B1FEF73EFF0020FEF7E3FEC8
:1017B00030467E61FFF7F9F90020FEF725FF00288B
:1017C00034D0DFF838826E6816B3FEF701FF814629
:1017D000C0EBC900C200D8F80000314600F58040D7
:1017E00018F0B8F8D8F80010C9EBC90001EBC00038
:1017F00000F58040046044608460C460046144611A
:101800008461C461046244628462C46204634463A8
:10181000E96841B1D8F800004FF4807200F5C0408B
:1018200018F098F802E0794800F084FD0120FEF7F6
:10183000EBFE18B91120FEF7E7FE28B1A9680029D0
:101840001CBF0120FFF700FF0220FEF7DDFE18B9E4
:101850001220FEF7D9FE28B1296900291CBF0220F9
:10186000FFF7F2FE3C72FC71BC61787A002078725E
:10187000602001F0B8FBBDE8F047602001F0A6BB96
:1018800010B50020FEF777FE00F00EFE5C48016800
:101890000968026821F0030141F00D7141F08051A7
:1018A000116001688968006821F0020141F00D7142
:1018B00041F08051816010BD602001F08BBB10B5FC
:1018C000602001F087FBFEF75DFE01280AD10020B1
:1018D000FEF751FE21210020FEF75BFE21210120B1
:1018E000FEF757FE4A480168496C006821F48031D0
:1018F00041640020FEF73FFE00F0D6FD404801683D
:101900000968026821F0030141F00D7141F0805136
:10191000116001688968006821F0020141F00D71D1
:1019200041F08051816010BD10B501F058FB10F0FE
:10193000600018BF012010BD2F48406970472E4835
:101940000078002818BF0120704770B5FEF71AFE16
:10195000002818BF70BD0025274C2572E571212194
:101960002846FEF716FE21210120FEF712FE257003
:10197000BDE870400120FEF7FEBD10B5FEF702FE87
:10198000002818BF10BD00201B4C2072E0712121DF
:10199000FEF7FFFD21210120FEF7FBFD0120FEF7F0
:1019A00006FE01202070BDE81040FEF7E4BD0020D7
:1019B000FEF7E1BD10490020C8710120FEF7DBBD34
:1019C0000D49C86170470C48C069704770B50A4C32
:1019D0000025E069411CE161207800281CBF00203F
:1019E000FEF7C9FD20212846FEF7D3FDA169002995
:1019F0001CBF284688470DE014400020E8D40100B1
:101A0000D8D401000200341203003412CC4200206A
:101A1000CCD40100FE48016841F02001016070BD96
:101A200070B5FC4C0125E069411CE161207800287B
:101A30001CBF0020FEF79FFD20212846FEF7A9FDD0
:101A4000A16900291CBF28468847F148016841F078
:101A50002001016070BDF0487047F0487047ED48C4
:101A6000006A7047EB48406A7047EA48806A7047EE
:101A70002DE9F00FE84E4FF0000C87B006F1380763
:101A8000E1464FF0FF3806F80C8007F80C900CF197
:101A9000010CBCF11C0FF6DB4FF0000C002807D93D
:101AA00012F80C4006F80C400CF1010C6045F7D818
:101AB0000024A4464FF0010A00280FD93257002A0B
:101AC00009DB082AB4BF1432083A1C2A3CBF0AFAC0
:101AD00002F242EA0C0C641C8442EFD3002214464A
:101AE0006D460AFA02FB1BEA0C0F1ABFAC54641CC9
:101AF00005F80280521C1C2AF3DB0022002817D9AB
:101B000016F902C0BCF1000F0FDBBCF1080FB4BF27
:101B10000CF1140CACF1080CBCF11C0F3ABF15F819
:101B20000CC007F802C007F80280521C8242E7D3BB
:101B3000B84C00220028C4F8209008D917F902C038
:101B4000944501D0276202E0521C8242F6D3B44F82
:101B50000020A7F1540CA7F11C060CF8008006F831
:101B6000009007F80090401C1C28F6DB002000299C
:101B700005D91A5C0CF80020401C8142F9D80020DD
:101B8000024600290BD91CF90230002B04DB1C2B68
:101B90003CBF0AFA03F31843521C8A42F3D30022D3
:101BA00013460AFA02FB1BEA000F1ABFAB545B1C78
:101BB00005F80280521C1C2AF3DB002200290AD9F6
:101BC0001CF90230002B03DB1C2B3CBFEB5CBB542D
:101BD000521C8A42F4D30022C4F82890002907D965
:101BE000BB56934201D0A76202E0521C8A42F7D34F
:101BF00011F0010F18BF1B2209D00AFA02F30342A9
:101C000003D10AFA02F2104301E0521EF5D5002278
:101C100013460AFA02F707421ABFAB545B1C05F8D9
:101C20000280521C1C2AF4DB002000290AD91CF96E
:101C30000020002A03DB1C2A3CBFAA5C3254401C53
:101C40008842F4D30020C4F8249000299EBF07B036
:101C5000BDE8F00F70473256824204D0666207B08A
:101C6000BDE8F00F7047401C8842F4D307B0BDE8D0
:101C7000F00F7047C0EB00106A4900EBC00001EBA9
:101C8000C0007047C0EBC00101EB0010664901EBDA
:101C900080007047DFF87CC1012B8CF802008CF8C3
:101CA000031003D9401C20F00100114600FB01F293
:101CB0004FF6FF718CF8040001EA4202ACF80C20E8
:101CC00001EA4000ACF80E007047524A5071917121
:101CD00070475048807970474E4840797047534A62
:101CE0001070517070475149085C704770B5494D8C
:101CF0000446687A002804BFE87917F0D2FE287AF3
:101D0000002808BF70BD4FF0000C6869634662464A
:101D1000614610F0020F1CBFDFF808C110F0040F7D
:101D200004D0AB893F4E23F00103334410F0010F80
:101D300004D010F0100F0CBF3B4A3B49ED69256001
:101D4000C4E90321C4E901C310F0200F14BF3848CF
:101D500000206061012070BD2E490020087270478C
:101D600010B50446FEF734FCC0EBC000C200314899
:101D7000006800F580412046BDE8104017F0EABD3C
:101D80002DE9F041FEF724FC04460020FFF7A2F9FC
:101D900000220546002C84BF0126264F21D93B682E
:101DA000C2EBC200002103EBC00C06FA01F028428E
:101DB00011D048080CEB800000F58040CB0700688C
:101DC000DB0E20FA03F3C3F30B00B0F57F6F02D9EB
:101DD0000020BDE8F081491C1C29E6D3521CA24218
:101DE000DDD30120BDE8F0812DE9F05F00F00F06A2
:101DF0000024104F8846750046EA0410FEF704FCE4
:101E0000002849D002218A460023C4EBC40013E015
:101E10004440002014400020CC420020E842002032
:101E20003C43002058430020904700201E400020E3
:101E3000EC470020E8D4010008EB001B002000293B
:101E400008D92AFA00F202F001029A421CBF401C93
:101E50008842F6D388421CD2A5F10209A144D7F8E2
:101E600000E0C3EBC302C9EBC9090BEBC20C0EEBDC
:101E70000919C0EBC000002209EBC00909EB820080
:101E800000F58040D0F838074CF82200521C0E2A8A
:101E9000F4D35B1C022BD1D3641C022CACD3BDE861
:101EA000F09F2DE9F05F00F00F0670000025DFF8CD
:101EB0007494A0F10208012746EA051A5046FEF77D
:101EC000A3FB002839D05046FFF711F907FA00F4B8
:101ED000022C88BF02245046FFF7FCF80022002C99
:101EE0002BD908EB0501D9F80030C1EBC10103EB98
:101EF000011BC2EBC20300210BEBC30A07FA01F37B
:101F0000034214D04B080AEB830303F580434FEAE6
:101F1000C17CD3F838374FEADC6C23FA0CF3C3F3F7
:101F20000B03B3F57F6F02D90020BDE8F09F491C79
:101F30001C29E3D3521CA242DBD36D1C022DBBD360
:101F40000120BDE8F09FC1EBC103F6494FF6FF7CCD
:101F5000096801EBC301430801EB830101F58041EE
:101F6000C007C00E0CFA00FC0B6802FA00F023EA6E
:101F70000C03184308607047EA4AC1EBC1011268BC
:101F800002EBC101420801EB820101F58041C0076B
:101F90000968C00E21FA00F080B270472DE9FF4FAA
:101FA000E04883B01D460068109C00F5804017464D
:101FB0000E460190FEF7E6FA5FEA00081CBF00201B
:101FC000FEF7D9FA0020FFF785F8824670190090D5
:101FD000B04284BF4FF0010B4FF6FF7E28D9019825
:101FE000C6EBC6014FF0000C00EBC101039B17E0EC
:101FF0000BFA03F010EA0A0F11D05808DD0751F868
:102000002020ED0E0EFA05F922EA090234F8029BAF
:102010000CF1010C09FA05F52A4341F820205B1C5C
:10202000BC4538BF1C2BE3D30098761C8642D6D320
:10203000B8F1000F04BF07B0BDE8F08F0020BA4927
:10204000C87107B00120BDE8F04FFEF794BA2DE942
:10205000F0470746B3489A46144600680E46089D66
:1020600000F58049FEF78EFA5FEA00081CBF0020E9
:10207000FEF781FA06EB0A03B34284BFAB4907EBD4
:10208000040C1CD9C6EBC6003C4609EBC0000FE0AF
:102090000A571C2A0BD202EBD27A4FEA6A0AD207FD
:1020A00050F82AA0D20E2AFA02F225F8022B641C5C
:1020B000644538BF1C2CEBD3761C9E42E2D3B8F1AA
:1020C000000F08BFBDE8F08700209749C871BDE840
:1020D000F0470120FEF74FBA2DE9F05F0027DFF847
:1020E0004882904A4FF6FF7600280C4647D0116888
:1020F00001F5804900F00F01C0F3031001290EBF64
:1021000000210229BDE8F09F022828BFBDE8F09F0A
:1021100001EB000AFEF736FA05001CBF0020FEF7AF
:102120002AFA0020CAEBCA0109EB0119C0EBC00171
:10213000002209EBC10153084FEAC27C4FEADC6C74
:1021400001EB830306FA0CFBD3F838A704FA0CFC66
:102150002AEA0B0A4AEA0C0C521CC3F838C71C2A9C
:10216000E9D3401C0228E1D3002D08BFBDE8F09F51
:1021700088F80770BDE8F05F0120FEF7FCB9106831
:1021800000F58049FEF7FEF905001CBF0020FEF7B0
:10219000F2F94FF0000CCCEBCC00002209EBC001AF
:1021A0005308D007C00E06FA00FB51F823A004FA2A
:1021B00000F02AEA0B0A4AEA0000521C41F8230008
:1021C0001C2AEDD30CF1010CBCF1210FE3D3002D3F
:1021D000CED1BDE8F09F10B5FEF726FF5249088228
:1021E00010BD514AC1B200F47063128A914288BF97
:1021F00011464FF0640C01FB0CF1B1FBF2F11A0A2D
:1022000002FB0C1189B210F4805F12BF08B2484281
:1022100000B270470028B8BF404280B2B4BF00216E
:102220004FF4805100F4706211433F4AC0B2128AE9
:10223000504341EA102070473D4800F07BB870B52C
:102240003B4800F077F8374840F6F801006800F5A1
:10225000804017F084FB0020FEF751FE0021084665
:10226000FEF75BFF0020FEF7E0FF00210120FEF7F4
:1022700054FF00211120FEF750FF00210846FEF711
:102280007BFF00210120FEF777FF00211120FEF7E0
:1022900073FF0120FEF750FE04460120FEF79AFE70
:1022A00006461120FEF796FE0546A64288BF264642
:1022B000A54288BF254631460120FEF79AFE2946F1
:1022C0001120FEF796FE0020FEF761FC002102209F
:1022D000FEF723FF00211220FEF71FFF002102203E
:1022E000FEF74AFFBDE8704000211220FEF744BF10
:1022F0000D4910B502204861FEF757FC094C4FF418
:102300008071206800F5C04017F029FB20684FF469
:10231000E76100F5804017F022FBBDE81040002087
:10232000FEF7EDBDE8D4010014400020E842002093
:10233000CC42002070B5144D04464FF480712868DB
:1023400000F5C04017F00BFB002101206256002A67
:1023500015DBD31702EB137C4FEA2C132E682CF0FD
:102360000F0C06EBC31303EB810303F5C043A2EB91
:102370000C0252001E6800FA02F232431A60491C35
:102380001C29E3D370BD0000E8D4010070B4002420
:102390006B4982B04FF0010C002814BF0C7081F81B
:1023A00000C0684D28680068674A10432A681060BA
:1023B0000978664A31B113686548D8601368654882
:1023C000986006E013686448D86013684FF0BB70EB
:1023D00098606248006830F0FF0305D11368DB683D
:1023E00060F303031068C36040F2E243C1B11068B8
:1023F0008068166840F01800B0600120009004E08A
:102400000198461E0196FBD20098461E009628BFF2
:102410000193F5D210688068166840F48050B0606F
:102420000120009004E00198461E0196FBD200981E
:10243000461E009628BF0193F5D21068C068166842
:1024400040F03000F0601068D0F8B000166840F03E
:102450000100C6F8B0000120009004E00198461E7B
:102460000196FBD20098461E009628BF0193F5D234
:102470001068C0F87CC013684FF4E0601861106801
:10248000C0F8884000291CBF1068C0F894C02868B4
:102490000068296820F0040040F00D7040F0805082
:1024A000086002B070BC704728480168C9680268BB
:1024B00021F03001D1602249097839B10168896879
:1024C000006821F0180121F4805181601D480168E5
:1024D0000968006821F0040141F00D7141F080515C
:1024E00001607047174801680968174A006811437E
:1024F000016013480178154831B10168896841F2DB
:1025000018021143026891600168C968026841F0CD
:102510003001D1600168D1F8B010006841F00101CC
:10252000C0F8B01070470E49C0B241EA0020074918
:1025300009680864704705490A48096808647047D3
:1025400040400020D8D4010004003412D4D401004B
:10255000057601002000760105F40100D0FE03009D
:1025600013005FA000005FA05948584902689161BC
:102570000268891CD1610268491E516302681268B1
:10258000036822F0030242F00D7242F080521A609A
:1025900002685269036822F0010242F00D7242F0B3
:1025A00080525A610268126911430268116102681F
:1025B0004849916000684849C16048490020086066
:1025C000704770B501F071F9444D2C682CB10020B2
:1025D000286001F06FF9204670BD30BF00F0A3FD08
:1025E0000028F2D000F0B2FD6860EEE72DE9F0417E
:1025F00001F05BF9354E364CDFF8E080771CD8F8F7
:1026000000503DB10020C8F8000001F053F9284601
:10261000BDE8F08172B6206846632068876120BFFC
:10262000206886612068476362B6BFF36F8FBFF38F
:102630004F8F00F078FD0028E1D000F087FDC8F84A
:102640000400DCE7224801680968026821F0030100
:1026500041F00D7141F08051116002682049916094
:10266000016809691F4A00681143016130BF704762
:1026700072B616491648026851630268C91CD161D6
:102680000068891E816162B6704711480168096857
:10269000154A00681143016070470D4801680968D8
:1026A000006821F0030141F00D7141F0805101609B
:1026B000704772B605490648026891610268891C34
:1026C000D1610068491E416362B670470000341250
:1026D000D8D401003C0034122800341244400020B9
:1026E000080034120100341203003412704700282D
:1026F00018BF0120B64909684860704700220029C8
:1027000009D950F8043BB3F1FF3F01D000207047D6
:10271000521C8A42F5D30120704730B44FF0000CB0
:102720006346002A13D950F8044B51F82350AC42A9
:102730001CBF0CF1010C1FFA8CFC5B1C9BB293427A
:10274000F1D3BCF1000F1EBF002030BC7047012048
:1027500030BC70472DE9F041054601F0B0F8002487
:102760009B4B21274FF482582646186807602E603D
:1027700018680068196840F004000860186800686C
:1027800010F0040FFAD11868C0F8008040202946E4
:10279000002251F804CBBCF1FF3F08D01868066056
:1027A000601CC4B2082CE0D30220BDE8F081521CAA
:1027B0008242EED3186806600120BDE8F0812DE961
:1027C000F041044601F07BF80020814B0925844646
:1027D00019680D60C4F800C0196809681A6841F0EA
:1027E000040111601968096811F0040FFAD121463B
:1027F0004FF48066002251F8047BB7F1FF3F09D007
:102800001968C1F800C0401CC0B20328E0D3022000
:10281000BDE8F081521CB242EDD31868C0F800C088
:102820000120BDE8F0812DE9F05F0F4680460426C7
:102830004FF0020A4FF0000BDFF8949101F03FF8DF
:10284000D9F8001044463846C1F800A00F21B0E87E
:102850002C10A4E82C10491EF9D2D9F80000006809
:10286000D9F8001040F004000860D9F800000068B2
:1028700010F0040F07D000BF00BFD9F800000068B7
:1028800010F0040FF7D1D9F80000C0F800B04546A9
:1028900038460F21D5E90023D5E902C4D0F800E07D
:1028A000964504BF42689A4205D18268624504BFDA
:1028B000C268A24208D0761E03D34046FFF74AFF03
:1028C000BCE70220BDE8F09F10301035491EE1D270
:1028D0000120BDE8F09F70B50D46044600F0EFFF03
:1028E0004FF480722146284617F034F8012070BD5D
:1028F0002DE9F041C0B014460E46054610F0FF0F1A
:1029000023D025F0FF086F4600F0D9FF4FF4807206
:102910004146384617F01EF8E8B2C0F58077A74266
:1029200088BF274668443A46314617F01DF84046AE
:10293000FFF710FF022843D069464046FFF773FFB8
:10294000022841D03D443E44E41BB4F5807F19D3B6
:102950004FF480723146684617F006F82846FFF7B4
:10296000F9FE02282CD069462846FFF75CFF0228B2
:102970002AD0A4F5807405F5807506F58076B4F547
:10298000807FE5D2C4B16F4600F099FF4FF48072AA
:102990002946384616F0DEFF22463146684616F0D4
:1029A000E3FF2846FFF7D6FE022809D069462846ED
:1029B000FFF739FF022807D040B00120BDE8F081C1
:1029C00040B00A20BDE8F08140B00B20BDE8F081A6
:1029D000BCD4010028490A6810600968086100F049
:1029E00016B825490A6810600968486100F00FB8F8
:1029F00021490968486770471F4909688867704717
:102A00001D480121026811660068016570471B4A74
:102A10001168096B10F0010F18BF21F4404110F04C
:102A2000020F1CBF21F4405141F4805110F0040FFB
:102A300018BF41F4406110F0080F18BF41F4407115
:102A400010F0100F18BF41F0C00110F0200F18BF98
:102A500041F0300110F0400F18BF41F00C0110F0B0
:102A6000800F18BF41F0030141F4BE00116840F02F
:102A70002040086370470000C4D40100CCD401009A
:102A8000FE4801688A68FE4903680A439A60026842
:102A9000D26811430268D16001684969F94A006847
:102AA000114341617047F54801684969026821F0A6
:102AB000010141F00D7141F0805151610168C96817
:102AC000026821F0400141F00D7141F08051D16068
:102AD00001688968006821F0400141F00D7141F002
:102AE00080518160704710B5E44C20688168E448EB
:102AF0002268014391602168C96808432168C86061
:102B000020684069DF49084321684861DE483F2169
:102B10000268D160026800219163026891640068D4
:102B2000C0F8B01003210A2000F007FA0A2000F0D4
:102B300028FA20684069216820F0010040F00D70FB
:102B400040F0805048612068C068216820F0400053
:102B500040F00D7040F08050C860206880682168A7
:102B600020F0400040F00D7040F08050886010BDB3
:102B7000C54A136818601368596048431168886033
:102B80007047C14A1368186013685960484310F0D1
:102B9000010F18BF401C116888607047BA49096866
:102BA000C1F8B0007047B84918B1096801208864BD
:102BB00070470968002088647047B3490A689063C9
:102BC0000868C068096840F00200C8607047DFF814
:102BD000B8C210B4DCF800402062DCF800004162AA
:102BE000DCF800008262DCF80000C362DCF8001050
:102BF00001200863DCF80000406B10F0010F09D0E1
:102C000000BF00BF00BF00BFDCF80000406B10F049
:102C1000010FF5D110F0020018BF4FF0FF3010BCCB
:102C2000704799480168C968006821F00201C160D5
:102C3000704795480168C968006841F00101C160AA
:102C40007047914BD3F800C0CCF82000186841625F
:102C5000186882621968012008641868406C10F0D6
:102C6000010F08D000BF00BF00BF00BF1868406C54
:102C700010F0010FF6D110F0060018BF4FF0FF3032
:102C8000704781480168C968006821F00101C1608E
:102C900070477D480168C968006841F00401C1605F
:102CA0007047027C017B02F03F0241EA0241764A12
:102CB00013689965136801685962136841689962DD
:102CC00013688168D9621368012119651168496D1B
:102CD00011F0010F08D000BF00BF00BF00BF116896
:102CE000496D11F0010FF6D11368DB6D8382136813
:102CF000DB6D1B0CC38213681B6E038313681B6E92
:102D00001B0C438313685B6E83831268526EC2F39D
:102D10000E42C28311F0020018BF4FF0FF3070471F
:102D200059480168C968006821F00401C160704712
:102D300055480168C968006841F00801C1607047E2
:102D4000DFF844C110B4DCF80040A267DCF80020D2
:102D50001062DCF800004362DCF800008162DCF8FD
:102D6000001001200867DCF80000406F10F0010F30
:102D700009D000BF00BF00BF00BFDCF80000406FFB
:102D800010F0010FF5D110F0060018BF4FF0FF3022
:102D900010BC70473C480168C968006821F0080110
:102DA000C160704701684FEA314237490B68C3F888
:102DB00098200A684068C2F89C000868C0680968E2
:102DC00040F02000C86070472F4A136818621068EE
:102DD000416211680120C1F890001068D0F8940099
:102DE00010F0010F09D000BF00BF00BF00BF106886
:102DF000D0F8940010F0010FF5D110F0060018BFC4
:102E00004FF0FF30704720480168C968006821F022
:102E10002001C16070471C480168C968006841F022
:102E20001001C1607047A3F1050C174B10B41C686A
:102E3000C4F888C0D3F800C0CCF8200018684262FB
:102E40001868816219680120C1F880001868D0F8FC
:102E5000840010F0010F09D000BF00BF00BF00BF09
:102E60001868D0F8840010F0010FF5D110F00600BA
:102E700018BF4FF0FF3010BC70470000D8D40100DD
:102E80004000341201003412DCD401000348016810
:102E9000C968006821F01001C1607047DCD40100EE
:102EA000234810B5026802211165026801211166EC
:102EB000036810225A67036841F206025A660368E3
:102EC00000229A660268C2F8881002689021C2F84F
:102ED00084100168D1F88410026841F00101C2F841
:102EE000841002684FF48171116600680166032046
:102EF00000F047F80021032000F01FF8002010BD6B
:102F000010B5032000F048F809484FF480710268BA
:102F1000116602680021116602681021916700683D
:102F200002214165002010BD024900200870704751
:102F3000C8D401004C400020704700F00303DA00C1
:102F40004FF0FF0C0CFA02F24FF0050C0CEBC30330
:102F5000994000F00C03002808DA30480068184453
:102F60004369114093431943416170472C480068FD
:102F70001844D0F80033114093431943C0F80013AC
:102F8000704700F01F01012202FA01F1244A4009B2
:102F9000126842F82010704700F01F01012202FA67
:102FA00001F11F4A4009126802EB8000C0F880104E
:102FB000704700F01F01012202FA01F1184A40098E
:102FC000126802EB8000C0F880117047144909684C
:102FD0000860704712490968C1F8800070471048BE
:102FE0000068006870470E490968C1F880017047A1
:102FF0000A4800688068704708490A68926809684A
:10300000886010467047054A1268926800F1100304
:1030100052F8230042F8231070470000B8D4010092
:10302000B4D4010002210C20FFF787BFC748016814
:103030008A68C74903680A439A600268D2680068D0
:103040001143C1607047C14801688968026821F472
:10305000805141F00D7141F0805191600168C96863
:10306000006821F4805141F00D7141F08051C16040
:103070007047B84881B00168096F11F4007FFAD138
:103080000168896E11F0010F09D00168D1F8841030
:1030900000910168D1F88410009A9142F9D001683A
:1030A000096F11F4007F03D102684CF271011166BF
:1030B000006842F24131816601B07047A5494FF482
:1030C0000D520B689A660A68126F0B68DA66002860
:1030D00008BF012080B24FF05C5242EA00200A682B
:1030E000506609684FF01140C1F88000C1E7994867
:1030F00081B00168096F11F4007FFAD10168896E0F
:1031000011F0010F09D00168D1F884100091016815
:10311000D1F88410009A9142F9D000684FF40D5113
:10312000816601B0704789480068806810F480505B
:1031300008BF704787480068806E00F00100704744
:1031400084480068406EC0F30F20704781480068D3
:10315000D0F88400704710B50C20FFF72AFF0C2030
:10316000FFF70FFF7B4902200968486710BD7949C6
:1031700010B50968032088670C20FFF70DFFBDE834
:1031800010400C20FFF715BF734A11681060084605
:103190007047704810B50168096F0068C1666E48D5
:1031A0000068002818BF80476C48016841F48051CE
:1031B000016010BD684840687047644810B50168F8
:1031C0008A68634903680A439A600268D2680068A3
:1031D0001143C1605F4C0320216888670C20FFF712
:1031E000DBFE0C20FFF7E5FE00F0B2F95C4B04209B
:1031F0001968C1F8880019684FF6FF70C1F88C0093
:1032000072B621684FF40D5088662068006F2168FF
:10321000C86621685348486621684FF01140C1F8DC
:103220008000FFF726FF19684FF40070086662B649
:1032300010BD38B572B647480168096F11F4007FB8
:10324000FAD10168896E11F0010F09D00168D1F837
:10325000841000910168D1F88410009A9142F9D04D
:1032600002684FF40D5191663D494FF400330A68EE
:10327000136662B60968D1F80412344C002948D0AC
:10328000354B4FF6FF72511A996022689269D4F853
:1032900000C002F00F02DCF81CC00CF00F0C6244FE
:1032A000121D9140A1F5EA42DFF8BCC0313A6245F7
:1032B0002FD20068D0F88400C0F10110D860B0F5BA
:1032C000803F26D20004B0FBF1F040F2C911484320
:1032D0001861B0F57A7F38BF4FF47A70DFF88CC090
:1032E000DCF80810002908BFCCF80800DCF804203E
:1032F000CCF80020DCF80810CCE901108A421FD974
:10330000824205D9814201D9596002E0586000E04B
:103310005A6000F02EF920688068216820F48050FF
:1033200040F00D7040F0805088602068C0682168CF
:1033300020F4805040F00D7040F08050C86038BDDF
:103340008242E5D88142E1D8DEE70000D8D401000E
:1033500000103412E4D4010050400020444000200A
:10336000E0D4010000FFFF372F6E16001848002040
:10337000134801688968134A006811438160124844
:1033800001684969026841F4007151610168096985
:10339000026841F00401116101680969006841F0A7
:1033A0001001016170470849096888607047BFF3E0
:1033B0004F8F054905480968C860BFF34F8FFEE786
:1033C000D8D4010004003412B8D401000400FA0576
:1033D000254801688968254A0068114381602448AE
:1033E00001684969026841F0010151610168096B96
:1033F000204A21F440511143026811630168096AAF
:10340000036821F00F021C490A431A621B4B8A1EF3
:103410001B68C3F8C4200068016570471448006841
:10342000006900F070007047114815490268116387
:103430000268144951630168496C026821F4003143
:1034400051640168496C40F2FF32114302685164D3
:103450000168496C006821F4803141647047044878
:103460000068406870470000D8D40100040034129E
:10347000CCD4010000205FA003005FA0D4D40100E1
:10348000C08C5FA095995FA0022824BF00207047E0
:10349000B84B53F8202043F820101046704770B501
:1034A000B54C2068006FB34D10F0010F06D02168B5
:1034B0000120C8662868002818BF80472068006F70
:1034C00010F0020F08BF70BD02202168C86668684E
:1034D000002808BF70BDBDE870400047A74810B580
:1034E00001688A68A64903680A439A600268D2683C
:1034F00011430268D160A04902220B681A65D1F815
:1035000000C00123CCF86030D1F800C00323CCF810
:103510006C3009684A6501688968026821F0800199
:1035200041F00D7141F0805191600168C9680068F7
:1035300021F0800141F00D7141F08051C1600920FE
:10354000FFF71FFD0221BDE810400920FFF7F5BC81
:103550008A4801688A688A4903680A439A6002684F
:10356000D26800681143C160834902200968086578
:103570007047814902200968486580480168896868
:10358000026821F0800141F00D7141F0805191609D
:103590000168C968006821F0800141F00D7141F0B7
:1035A0008051C1607047754800688068C0F3C010E2
:1035B000704771480168096F11F4007F04D00068FA
:1035C0004FF440710166704700684FF480710166E6
:1035D000704710B5684C2068C06F10F0020F4FF0B4
:1035E000010018BF03202168486700F0F3F8634921
:1035F0000A689269096802F00F02D040C96922681E
:1036000001F00F01C8400521B0FBF1F04FF4057146
:103610000009C2F8801017F062FE5A4A5A4B17F0A0
:1036200071FE17F02FFE2168C1F884002068006F3A
:1036300010F4007F04D021684FF44070086610BD7C
:1036400021684FF48070086610BD4B480168096F0F
:1036500011F4807F04D000684FF440710166704718
:1036600000684FF4007101667047434B30B41A682C
:10367000D26F12F0010F1DBF4FF0030C1A68C2F891
:1036800074C0022204BFD3F800C0CCF874204FF0FD
:10369000020C00EB4005C5EBC0104FF49674C1EB73
:1036A000C0004C4300EB8000384904EB4010A1FB04
:1036B000001032490022C0080C68A469096804F0AF
:1036C0000F04C96901F00F012144C8400521B0FB76
:1036D000F1F0B0F5803F05D3511C4008CAB2B0F5F7
:1036E000803FF9D242EA0C211A6841F01001C2F879
:1036F00088101968C1F88C001868006F10F4807F7A
:1037000005D019684FF44070086630BC70471968DE
:103710004FF40070086630BC704717480168096FA5
:1037200011F4003F04D000684FF440310166704747
:1037300000684FF48031016670470F480168096FD7
:1037400011F4803F04D000684FF4403101667047A7
:1037500000684FF400310166704707480068006F49
:10376000C0F30020704704480068006FC0F3402099
:103770007047000064400020E0D40100D8D401006C
:10378000800034127B14AE47E17A843FCDCCCCCCA0
:10379000244900200A68906009680860224948604E
:1037A000704710B51F4C2168486021680020886070
:1037B0000221401EFFF7C1FB21680720086010BDF1
:1037C0001849002009680860704717480188491C9B
:1037D000018070471448806870472DE9F041124C11
:1037E000002705462780A0684FF47A71B0FBF1F0FE
:1037F0000C4E401E31684860306887600221C81E48
:10380000FFF79BFB3168072008602188A942FCD3A1
:1038100030680760BDE8F081044948430249886088
:1038200070470000B0D401006C40002040420F00FF
:10383000704770B52C4C05464FF40D5021688866D2
:1038400021680320C86621682848486621684CF230
:103850007100086621682648C1F88000216842F29C
:103860004630886602210020FFF767FB0020FFF743
:1038700088FB002D08BF70BD2068806E42F2413188
:1038800008432168886670BD174810B50268012199
:10389000916700684FF40D5181660020FFF77CFBB3
:1038A000BDE810400020FFF784BB0F4901200968E4
:1038B000486770470C4901200968886770470A49C2
:1038C0004CF27100096808667047074881B04CF2F5
:1038D0007101026811660168096F0268D1660068AB
:1038E000006F009001B07047C0D40100073839372D
:1038F000009C1C9170B5FF4D00244FF480612C702A
:103900006C70FD4816F02BF84FF48061FB4816F000
:1039100026F8FB486C60AC70046044608460C4604E
:10392000046144618461C461046244628462C4626B
:10393000046344638463C463046444648464C4644B
:10394000046544658465C465046644668466C4662B
:10395000EC705821703016F002F85821E94815F043
:10396000FEFFAC6070BDE3488078002818BF0120DE
:103970007047E048C078002818BF01207047DD4834
:103980004078002818BF01207047DF48704770B5A5
:10399000DE4EDF4D0446014632782878DA4B10447B
:1039A0004200184615F0E0FF32782878D54B1044D5
:1039B00042002146184615F0D7FFCE490120C870B5
:1039C00070BDCC4880687047CB4870472DE9F04106
:1039D000C84F80463878002814BFCE48CE480578B6
:1039E00014BFCE48CE48047805FB04F6FFF748F82C
:1039F00021462846FFF7BCF8C04A4346A2F580613D
:103A00000846FFF7E4F8FFF74EF872004146BB485E
:103A100015F0AAFF01207870BDE8F0812DE9F0478C
:103A2000B44D044601462878DFF8CCC2DFF8E482C2
:103A3000DFF8E492B94EBA4F002815BF98F800207D
:103A400099F8002033783B7802FB03F04FEA4002FC
:103A5000604615F089FF2878DFF8A0C221460028CB
:103A600015BF98F8002099F8002033783B7802FBC6
:103A700003F04FEA4002604615F076FF01206870BF
:103A8000BDE8F0879B484068704770B5A54C054677
:103A9000014622789A48520015F066FF227829469E
:103AA0005200A14815F060FF92490120887070BD56
:103AB0002DE9F04F8F4DADF2344D95F801B095F8EA
:103AC00002A095F80390FDF769FDCDF82C04FDF7F1
:103AD00036FFCDF82804FDF763FD0020FDF70FFA4F
:103AE000CDF82404FDF749FF00240127CDF8184440
:103AF00004F0F2FD012811D00DF58060FEF7F6F814
:103B0000002800F07F810DF5806005F029FBDDF8CD
:103B1000080410B3BAF1000F05D01EE00120CDF863
:103B2000180400F072B906460CB3FEF7A9FF7D4DEC
:103B300001212878FFF71CF87B4A3346A2F13801AF
:103B40000846FFF744F8FEF7AEFF287831464200FA
:103B5000754815F009FF67488770DDF804040028F0
:103B600000F0B480BBF1000F11D000F0AFB86D4D84
:103B7000314628784200624815F0F6FE2878314632
:103B80004200694815F0F0FE5A488770E5E7DFF813
:103B90006481054698F8000000283DD1D8F80460FB
:103BA00026B35C480078CDF820045C480078CDF856
:103BB0001C04FEF765FFDDF81C14DDF82004FEF799
:103BC000E0FF294632460846FFF73BF8FEF76BFF59
:103BD00056480078022804BF304605F07FF8534865
:103BE0000078092804BF284605F078F85048007886
:103BF000012811D94D4E3078042804BF284605F01D
:103C00006DF82946684616F0ABFB05463078052866
:103C100004BF284605F062F844B3CDF81C5498F868
:103C2000000000280CBF3C483A48057814BF3B48C8
:103C30003B48067805FB06F8FEF722FF314628468A
:103C4000FEF796FF2D4ADDF81C34A2F58061084688
:103C5000FEF7BDFFFEF727FF4FEA48022748DDF8D1
:103C60001C1415F081FE2348477028E098F80000E6
:103C7000214B2946002814BF26482748027814BF44
:103C800026482748007802FB00F04FEA4002184619
:103C900015F06AFE98F8002018482946002A14BF3B
:103CA0001C4A1D4A127814BF1C4B1D4B1B7802FB8B
:103CB00003F24FEA420215F057FE88F801701B48E4
:103CC0000078032804BF0C4805F008F8DDF810045C
:103CD000002877D0B9F1000F74D1DFF818800546BD
:103CE00098F8000030BBD8F808601EB30748017888
:103CF000074820E07840002024480020244C002081
:103D000024540020EC5400209454002093400020C0
:103D100094400020914000208E40002092400020DE
:103D20008F400020954000205C540020FD40002082
:103D30009040002021E000780844401C4008019099
:103D400002200090FEF79CFEDDE90010FEF719FF4F
:103D5000294632460846FEF774FFFEF7A4FEFE48E9
:103D60000078022804BF304605F0CEF8FA48007803
:103D7000092804BF284605F0C7F85CB32E46F7486B
:103D80000178F74800780D18FEF77AFE681C4008A5
:103D90000221FEF7EDFEF34A3346A2F15801084630
:103DA000FEF715FFFEF77FFE6A003146ED4815F07D
:103DB000DBFD88F80370E8480078032804BFEA4870
:103DC00005F0A2F8FDF7C8FF641C042C1DD2FDF716
:103DD000D4FD8DE6E14EE248E34B32780078294687
:103DE00010444200184615F0BFFDDD483278DD4B27
:103DF0000078294610444200184615F0B5FD88F8B1
:103E00000370D8E701F0E6F972E6FDF7C9FBDDF8CB
:103E10002404FDF774F8DDF82C0438B1DDF828042B
:103E200010B1FDF7AAFD01E0FDF78FFDDDF81804E4
:103E300030B1CE4880F801B080F802A080F803903D
:103E4000DDF818040DF2344DBDE8F08F10B50024F4
:103E5000FDF772FDC54910F0020F0AD04A78002A1A
:103E600008BF012410F0040F03D08A78002A08BF8D
:103E7000012410F0010F18BF10F0100F03D0C87804
:103E8000002808BF01240020002C08BF10BD00201E
:103E90000870BDE810400BE608B50F2101F03CFAB0
:103EA000012804D1FFF7D2FF009001F08BFBAF484F
:103EB000417800291CBFC178002904D080780028EF
:103EC0001CBF012008BD002008BD08B50F2101F06E
:103ED00023FA012804D1FFF7B9FF009001F072FB2B
:103EE000A248417800291CBFC178002904D08078FD
:103EF00000281CBF012008BD002008BD70479B4959
:103F0000002048708870C870704710B54FF4806109
:103F1000974815F024FDBDE810404FF480619548A6
:103F200015F01DBD2DE9F047904F8146089839786E
:103F3000002914BF904991490D78A0EB030805FBB7
:103F400008F603FB05F4FEF79BFD41462846FEF705
:103F50000FFE884809EB440500EB4408A0F5806C8F
:103F60000CEB44012B4642460846FEF730FEFEF7B6
:103F70009AFD72002946404615F0F6FC0120787043
:103F8000BDE8F087002818BF0120784948707047C5
:103F900010B5764C002804BF606010BDDFF8E0C1AA
:103FA00075490B7877490A7801465A4352006046B2
:103FB00015F0DAFC7248606010BD7349002008609B
:103FC00048608860C860086148618861C8610862AB
:103FD00048628862C862086348638863C86308648B
:103FE00048648864C864086548658865C86508666B
:103FF00048668866C866704763487047002818BFDF
:1040000001205A498870704710B55821564815F05C
:10401000A6FCBDE810405821524815F0A0BC00286D
:1040200018BF01205149C870704710B54F4C002887
:1040300004BFA06010BDDFF854C148490B7848495F
:104040000A7801461A445200604615F08DFC4F482C
:10405000A06010BD4549002200284A708A70CA70CD
:1040600018BF0120087023E52DE9F04F87B04FF409
:1040700080613F4815F073FC4FF480613D4815F0B6
:104080006EFC5821384815F06AFC5821354815F067
:1040900066FCFDF751FC0446FDF782FA0020FCF7B0
:1040A0002EFF0690FDF769FC00252E4604F014FB58
:1040B000012875D06846FDF719FE002878D06846BB
:1040C00005F04EF814F0020F1CD02B48DFF8A0B01A
:1040D000DDF8049090F800802A48DA460778FEF769
:1040E000CFFC0120FEF75FFD39464046FEF749FD53
:1040F000524649465846FEF7A4FD0020FEF753FD00
:10410000FEF7D1FC14F0010F18BF14F0100F20D0EF
:104110001248DFF854B04FF0020801781048DA4630
:10412000DDF8109000780844401C4708FEF7A8FC12
:104130000120FEF738FD41463846FEF722FD524683
:1041400049465846FEF77DFD0020FEF72CFDFEF7A0
:10415000AAFCFDF701FE1DE0024100209340002073
:1041600094400020EC54002094540020784000201B
:1041700024480020244C0020914000208E40002044
:104180002450002092400020245400204455002058
:1041900006E00DE06D1C102D03D2FDF7EEFB85E768
:1041A0000126FDF7FDF90698FCF7A9FE1EB136E0E1
:1041B00001F010F87AE714F0020F14D01C481B4BE2
:1041C0004FF0100501781B481A46007848434FF01D
:1041D000000108D032F911C09CFBF5FC23F811C096
:1041E000491C8842F6D814F0010F18BF14F0100FC4
:1041F00015D01248DFF840C04FF010020178104887
:104200006346007809184FF0000008D033F91040D9
:1042100094FBF2F42CF81040401C8142F6D807B011
:104220003046BDE8F08F0120704700002448002090
:1042300091400020924000209454002093400020A0
:1042400094400020FE480078012818BF00207047E5
:104250002DE9FF4FFB4881B0984690F800A0FA483E
:1042600091468B460026057804240E9F05F0F4FE47
:1042700001465FEA0800DFF8C88328D12A1F2046DC
:10428000042AC8BF2A1B09DD31F91030142B01DBC9
:10429000012603E0401C00B29042F5DBB7F1FF3F7E
:1042A00018BF002E13D1B9F1000F10D00198FFF7FD
:1042B0006EFB98F80200052898BF401C08D9281BFF
:1042C00000902346524600215846FFF72BFE00205F
:1042D00088F8020005B0BDE8F08FD94800790128C0
:1042E00018BF002070470021D54881714171704787
:1042F0002DE9F05F00248A46B0F90020B0F90210E1
:1043000005462746A046A3462646A146501A48BF62
:10431000881A03B205EB4A0030F9021C30F9042C6C
:10432000881A48BF501A00B2082BA8BF082807DB1C
:1043300008F03CF9002804BF0123AAF1020002D0D2
:104340000023AAF1010001B218468B422ADC35F99C
:1043500010204245C4BF904600F0FF0998421DDD81
:1043600005EB400C3CF902CCACEB0202D21D0E2A4C
:1043700005D804F1010C0CF0FF0488420ED1A742CD
:104380000BD22746884203D10E2A98BF46B201D9E4
:10439000421E56B2F21B4FFA82FB0024401C80B230
:1043A0008142D4DAAAF10400874205DDCB45DEBFA5
:1043B000B1450020BDE8F09F0120BDE8F09F70B539
:1043C000A34AA24906461478097800EB4402104635
:1043D000FFF78EFF054621463046FFF789FF002292
:1043E0009749002D1CBF00288A7108D18879401C8C
:1043F000C0B288710A2882BF8A71002070BD012076
:1044000070BD2DE9F34F8E498BB000200870DDE9B7
:104410000B1202AB089303AB079304AB069305ABF7
:1044200001938A4B80461B780993894BB1F9006050
:10443000B2F900E01B78354631F9134032F91370B8
:104440000097ADF80C00ADF814000120A4464746D3
:10445000ADF80830ADF81030012B2DDD31F910909A
:10446000B145C8BF4E4632F910A0F245B8BFD64696
:10447000A94504DA4D46DDF80490A9F8000001EBE7
:10448000400931F910A039F902BCBBEB0A0948BF59
:10449000AAEB0B090FFA89F9C14509DDC846D345D6
:1044A000D4BF8146A0F10109DDF81CA0AAF8009054
:1044B000401C00B28342D1DCDDF82490581C09EB8B
:1044C000030B83452CDD31F91030A342C8BF1C46D5
:1044D00032F91090DDF800A0D145B8BFCDF80090BA
:1044E000634502DA9C46069B188001EB400331F9D4
:1044F000109033F902ACBAEB090348BFA9EB0A03E9
:104500001BB2BB4208DD1F46CA45D4BF0346431E4B
:10451000DDF82090A9F80030401C00B28345D2DCC1
:104520004C48A4EB0C0C0168012091F81F319C450C
:10453000C4BFA6EB050C9C4505DD91F81E31BB42BE
:10454000B8BF434521DB089BB1F91C11B3F900301A
:1045500032F91330994218DB069BB3F9003032F977
:1045600013C04B429C4510DBDDF81CC0BCF900C0F9
:1045700032F91CC0614508DB0199B1F9001032F92C
:1045800011108B42D8BF002500DD0546CDB1BDF925
:104590001410BDF91000CDE90001BDF90C30BDF9D2
:1045A0000820DDE90B0100F0B8FC012808BF4FF03E
:1045B000FF350B98FFF703FF002808BF4FF0FF35CA
:1045C00089E01F4A0021917151711E490C9A0F78A0
:1045D0001D4991F8009000210091B2F900C0B2F994
:1045E00002400E4602EB4903BCEB040148BFA4EBBA
:1045F0000C010FFA81FC0121A9F1010B4FF0000819
:10460000BBF1010F1BDD02EB410432F911E0B4F9FB
:1046100002A0BEEB0A0448BFAAEB0E0424B2644514
:10462000C4BFA4464FFA81F8491CC9B25945EADB18
:10463000B8F1000F1CBFA9F10201884510D10BE0B1
:10464000844000208E4000208F40002093400020B6
:104650009440002084410020BCF1190FC8BF0126FE
:10466000B3F90020B3F902C0B2EB0C0148BFACEBC8
:1046700002010AB20121A7F1010A4FF00009BAF1C3
:10468000010F1BDD03EB410C33F91140BCF9028033
:10469000B4EB080C48BFA8EB040C0FFA8CFC944553
:1046A000C4BF62464FFA81F9491CC9B25145E9DBE2
:1046B000B9F1000F1CBFB91E894501D1192A04DCCC
:1046C0000099002908BF002E02D0FE49487002E080
:1046D000FC49002048700DB02846BDE8F08F2DE958
:1046E000F04FDFF8E493064685B0D9F8000090F863
:1046F000241100291CBFB0F8380100280AD0FDF7AA
:1047000062F9D9F8001091F82411B0FBF1F201FB25
:10471000120018B105B00120BDE8F08F02F02CF8AE
:104720000546FFF74EF90446D9F80000002DB0F910
:1047300038110491B0F93A7168D0E4480078102833
:1047400004BF284604F0E0FBE1484FF00008002CCD
:104750000378E04802781FBF002113EB020CD9F860
:104760000000B0F8289109D034F9020B0028B8BF36
:10477000404248454CDC491C8C45F5D8CDE90082C7
:10478000C6460020CDE902235DF820A002AA06EB70
:104790004A0352F820B033F9024B4FF000080121D0
:1047A000C146A446BBF1010F0CD933F9022B944248
:1047B000BCBF144689469445C4BF94468846491CEC
:1047C0008B45F2D8A4EB0C010AB204998A421ADB99
:1047D0000AEB09010AEB080335F8111035F813301C
:1047E000C91A511A09B20029B4BF4B420B46002A1C
:1047F000B8BF5242934206DA0029B8BF4942B942D3
:1048000001DAF04604E0401C0228BDD34FF0010855
:10481000B8F1000F08BF01F0B9FF404605B0BDE890
:10482000F08F2DE9F04F95B0054600201290AA4870
:104830000F460478A948007803900020049007F000
:104840008AFE18B10EF067F801281BD0264600201A
:10485000059080460990079081460B900A906FF072
:104860000B004FF0060A4FF00C0B1390FFF7ACF85B
:10487000089007F070FE002840D00EF04CF8082891
:1048800006D03BE09048006890F83D01461CDEE70A
:104890000398A0428CBF401E601EC2B2039884429F
:1048A00034BF601E401EC1B20420CDE900020023C7
:1048B00006A8029204F0EAFE9DF819109DF81B006C
:1048C000884228BF002319D39DF818009DF81A20AC
:1048D00082420DD301FB0402DDF820C0401CC0B2AF
:1048E0002CF8123027F812309DF81A208242F1D2AB
:1048F000481CC1B29DF81B008842E5D20CA938467D
:1049000005F07DFA00B2584548DDDDE90302A0EB71
:10491000020C944566DD0021002E3AD902FB0410FA
:1049200083B237F913000028B8BF404258452CDD48
:1049300035F91300584508DD0A9B9842C8BF0A9014
:10494000079B5B1C1BB2079306E0139B9842BCBFFE
:1049500008F101030FFA83F8099B5B1C9BB20993D2
:104960000028B4BF43420346DDF82CE09E450CDA34
:104970000028ACBF034643429B4506DA0028B8BF77
:10498000404200B2914605910B90481C81B2B14261
:10499000C4D3501C82B29445BDDC23E0DDE90301A1
:1049A000A0EB010C8C451DDD0020002E16D901FB6B
:1049B000040293B237F91320002AB8BF52425A4575
:1049C00008DD35F91330139A9A42C4BF08F1010289
:1049D0000FFA82F8401C80B2B042E8D3481C81B282
:1049E0008C45E1DC079850EA08001DD007980028A4
:1049F00021D040F33A8107F0AEFD78B10DF08BFF86
:104A0000082824D00DF087FF012820D00DF083FF67
:104A100009281CD00DF07FFF0A2818D029480078FB
:104A2000012814D000F021B926490020C871C870AF
:104A300015B0BDE8F08FB8F1000F40F316812149A1
:104A40000020C871C87015B0401EBDE8F08F1298E4
:104A50000028059809FB040017D035F91010A6F1BD
:104A6000010C059800231FFA8CF2C8B309FB040857
:104A70001FFA88F800297CDD05EB480838F9028C1C
:104A8000C24576DD401E83B278E035F910C0A6F14C
:104A90000108059800231FFA88F228B309FB0401D6
:104AA00089B2BCF1000F20DD35F911B005EB4101F1
:104AB00031F9021CBBEB010B14D40029B8BF4942E9
:104AC00051450EE084400020844100200241002036
:104AD00093400020944000208E4000208F40002012
:104AE0004CE013DA401E83B214E00FDA35F911B04E
:104AF00005EB410131F9021CABEB010BBBF1000FDF
:104B0000F0DC0029B8BF49425145EBDB401E0004F0
:104B1000000CC3D10598404546DA09FB040189B26F
:104B2000BCF1000F0EDD35F911B005EB4101B1F913
:104B30000210BBEB010B30D40029B8BF49425145EC
:104B40002BDB10E00FDA35F911B005EB4101B1F9BB
:104B50000210ABEB010BBBF1000F1EDC0029B8BF4C
:104B60004942514519DB401C80B24045D5DB1BE072
:104B7000FFE7401E0004000C7FF478AF0598604505
:104B800012DA09FB04081FFA88F8002908DD05EB92
:104B90004808B8F90280C24502DD401C82B203E039
:104BA000401C80B26045ECDB059809FB040081B233
:104BB00009FB043083B209FB0420089A1FFA80FC29
:104BC000089832F9132037F8133030F911001344E4
:104BD0001DB2089B37F8111033F91C3037F81CC090
:104BE000014409B29C440FFA8CFCB1EB050848BFA4
:104BF000A5EB0108B1EB0C0548BFACEB010508EBD8
:104C000005010FFA81F8811A48BF111AC21A48BF6C
:104C10001A1A881805B2129878B1A84525DAF7490A
:104C2000C878821E032A9CBF401CC8706CD9002023
:104C3000C87015B0401EBDE8F08F07F08CFC18B1AD
:104C40000DF069FE01280ED0A84507DBB8EB050082
:104C500048BFA5EB0800B0EB4A0F06DA15B04FF0DD
:104C6000FF30BDE8F08FA845F8DB03984FF000094E
:104C7000C01E1FFA80FB0A984FEA540CC8464FF436
:104C8000FA65BE283DDAABF102000CFB00F1099891
:104C9000814236DADDE90302A0EB020E724521DA29
:104CA00000231946002E13D902FB041080B237F9F5
:104CB00010008245BEBF82285B1C9BB24045C8BF26
:104CC0008046A842B8BF0546481C81B2B142EBD32A
:104CD0009C453CBF09F101001FFA80F9501C82B2CB
:104CE0009645DDDC07F037FC58B9B8F1BE0F08DA9D
:104CF000D94506D315F11E0FC2BF032015B0BDE87C
:104D0000F08F0221BD48C17015B00120BDE8F08FC1
:104D10002DE9F05FDFF8E8A280460026DAF800000F
:104D2000374690F8241100291CBFB0F83001002844
:104D30006CD0FCF748FEDAF8001091F82411B0FBB3
:104D4000F1F201FB1200002860D101F083FC5FEA60
:104D500000095BD0AB480078102804BF484603F038
:104D6000BDFFA9484FF0000C444690F800B0A7489A
:104D7000634690F800E0BEF1000F19DD34F9020B34
:104D80000125BBF1010F10DD34F9022B101A01B21D
:104D90000029B8BF494208B2604502DD84461E467C
:104DA0002F466D1C10465D45EEDB5B1C7345E5DB55
:104DB000DAF80020B2F83001844527DB06FB0B70DF
:104DC00008EB400338F8101033F8023CC91A39F8E0
:104DD000103009EB400009B230F8020C181A081A1A
:104DE00000B20028B4BF434203460029B8BF49427D
:104DF0008B420BDA0028B8BF4042B2F83211884229
:104E000004DA01F0C3FC0020BDE8F09F0120BDE8FA
:104E1000F09F70B515460E46044607F0E3FA002CE5
:104E200018BF70BD042818BF052806D07448006854
:104E300090F82400A84288BF70BD3046BDE870409D
:104E400014F0A8BF2DE9F0471E4617460C4605464C
:104E5000DDF82C9007F0C6FA804607F07CFB78B1AD
:104E60000DF059FD082822D00DF055FD01281ED067
:104E70000DF051FD09281AD00DF04DFD0A2816D06D
:104E8000AEB1012C07D15D48007801281CBF002D70
:104E9000B5F1FF3F0BD007F05EFB80B10DF03BFD9D
:104EA000092806D00DF037FD0A2802D007E02C466D
:104EB000F1E707F080FB012808BF4FF0FF34B4F1A1
:104EC000FF3F1CD0002C18BFBDE8F087B8F1040FDD
:104ED00018BFB8F1050F04D0B9F1000F08BFBDE845
:104EE000F087002F1CBF3846FEF770FD002E08BF6C
:104EF000BDE8F0873046BDE8F04714F02BBF002F27
:104F00001CBF3846FEF78AFD002E08BFBDE8F087BB
:104F10003046BDE8F047FEF73ABD2DE9FF4F0E469B
:104F200004463C493A488BB091F800B00078002123
:104F300058440690401ECDE904B0ABF10100CDE924
:104F400002100D9888468A4634F9100008900E9891
:104F50008946474634F91000009101910790FEF709
:104F600014FD054600200146099024484078012898
:104F70000AD00E98814222DC34F91030079AB3EB44
:104F8000A20F18DA02901AE00E98022102280BDB19
:104F90000E98ABF10302824206DB0698C21E0D9802
:104FA0008242A8BF0228E4DA1448012101700FB040
:104FB0000020BDE8F08F401E00B28142DCDD0E987B
:104FC000ABEB010282420BDD34F910C0079BBCEB56
:104FD000A30F01DA039003E0401C00B29042F3DB20
:104FE0000D980BEB010282421ADC34F910C0089BC9
:104FF000BCEBA30F10DA049012E000008440002004
:1050000084410020FD4000208E4000208F40002081
:105010009340002094400020401E00B28242E4DD14
:10502000069A0D98511A81420BDD34F91030089A16
:10503000B3EBA20F01DA059003E0401C00B28842F6
:10504000F3DBDDE9042082422ADA06EB420036F97E
:105050001230B0F90210581A48BFC81A0199084412
:1050600000B2019005EB420035F91210B0F90230A0
:10507000C81A48BF581A0099084400B2009004EBBF
:10508000420034F91230B0F90210581A48BFC81A59
:1050900050440FFA80FA501C02B205988242D4DBC9
:1050A000DDE90201884227DA06EB400136F91030CB
:1050B000B1F90220991A48BFD11A41440FFA81F878
:1050C00005EB400135F91020B1F90230D11A48BF83
:1050D000991A49440FFA81F904EB400134F9102080
:1050E000B1F90230D11A48BF991A39440FB2401CA5
:1050F000039900B28842D7DBDDE90010081A0024CA
:10510000B0EB6A0FDCBFA9EB0800B0EB670F16DC51
:1051100007F04CFA68B9189835F910101048006873
:10512000B0F91C0181420ADC199935F9111081424C
:1051300005DC0998002804BF0A4844710BD00949CE
:105140004879401CC0B24871032881BF4C710120CE
:105150000FB0BDE8F08F00200FB0BDE8F08F000069
:10516000844100208440002010B505F0B7FB05F015
:1051700041FC002010BD0000FE4800787047FD484B
:105180000078022805D005281CBF0020704704F0D5
:105190005AB907F027B9F7490870704710B50446A7
:1051A000062C28BF10BDDFE804F01203070F120B16
:1051B000084600F013FA0AE0084607F008F906E08E
:1051C000084604F035F902E0084606F09FFEE9487B
:1051D000047010BDE84900200968B1F8641011F4AA
:1051E000807F08BF7047FDF7ECB9E34900200968EC
:1051F000B1F8641011F4807F08BF7047FDF7F6B96D
:10520000DD4900200968B1F8641011F4007F08BF7F
:10521000704714F0BFBCD84900200968B1F8641089
:1052200011F4806F08BF704714F0F3BCD14948787F
:1052300000281CBF401E4870704770B5CF490868F1
:10524000D0F8CC00CB4C10F0030F0BD0096840F421
:10525000BE0040F02040C1F8C8006078002804BFBC
:1052600001206070C64800688068C34D10F0020FCE
:10527000296807D1C3480068406910F0010F01D0C8
:10528000607840B1B1F86410002011F4807F18BF3D
:10529000FDF7ACF907E0B1F86410002011F4806F5D
:1052A00018BF14F0B6FCB849084208BF70BD2968A1
:1052B000496E090C617070BD10B572B6FEF7E4FA64
:1052C000BDE81040FEF773B810B54FF42F30FDF76E
:1052D00041FA72B6FEF7D8FABDE81040FEF767B89B
:1052E000A44800697047A348C0687047A149486155
:1052F0007047A048406970479E49886170479D4843
:10530000806970479C48026802F5B073118A508A20
:1053100002F5A072FCF7ACBB2DE9F04FDFF8549218
:1053200095B00E46C9F8100005F03EFAC9F80C0019
:1053300000287DD090F800C089F802C0417889F833
:105340000310837804460CF1010089F8043000F062
:10535000FE0089F80500E27889F80620207989F8AE
:105360000700607989F8080009F10A004FF0000B86
:1053700080F800B080F801B0207889F80900604614
:10538000FCF788FC99F8081099F80700FCF79DFCD9
:105390006946204605F025FA608AD9F8145000289D
:1053A0001CBF6843050B678BD9F81880002F08BF16
:1053B0004FF480574FF4805A002016F0020F18BFA8
:1053C000112016F0040F18BF40F00A0016F0080F65
:1053D00018BF40F0040016F0010F18BF40F0200085
:1053E000616A01EA000600981090049811900898EC
:1053F000129001981390CDF850B010A93046FCF7E8
:10540000B6F916F0020F72D004F0DBFE5FEA000B73
:1054100035D004F0EDFE6843050B59460020FBF73C
:105420009AFD218A00291CBF0020FBF7E2FD00E065
:1054300018E004F0FDFE08FB00F0000B00F5006032
:10544000020A0820012101FA00F3134201D1401E93
:10545000F9D5A0F10408A07B002818BFA0F1010B2A
:1054600017D112E044480068B0F8640010F4807F5F
:1054700018BFFDF7BBF8002015B0BDE8F08FB4F8F9
:105480000CB0BBF1000FC8D1CBE70020FBF72FFE1B
:105490008346E07B002814BF401EFBF757FE0BEB52
:1054A0000801042905DDA8EB010101F1040804212C
:1054B00004E00029BCBFA8EB010800218044B8F13A
:1054C000040F05DDA8F10400C5404FF0040807E013
:1054D000B8F1000F04DAC8F1000085404FF0000871
:1054E0000020FBF71AFE41460020FBF745FE16F0B0
:1054F000010F30D0A18A00291CBF0120FBF72BFD32
:10550000B4F81880B8F1000F07D041460120FBF72E
:1055100070FD41461120FBF76CFD94F81680B8F140
:10552000000F09D0A8F101010120FBF7F6FDA8F159
:1055300001011120FBF7F1FD94F81780B8F1000F7D
:1055400009D0A8F101010120FBF716FEA8F1010125
:105550001120FBF711FEE07A00281CBF0001FBF7C9
:1055600074FC029804F087F8039898B12B4699F8D8
:1055700003200BE08C40002084410020D4D40100A3
:10558000D8D40100CCD401000800030099F802101F
:1055900004F0A8F852463946284604F056F9059812
:1055A000FEF7F6FC069800F0D1FF16F0100F05D0BC
:1055B0000998FEF73AFD0A9801F056F815B0012057
:1055C000BDE8F08F10B5FCF77AF904F05CF80249F9
:1055D0000020C860012010BD8C400020FE494870AA
:1055E0007047FD4840787047FC4810B4FC4A016899
:1055F000914218D14168B1F5887F14D80022D0F8C3
:1056000008C003461146B2EB9C0F24BF10BC704784
:1056100053F82140491C2244B1EB9C0FF8D3002AD7
:1056200004BF10BC7047002010BC7047EB48FDF76A
:1056300091B8E949012048707047E7490020087097
:1056400070472DE9F34FDDB000208A4646904D901B
:105650004C9072B6FCF770F90546FDF7A4FF48B10F
:10566000FEF77BF84D90FEF758F8FEF77CF84C906B
:10567000FEF763F8FCF76CF8FBF790FF5690FCF729
:105680005EF95590FBF78CFFFDF74DFD5490FDF74B
:105690002EFD4FF49350FDF7A6FC62B60022914612
:1056A00030AE46F82290521C062AFAD3CD4F15F0A0
:1056B000020F4FF0010407D0309438684FF4E761CF
:1056C00000F5804014F04BF9C64A15F0010F44F282
:1056D0003870126802EB000510D04FF4E0712846D4
:1056E00014F03DF90120FAF78FFF002818BF32941B
:1056F0001120FAF789FF002818BF3394DFF8E8B2C9
:10570000DFF8D482309868B30020FBF7E3FC009008
:105710009BF800008DF80400B4480078012894BF7D
:10572000B348B44800788DF805000020FBF7A0FDD1
:10573000002818BF4FF0FF3003908DF806A0B8F88E
:105740000400ADF808000020FBF76EFCADF80A007D
:10575000386800F58040059038680690386800F594
:105760000050079031984FF0FF0A48B30020FBF734
:10577000B1FC08909BF800008DF824008DF82540BE
:10578000CDF82C908DF826A0B8F80400ADF82800CC
:105790000020FBF749FCADF82A009DF805003A68A7
:1057A000C0EBC00102EBC10101F580410D919DF8F4
:1057B0000410484302EB40000E9000F500500F909B
:1057C000DFF83492DFF834B2329870B30120FBF77F
:1057D00081FC1090FBF7E5F900280CBF9BF8000056
:1057E00099F800008DF844000120FBF780FC04FAD2
:1057F00000F08DF845000120FBF72CFDC04313900D
:105800008DF846A0B8F80600ADF848000120FBF777
:105810000BFCADF84A001595386842F2204100F5BE
:1058200084601690386808441790339890B311201C
:10583000FBF750FC1890FBF7B4F900280CBF99F85F
:1058400000009BF800008DF864001120FBF74FFC6E
:1058500004FA00F08DF865001120FBF7FBFCC04353
:105860001B908DF866A0B8F80600ADF8680011200E
:10587000FBF7DAFBADF86A00386844F2A871084417
:105880001D90386842F2206100F5C4601E903868AF
:1058900008441F909DF845100220022988BF8DF80A
:1058A00045009DF86510022988BF8DF865004FF00E
:1058B00055301B901390FBF7C7FC57900120FBF766
:1058C000B4FC0120FBF7EAFC5A900020FBF7ADFE88
:1058D00059900020FBF79EFE58900020FBF70FFB2D
:1058E0005B90FCF74AF800204890499037903E9032
:1058F0004698002840F0D18302F0EEFE012800F027
:10590000CC834998802800F2C88340A8FCF7EEF9C0
:10591000002800F0BC8340A803F022FC4898401CFB
:10592000489000F0AB83002048904998401C499073
:10593000002038AA012142F82010401C0628F8D384
:105940003798002808BF369013D0012804BF0020E4
:10595000369000F00181022804BF0020369000F04C
:105960003482032804BF0120469000F0668300F0D3
:1059700094BB369930A850F8210000287CD0369A84
:10598000684600EB42100022479207794279D0F82E
:1059900000803F92B0F9086042694B923E9982695B
:1059A000C068C1F104054A90A9B1002D65DB3F989C
:1059B0004FF0000900287DD905F10800012101FA06
:1059C00000FBE81D01FA00F0509001234A9803FA09
:1059D00009F1084014E01EE0A840002000AF0200DA
:1059E00054435246E8D401009140002090400020EA
:1059F0008F400020924000209340002094400020DF
:105A000018BF0120002151904B98C9EBC9038C4667
:105A100000EBC30A87E03F984FF0000A002849D9FD
:105A200001214A9801FA0AF3034214BF4FF0010E14
:105A30004FF0000E00204B99CAEBCA03844601EBDD
:105A4000C30B30E00121814011EA080F28D0410842
:105A50004FEA19434E915BF82190C1074FEA034387
:105A6000CC0E29FA04F132F9023B89B29B1B0CF1EE
:105A7000010CBEF1000F01E066E060E018BF5B4280
:105A8000002BC8BF41F4805141F400614FF6FF7311
:105A9000A34029EA0303A1400B434E994BF8213060
:105AA000401C1C2801D2BC45CCD33F980AF1010A06
:105AB000824500E03FE0B3D33DE00120884010EA9A
:105AC000080F2DD048084F905AF82000CB07DC0E65
:105AD0004E90E04032F9023BDDF844E19B1B80B27E
:105AE0000CF1010CBEF1000F18BF5B4210F4805F97
:105AF00002D0002B04DA01E0002B01DD20EA0B00CC
:105B0000002DC4BF509B18434FF6FF7E0EFA04FED3
:105B10004E9BA04023EA0E0303434F984AF82030DF
:105B2000491C1C2901D2BC45C7D33F9809F1010982
:105B30008145FFF44AAF002D04BF0120479038A9EA
:105B4000369A479841F822003698401C369006282D
:105B5000FFF40FAF00F071BA369930A850F8210069
:105B6000002800F02A81369A684600EB4210002295
:105B70004E9204794679837905684793B0F9088095
:105B800042694A92C368826950934089479B3E9913
:105B90001840C1F108074F90E9B1002F77DB4FF0B3
:105BA000000A002E72D90120B8404B90781E0121C6
:105BB00001FA00F053900123509803FA0AF10840CB
:105BC00018BF012000213F904A98CAEBCA038C46B7
:105BD00000EBC30B95E04FF0000A002E56D90123CD
:105BE000509803FA0AF1084018BF012000213F90A5
:105BF0004A98CAEBCA038C4600EBC30B40E0012075
:105C00008840284239D0480851905BF82000CB07E3
:105C10004FEAD3694B9020FA09F032F9023BDDF8E4
:105C2000FCE080B2A3EB08030CF1010CBEF1000F05
:105C300018BF5B4210F4805F09D0002B0EDA10F41D
:105C4000706018BFA0F5807040F4805006E0002B13
:105C500004DD10F4706018BFA0F5807040F0800083
:105C60004FF6FF7E4B9B0EFA09FE23EA0E0300FA65
:105C700009F0034351984BF82030491C1C2901D2EC
:105C8000A445BCD30AF1010AB245A8D340E043E0E1
:105C900001208840284231D0480852905BF820000B
:105CA000CB074FEAD369519020FA09F032F9023B51
:105CB000DDF8FCE080B2A3EB08030CF1010CBEF1AF
:105CC000000F18BF5B4210F4805F02D0002B04DA93
:105CD00001E0002B01DD4B9B9843002FC4BF539B79
:105CE00018434FF6FF7E519B0EFA09FE23EA0E037E
:105CF00000FA09F0034352984BF82030491C1C2944
:105D000001D2A445C4D30AF1010AB245FFF453AF4E
:105D1000002FC8BF4E984CDC4FF0000A002E46D929
:105D20004798C0F580703F90479840F4807B4A992F
:105D30000020CAEBCA034FEA174C02464FEA0C4C4C
:105D400001EBC3092DE001218140294226D04FEA11
:105D50005008C10759F82870CB0E27FA03F11FFA33
:105D600081FCDDF8FCE00CF0FF0101EB5E01DDF8E9
:105D70003CE101EA0B01521C714588BF71462CF0D1
:105D8000FF0C4CEA01014FF6FF7C0CFA03FC27EAFA
:105D90000C0C99404CEA010149F82810401C1C28C1
:105DA00001D2A242CFD30AF1010AB245BFD30120EA
:105DB0004E90369A38A941F822003698401C369009
:105DC0000628FFF4C9AE00F038B9369930A850F86B
:105DD0002100002800F02B813E985290684600EB8D
:105DE000411000214E91016850910179479141790C
:105DF0003F918179B0F9089042695192D0E90684C7
:105E00004289C0684F905298C1F5807602EA010736
:105E100010F0010F15D03F984FF0000B00287DD9EE
:105E200001214F9801FA0BF2104018BF01204A904F
:105E30005199CBEBCB02002001EBC20182464B9182
:105E4000E2E00020FBF72AFA054647993F984143D4
:105E5000032000EB410020F003024146204613F0EE
:105E600083FD2846FBF71AFA3F984FF0000B0028F5
:105E700054D901224F9802FA0BF1084018BF0120B3
:105E800000214A905198CBEBCB020D4600EBC20E9D
:105E900050E0012000FA01F25098024247D038F950
:105EA000020B6D1CA0EB09034A98002818BF5B4247
:105EB000480853905EF82000CA074FEAD26A4B9018
:105EC00020FA0AF082B2C2F3032002F0FF0C12F4AF
:105ED000805F02D0002B02DB04E0002B02DDACEB84
:105EE000060401E00CEB0604BC4205DD0F28AEBF42
:105EF0003C460024401C06E0002C04DA0028C6BF03
:105F00003C46401E002402F4805242EA00204FF634
:105F1000FF72204302FA0AF24B9B00E07DE023EA85
:105F2000020200FA0AF0024353984EF82020491C5E
:105F30001C2902D247988542ABD33F980BF1010B45
:105F4000834596D369E0012101FA00F250990A4293
:105F500057D034F9021B4A9AA1EB09010AF1010A50
:105F6000002A18BF494238F9022BA2EB090218BFD8
:105F700052420029B4BF4B420B46002AB8BF5242DE
:105F80009A423ED94B9B4208539253F82220C307B2
:105F90004FEAD36E5C9222FA0EF293B2C3F303225D
:105FA00003F0FF0C13F4805F02D0002902DB04E051
:105FB000002902DD0CEB060501E0ACEB0605BD4255
:105FC00005DD0F2AAEBF3D460025521C06E0002D20
:105FD00004DA002AC6BF3D46521E002503F4805154
:105FE00041EA022129434FF6FF735C9A03FA0EF34C
:105FF0009A4301FA0EF142EA0103539A4B9941F890
:106000002230401C1C2802D247998A459BD33F98D6
:106010000BF1010B8345FFF403AF5298032826BF11
:1060200001204E904E9838A9369A41F822003698B1
:10603000401C36900628FFF4C8AE0123002038A982
:1060400051F82020EAB1401C0628F9D3CBB137988B
:106050001F2811D2401C012101FA00F237905D98EF
:10606000024209D13798401C3790032804D801FA1E
:1060700000F25D980242F5D000203E90469818B19B
:106080000BE03E98401CF8E7FBF777FC34E4FFF7A1
:10609000ACF8469800283FF42FACFBF781FA5798EC
:1060A000FBF7C3F85A98FBF7F9F85998FBF7BDFAD4
:1060B0005898FBF7AFFA5B98FAF721FF569830B182
:1060C000559810B1FBF759FC01E0FBF73EFCFDF7DA
:1060D0006AFA48B14D98002818BFFDF76AFA4C9843
:1060E000002818BFFDF7B1FA5498002818BFFCF734
:1060F000C0FF469800280CBF012000205FB0BDE81B
:10610000F08F2DE9F04FADF2047D4FF00008074607
:106110004646CDF80087E5E0304604F045FB002810
:106120007ED0008900EA070424F0CC0030F47C40E3
:1061300076D00F213046FFF7EFF8002870D0FBF73C
:10614000FBFB0546DDF8000700286AD105F00E00CC
:10615000FBF7FAFA03210020FBF71FF8DDF8000730
:1061600000285ED114F0010F1ED0FF210F20FFF791
:1061700068FACDF80007FBF713FADDF800070028EE
:106180004FD1FFF7B0F88146EA464FF0040B504676
:10619000FBF7E6FD99F92C105246584604F043FBF4
:1061A000DDF8000700283CD114F0060F33D0FDF7CE
:1061B0005BFFCDF80007FBF7F3F9DDF800070028D7
:1061C0002FD114F0020F11D0FDF7FEFB8146FFF72F
:1061D0008AF805235FEA090204D090F92D101846C9
:1061E00004F021FBDDF80007002878D114F0040F3B
:1061F00011D0FDF7E9FB8146FFF775F806235FEA4A
:10620000090204D090F92E10184604F00CFBDDF8BA
:106210000007002863D105F01100FBF795FA01E0B3
:106220005FE04DE0DDF80007002858D114F0100FB2
:106230001DD0FF210F20FFF704FACDF80007FBF770
:10624000AFF9DDF80007D8BBFFF74DF88146EA4605
:106250004FF0080B51460120FBF7C6FD99F93010AD
:106260005246584604F0DFFADDF8000740BB14F050
:10627000600F34D0FDF7F8FECDF80007FBF790F97A
:10628000DDF80007E0B914F0200F13D015F010006E
:1062900018BFFDF77AFB8146FFF725F809235FEA6F
:1062A000090204D090F93110184604F0BCFADDF868
:1062B000000728B914F0400F11D015F0100000E0CD
:1062C0000DE018BFFDF761FB0446FFF70CF80A2349
:1062D000220004D090F93210184604F0A4FAFFF717
:1062E00071F9761C04F05CFAB04204D9DDF80007BD
:1062F00000283FF411AFFE4880F80080DDF8000769
:1063000000280CBF012000200DF2047DBDE8F08FB5
:106310002DE9F04FF648CDB04478FEF72DFF012867
:1063200070D1F4480068B0F93610B0F9340003F0C9
:1063300063FD14F0020F7CD00DF5807BFFF754F95C
:106340000025ED4F30264FF488784FF050094FF07C
:10635000FF3A78B1B0E80E108BE80E10B0E80E10DE
:106360000DF5887B8BE80E100FC80DF5907B8BE840
:106370000F0013E0FF223021584613F0FAFACDE95E
:106380004495CDE94265CDF82CA1CDF828A1CDF8F2
:1063900024A14695CDE9475ACDE94078DFF85CB3B2
:1063A0005846FCF7D7F94598401C459040F2777065
:1063B000FFF7A7FE012803D1FDF735FF012817D00D
:1063C00047980022401C47901F21CDF810910220D1
:1063D00005F0DBFC0DF5807904F0C6F998B1816910
:1063E0004891C169499141694A91C0684B9012E056
:1063F00014F0080F14BFA220A12044904698401C1E
:106400004690E7E74EE0CDF82CA1CDF828A1CDF8D5
:1064100024A1CDF820A1CDE94265CDE94078002145
:10642000D9F808304A46084652F820C0401C61445A
:1064300000E01FE0B0EB930FF6D34D42FF22511C5A
:106440006846C9F80C5013F094FAD9F80820F9E816
:1064500004018DE82700B9E80F0004AD85E80F00BE
:1064600099E80F0008AD85E80F0058466946FCF72B
:10647000DAF910E014F0010F0DD040F22220FFF7FE
:1064800040FE012808BFFDF7CEFE20B901221F21E2
:10649000022005F07AFCFDF732FD01212246084674
:1064A00005F073FC4DB0BDE8F04F02F011B9904912
:1064B000888070478E49C880704770B50126FFF705
:1064C00093F820B10069A12818BFA22801D00020AC
:1064D00070BD002404F064F9002831D9204604F08E
:1064E00063F900281EBF058925F0CC0030F47C40FC
:1064F00021D00F212046FEF70FFFE0B115F0010F6C
:1065000009D0FBF73DFC30B944F480721E21022013
:1065100005F03BFC002615F0100F0AD00120FBF718
:10652000C0FC30B944F480521E21022005F02DFC3D
:106530000026FFF747F8641C04F032F9A042CDD8DA
:10654000304670BD00207047002070472DE9F04FA5
:10655000674EADF20C4D0028B06004BF0DF20C4D3B
:10656000BDE8F08F317811F0020F6BD16449DFF88C
:1065700098810C7863490D78C6F80C800090FDF77F
:1065800081FACDF80404614890F8009060480778DB
:10659000604890F800A0BAF1010F8CBF0DF1040B18
:1065A000C346DDF804040099002809FB07F04FEA10
:1065B00040024BD001A813F0D7F94B4601AA00972F
:1065C0005846DDF8041414F015FEBAF1010F0FD986
:1065D0005946404613F0C4FE404509D0484A01469A
:1065E00040461378474A12785A43520013F0BCF9D8
:1065F0000027F068B846002D18D930F9021B012297
:10660000012C0FD930F902CBACEB010109B2002902
:10661000B8BF49420BB2BB42C8BF1F466146521CBD
:10662000A242EFD308F10108A845E6D3314800683B
:10663000B0F82C01B842C4BF0020F060307840F0C0
:10664000020030700DF20C4DBDE8F08F584613F08B
:106650008BF9BAE72648816800291BBF017811F041
:10666000020F0020C06870472DE9F84F204E002827
:10667000306108BFBDE8F88F317811F0100F18BFF6
:10668000BDE8F88F244D824624484FF00009047875
:1066900023480778FBF750F910F0100F02D0FDF7F0
:1066A00090F9814604EB07084FEA48025146284614
:1066B00013F05AF9B9F1000F09D00220009008F147
:1066C000010043082A464946104614F093FD002075
:1066D000B5F90030A91C0122012F2AD931F902CBCA
:1066E000ACEB03031BB2002BB8BF5B421BB219E03B
:1066F000A8400020844100205443524600AF0200CD
:106700008E4000208F4000209C55002091400020AA
:1067100092400020904000209C590020934000208F
:10672000944000208342C8BF18466346521CBA42B8
:10673000D4D331F9023B0122012C0FD931F902CB1C
:10674000ACEB03031BB2002BB8BF5B421BB283420E
:10675000C8BF18466346521CA242EFD314490968C9
:10676000B1F82E118142C8BF00257561307840F024
:1067700010003070BDE8F88F0E48016900291BBF7A
:10678000017811F0100F002040697047084809494E
:10679000006890F825218878401CC0B28870824239
:1067A00028BF70470020887001210846FEF7F6BC1C
:1067B00084410020A840002070470020704708B5A1
:1067C00003F0070001280AD103F084FF38B101204B
:1067D0008DF80000024669460C2001F059FF0020A8
:1067E00008BD08B503F0070001280AD103F072FFC5
:1067F00038B100208DF80000012269460C2001F01C
:1068000047FF002008BD10B503F00700012808BFAE
:10681000FEF752FD002010BD08B503F00700012867
:106820000AD103F057FF38B103208DF80000012290
:106830006946022001F02CFF002008BD08B503F0D6
:10684000070001280AD103F045FF38B10B208DF86D
:10685000000001226946022001F01AFF002008BD55
:1068600008B503F0070001280AD103F033FF38B15F
:1068700001208DF8000002466946022001F008FF61
:10688000002008BD1FB513F0070F0BD19DF80800BD
:10689000F0280AD003F01EFF20B1012202A908202F
:1068A00001F0F6FE04B0002010BDFEF7BFFEF9E7D0
:1068B0001FB513F0070F07D103F00CFF20B1012221
:1068C00002A9032001F0E4FE04B0002010BD2DE970
:1068D000F84F804603F007000026F84D0A9C0F464B
:1068E000012802D0022806D002E00520A8702E81DF
:1068F0000020BDE8F88FA878052832D12889A04269
:1069000027D2FCF7ACFD4FF0AC098DF80090010ADE
:106910008DF801108DF8020003F0DCFE90B1DFF875
:10692000A0A3DAF8000003F0BAFF58B1DAF80000CB
:1069300090F8200010F0020F04D08DF80190432051
:106940008DF8020028891DF8001088F80010401CFE
:10695000288180B2A04204D12E810120387003200A
:10696000A8700120BDE8F88F2DE9F04103F007027F
:10697000D44C0025D14EDDF818C0012A02D0022ADD
:1069800056D052E0FCF76BFD0521B1700021226862
:106990005554491C0E29FADB2268AC21117022687B
:1069A000010A51702168887003F094FE00283BD0E2
:1069B000C34F386803F073FF002835D0386821686A
:1069C000807CC87038682268017C1171017E11F0EA
:1069D000040F0ED0C18A2268090A51712268817D94
:1069E0009171818A0A0A2168CA712268017D117237
:1069F0000DE0818A2268090A51712268017D917136
:106A0000C18A2268090AD1712268817D11722268C7
:106A1000202151722268022191722168CD72216871
:106A20000D73017E2068417335810020BDE8F0813F
:106A3000B278052A0FD13289624504D223689B5C63
:106A40000370501C30813089604504D135810120AC
:106A500008700320B0700120BDE8F08130B403F06D
:106A60000704984B954D029A4FF0000C012C02D070
:106A7000022C3AD036E00220A8704FF42F30A5F84F
:106A800008C00168880A444211EB842418BF401CE6
:106A9000404201EB8000C01C20F0030041F6E87189
:106AA0000144B0F5283F14D8CC78086864F31F601F
:106AB000854CA0420DD10020002A13D901EB000C17
:106AC0001C689CF804C004F800C0401C8242F5D841
:106AD00008E00020002A05D9196801F800C0401C10
:106AE0008242F9D830BC00207047AC78022C10D11B
:106AF0002C89944204D21B681B5D0370601C2881A2
:106B00002889904205D1A5F808C00120087003200B
:106B1000A87030BC0120704730B403F00704694B03
:106B2000664D029A4FF0000C012C02D0022C51D07D
:106B30004DE00220A8704FF42F30A5F808C001687E
:106B4000880A444211EB842418BF401C404201EBE8
:106B50008000C01C20F0030141F6E8700844B1F544
:106B6000283F2BD8C478016864F31F61564CA142BA
:106B700024D11A68017C11701A68417C51701A681E
:106B8000817C91701A68C17CD1701A68017A117188
:106B90001968427A4A711A68817A91711A68C17AC1
:106BA000D1711A68017D11721A68417D51721A689B
:106BB000817D91721968C07DC87208E00020002AAA
:106BC00005D9196801F800C0401C8242F9D830BCD0
:106BD00000207047AC78022C10D12C89944204D24A
:106BE0001B681B5D0370601C28812889904205D1B9
:106BF000A5F808C0012008700320A87030BC01204F
:106C000070472DE9F04103F0070200262D4D2B4F70
:106C1000069C012A02D0022A3AD036E003F0A4FDF5
:106C200040B3D0E906212B68C0681A70D5F800C0BF
:106C3000130A8CF80130D5F800C0130C120E8CF832
:106C400002302B68DA702A6811712B680A0A5A71AF
:106C50002B680A0C090E9A712A68D171296808728A
:106C60002A68010A51722A68010C9172010E286883
:106C7000C17207E00020002C04D929680E54401C82
:106C80008442FAD80220B8703E810020BDE8F0812D
:106C9000BA78022A0FD13A89A24204D22B689B5CAF
:106CA0000370501C38813889A04204D13E810120F4
:106CB00008700320B8700120BDE8F081C8400020B2
:106CC00084410020ECD4010034CD12AB70B403F049
:106CD0000703F84CF84D039A4FF0000C012B02D03B
:106CE000022B50D04CE00220A8704FF42F30A5F8B2
:106CF00008C001680026880A434211EB832318BFAD
:106D0000401C404201EB8000C01C20F0030101F553
:106D10000050B1F5283F98BF10F0030F27D1E74B83
:106D20000168994204BF0023194620D150F8215030
:106D3000491C2B440729F9D303B1C6B12268017C51
:106D400011702268417C51702168827C8A702268AF
:106D5000C17CD1702268017D11712268417D517121
:106D60002268817D91712168C07DC87108E0002092
:106D7000002A05D9216801F800C0401C8242F9D8D8
:106D800070BC00207047AB78022B10D12B89934246
:106D900004D22468E45C0470581C2881288990423D
:106DA00005D1A5F808C0012008700320A87070BCA8
:106DB000012070472DE9F04103F007040027BE4E83
:106DC000DDF818C0012C05D013F0070F06D0022CF7
:106DD00043D03FE00220B07037813BE00125002422
:106DE00012F0010F1FD04FF42F300168880A434280
:106DF00011EB832318BF401C404201EB8000C01CF4
:106E000020F00303B3F5283F23D800204FF40051AE
:106E1000B0EB930F07D251F804CB401C6444B0EBA5
:106E2000930FF8D3ADB112F0020F0ED003F09CFC1B
:106E300078B182680021B1EB920F06D250F8043B82
:106E4000491C1C44B1EB920FF8D3002D18BF3462DB
:106E500000D137620020BDE8F081B278022A13D158
:106E60003289624508D2C2F10303346ADB0024FA96
:106E700003F30370501C30813089604504D13781A1
:106E8000012008700320B0700120BDE8F08130B40B
:106E900003F007030024DFF820C2029A012B02D07E
:106EA000022B0BD007E005208CF80200ACF808405C
:106EB00020208CF8030030BC002070479CF8023082
:106EC000052B14D1BCF80830934205D29CF803502E
:106ED0000570581CACF80800BCF80800904206D1B8
:106EE000ACF808400120087003208CF8020030BC88
:106EF000012070472DE9F04383B003F007056D4E84
:106F00006D4FDDF828C04FF00008012D0AD013F0B6
:106F1000070F3B461B8903F10104A4B211D0022DD7
:106F200022D01DE001A9684601F007FE0520B870D7
:106F3000316801980870316800984870A7F8088097
:106F40000EE0634502D23068C2543C813889604506
:106F500006D1A7F8088030680178407801F0E4FD98
:106F600003B00020BDE8F083BA78052A0ED163454E
:106F700003D23268D25C02703C813889604505D109
:106F8000A7F80880012008700320B87003B0012022
:106F9000BDE8F08370B503F007000026464C454D70
:106FA000DDF810C0012803D013F0070F06D024E04D
:106FB000268128680670286846701EE02089604592
:106FC00003D22B681A54401C208180B2604514D132
:106FD0003BA00122006826810A702968C2B20978A4
:106FE00091420AD12968C0F307204978814204D12F
:106FF00000221146052001F04BFB002070BD10B5AA
:1070000003F00700012808BF02F076F9002010BD48
:1070100070B503F00704284D012C09D013F0070FB9
:107020002B46D3F820C01B8908D0022C17D014E0BF
:107030000020288104F0A3FE28620EE0002B04BF8C
:107040001002286206D0012B04D14CEA020028620B
:1070500004F08EFE2889401C2881002070BD002B82
:1070600004BF4FEA1C21017005D0012B03D180F829
:1070700000C001200870581C2881012070BD70B527
:10708000064603F007000C4C0D46012808BF0020FF
:107090000DD013F0070F02D0022813D008E020898A
:1070A000002804BF10460FF000FF2089401C2081FB
:1070B000002070BDECD40100C84000205446495364
:1070C00055AC00000FF0EEFE307001202870F0E7A4
:1070D0002DE9F047074603F00700DFF8F4938A46EE
:1070E00001280AD013F0070F4B46DFF8E883FA4D6A
:1070F000DE7808D0022841D03DE00020A9F8080041
:10710000A9F80A0037E0B9F80800002808BF89F894
:1071100003202BD0012804BF1002C9F8200025D07D
:10712000022823D1D9F82000104384B2C9F82000E6
:1071300003F0D0FAD0B1062E18D2DFE806F003062D
:10714000090C1014A8F80E4010E0A8F80C400DE04F
:10715000286884860AE02868A0F80C4106E02868C0
:10716000A0F8504002E02868A0F85240B9F80800A2
:10717000401CA9F808000020BDE8F087B9F80A0013
:1071800002282AD2002403F0A5FAD0B1062E18D284
:10719000DFE806F00306090C1014B8F80E4010E002
:1071A000B8F80C400DE02868848E0AE02868B0F832
:1071B0000C4106E02868B0F8504002E02868B0F8BA
:1071C0005240B9F80A00002804BF200A387004D0E1
:1071D000012802D13C708AF80000B9F80A00401C6E
:1071E000A9F80A000120BDE8F0872DE9F0411C460E
:1071F00015460E46074603F06DFA80B1B54814F007
:10720000070F04D004F0070102290BD007E0002D7E
:107210001ABF90F86C00C008002007F0C9FC0020DD
:10722000BDE8F08190F86C00C00838700120307023
:10723000BDE8F08170B50D46044613F0070F04D089
:1072400003F00700022805D002E010460BF0A9FB6E
:10725000002070BD0BF0A8FB20700120287070BDCD
:1072600070B503F0070200269C4C994DDDF810C064
:10727000012A02D0022A15D012E005F0E0F82168B8
:107280000870FDF779FF2168487002F097FF2168C8
:107290008870FDF774FF2168C8700520A8702E81E2
:1072A000002070BDAA78052A0FD12A89624504D230
:1072B00023689B5C0370501C28812889604504D199
:1072C0002E81012008700320A870012070BD70B5C8
:1072D000064603F007000D4602281CBF002070BDC3
:1072E00001F0F0F9002814BF0124002401F0EDF9A9
:1072F000002814BF0222002222433270012028708D
:1073000070BD70B503F00702744C0025704EDDF8B7
:1073100010C0012A02D0022A42D03FE0FEF764F9F1
:10732000002828D04169FF292CBFFF21C9B222685B
:1073300011708169FF2934BFC9B2FF2122685170E1
:10734000C169FF2934BFC9B2FF2122689170226848
:10735000017CD170226890F820101171018C0A0A0A
:1073600021684A71016A2268090C9171006A2168DA
:10737000000EC87111E02068057020684570206813
:10738000857021685020C8702168FF20087121682D
:107390004871216888712168C8713581002070BDED
:1073A0003289624504D223689B5C0370501C308193
:1073B0003089604502D1358101200870012070BDFF
:1073C0002DE9F04703F007020026414D089C0F46C7
:1073D0008046012A02D0022A06D002E00520A870C9
:1073E0002E810020BDE8F087A87805281AD12889C9
:1073F000DFF8E890002804BFD9F8000012F080FD03
:107400002A89A24206D2D9F80000805C88F80000E0
:10741000501C28812889A04204D12E810120387077
:107420000320A8700120BDE8F08770B503F00702C3
:107430000025274C012A02D0022A11D00EE0052097
:10744000A07000212581084601F077FB4FF6FF71FF
:1074500001EA4000A08101F07CFB6061002070BD6A
:10746000A278052A16D12289B4F80CC0624507D249
:1074700012F0010F1CBFE37803700DD0501C208167
:107480002089604506D12581012008700320A07065
:1074900001F06DFB012070BD666922F00103F35A13
:1074A0001E0A0670E370E9E770B503F007020025D5
:1074B000074C012A02D0022A12D007E00520A07052
:1074C0002581D020A08101F0D5FC6061002070BD35
:1074D000C84000200C83002084410020ECD401002F
:1074E000A278052A16D12289B4F80CC0624507D2C9
:1074F00012F0010F1CBFE37803700DD0501C2081E7
:107500002089604506D12581012008700320A070E4
:1075100001F0BEFC0120DAE7666922F00103F35AAC
:107520001E0A0670E370E9E77FB51C460E46054665
:1075300013F0070F08D103F0CDF828B1012202A9FA
:107540000B2001F0A5F803E004F00700022802D0A8
:1075500004B0002070BD04F072FF2870012030706C
:1075600004B070BD10B503F00702F64C012A02D03A
:10757000022A0DD00AE003F09AFA00216062002886
:107580001ABF4FF40560E081E1812181002010BD28
:107590002289E3899A4207D2D4F824C01CF802C099
:1075A00080F800C0501C20812089984204BF01202F
:1075B0000870012010BD10B4DFF88CC313F0070F62
:1075C00004D003F00702022A2ED02AE0012A01D0BB
:1075D0009AB126E0DCF800004069DCF8001040F0C9
:1075E00001004861DCF80000006BD84920F44050ED
:1075F0000843DCF80010086313E0DCF80000006BBF
:10760000DCF8001020F4405040F4BE0040F0204070
:107610000863DCF800004069DCF8001020F001008D
:10762000486110BC00207047DCF80020526902F06D
:10763000010202700120087010BC704770B50D4641
:10764000044613F0070F04D003F00700022808D007
:1076500005E0002A14BF0120002001F03FFE0020B9
:1076600070BD01F042FE002814BF012200222270EA
:107670000120287070BD70B503F00700B14D1446AD
:10768000012808BF002017D013F0070F15D1288953
:10769000002808BFEA700DD001280BD1E878FBF76D
:1076A00099F9AB49E8780B6800EA04021A630968A3
:1076B000A04348632889401C2881002070BD70B514
:1076C0000E4603F0070C9F4D04990446BCF1010FD0
:1076D00004BF0020288118D013F0070F03D0BCF19D
:1076E000020F14D011E028899A4B02283CBFD3F82E
:1076F00000C00CF80020401C80B22881884204D1D0
:1077000002220F20196800F0C3FF002070BD09F0AD
:1077100041FE2A89002A04BF000A207004D0012AF1
:1077200002D1207001203070501C2881012070BDD2
:1077300070B50E4603F0070C824D04990446BCF167
:10774000010F04BF0020288118D013F0070F03D0C9
:10775000BCF1020F14D011E028897E4B02283CBFF7
:10776000D3F800C00CF80020401C80B22881884269
:1077700004D102221020196800F08AFF002070BD99
:1077800009F01DFE2A89002A04BF000A207004D0D7
:10779000012A02D1207001203070501C2881012064
:1077A00070BD2DE9F04103F0070C664E069D0F46B3
:1077B0000446BCF1010F04BF0020308117D061499D
:1077C00013F0070F0B8903D0BCF1020F12D00EE0AB
:1077D0006049022B3CBF0868C254581C80B23081FB
:1077E000A84204D102220968112000F051FF0020B4
:1077F000BDE8F08113B1012B05D009E009F008FEC6
:10780000000A207004E009F003FE207001203870A7
:107810003089401C30810120BDE8F0812DE9F04124
:1078200003F0070C474E069D0F460446BCF1010FBE
:1078300004BF0020308117D0424913F0070F0B8995
:1078400003D0BCF1020F12D00EE04249022B3CBF24
:107850000868C254581C80B23081A84204D1022268
:107860000968122000F014FF0020BDE8F08113B178
:10787000012B05D009E009F0BFFD000A207004E0EB
:1078800009F0BAFD2070012038703089401C308129
:107890000120BDE8F08110B503F00702294C012A50
:1078A00002D0022A27D024E003F001F900230028A7
:1078B00004BF6362E3811BD000F150016162416843
:1078C000B1F5887F90F820100CD390F8212001EBBF
:1078D000020C01FB02C190F8222090F82300104412
:1078E000084404E090F822000A1801FB0020E0811F
:1078F0002381002010BD2289E3899A4207D2D4F85F
:1079000024C01CF802C080F800C0501C20812089CF
:10791000984204BF01200870012010BD10B513F07B
:10792000070F04D003F00702022A05D002E0104638
:1079300001F02AF9002010BD074A127802700120D8
:10794000087010BDC8400020CCD4010000205FA00A
:10795000C4D40100ECD40100FD40002010B513F0A8
:10796000070F04D003F00702022A05D002E01046F8
:1079700001F0B0FA002010BDF74A12780270012021
:10798000087010BD1FB513F0070F07D102F0A2FE5B
:1079900020B1012202A90A2000F07AFE04B00020E2
:1079A00010BD70B503F00700EC4C1646012804BF6B
:1079B0000020208128D013F0070F25D102F08AFE85
:1079C00010B32089E64D03283CBF29680E54401CA3
:1079D00080B22081032817D1F9F7BAFE2868B0F8E1
:1079E000010046BAF9F7DAFD040018BFF9F7DFFF26
:1079F00028680078002818BF01203146F9F7ABFA53
:107A0000002C18BFF9F7D6FF002070BD70B503F049
:107A10000700D24C1646012804BF002020812DD03B
:107A200013F0070F2AD102F055FE002826D0208936
:107A3000CB4D02283CBF29680E54401C80B22081E7
:107A400002281BD1F9F784FEF9F7A8FD040018BF3E
:107A5000F9F7ADFF2868007800282868417808BF4A
:107A6000002005D00120F9F7C4FA286841781120D8
:107A7000F9F7BFFA002C18BFF9F79CFF002070BD82
:107A80007FB51C460E46054613F0070F08D102F0DD
:107A900021FE28B1012202A9132000F0F9FD03E024
:107AA00004F00700022802D004B0002070BD04F0EA
:107AB00089FC002814BF012200222A7001203070A6
:107AC00004B070BD7FB51C460E46054613F0070F87
:107AD00008D102F0FFFD28B1012202A9142000F014
:107AE000D7FD03E004F00700022802D004B0002014
:107AF00070BD04F058FC28700120307004B070BDD7
:107B000070B503F00700954D049C1646012804BF8C
:107B1000002028811AD013F0070F17D102F0DAFDE8
:107B2000A0B128898E4903283CBF0A681654401C1E
:107B300080B22881A04209D108680968B0F8010024
:107B4000097840BA00B219B1FEF7B4FC002070BD4C
:107B5000FEF7ADFCFAE770B503F007007F4D049C1B
:107B60001646012804BF0020288118D013F0070F03
:107B700015D102F0AFFD90B12889794B03283CBFA5
:107B800019680E54401C80B22881A04207D11868A1
:107B9000B0F8010041BA18680078FAF79DFA0020A1
:107BA00070BD70B503F007026C4CDDF810C0012AFF
:107BB00002D0022A07D004E000202081FBF7FAFA65
:107BC0002062002070BD2289624506D2C2F1030303
:107BD000256ADB0025FA03F30370501C80B2208174
:107BE000604504BF01200870012070BD7FB51C46B0
:107BF0000E46054613F0070F0DD102F06BFD50B194
:107C00009DF8080010F0010F09D0012202A91520EB
:107C100000F03EFD03E004F00700022802D004B0AB
:107C2000002070BD04F06CFC28700120307004B09E
:107C300070BD2DE9F0411C4617460E46054613F06F
:107C4000070F06D102F046FD18B138460AF0A6FE2D
:107C500003E004F00700022802D00020BDE8F08114
:107C60000AF059FE287001203070BDE8F081002034
:107C700070477FB51C460D46064613F0070F08D126
:107C800002F028FD28B1012202A9072000F000FD22
:107C900003E004F00700022802D004B0002070BD09
:107CA000FDF76AFA022808BF00200BD0032808BF9E
:107CB000022007D0042808BF032003D0052814BFE2
:107CC000FF20012030700120287004B070BD2DE924
:107CD000F0411C4617460E46054613F0070F0BD120
:107CE00002F0F8FC40B1384604F034FB00221146A3
:107CF000012000F0CDFC03E004F00700022802D0D0
:107D00000020BDE8F08104F028FB287001203070CD
:107D1000BDE8F08110B5104613F0070F08BF04F05E
:107D200070FB002010BD10B5104613F0070F08BF00
:107D300004F073FB002010BD70B5044603F007008B
:107D40000D4602281CBF002070BD04F073FB20709C
:107D50000120287070BD000002410020C8400020B2
:107D6000ECD4010070B403F007020024FE4BDDF8F0
:107D70000CC0012A05D0022A04BF9A78022A0AD030
:107D80001BE002209870F9481C816FF07F41006869
:107D9000081A186211E01A89624506D21E6AD500D7
:107DA00026FA05F50570501C18811889604504D124
:107DB0001C81012008700320987070BC012070475E
:107DC00013F0070F04BFEA4802700020704710B597
:107DD000944603F00700E449029A012804BF0020FA
:107DE000088112D013F0070F0FD10889E14B9042A0
:107DF0003CBF1C6804F800C0401C80B2088190425F
:107E000003D10E20196800F043FC002010BD2DE9BD
:107E1000F047174603F00702DFF84C834FF0000CE1
:107E2000012A04BFA8F808C0A8F80AC041D013F07E
:107E3000070FCD4BDFF840939D895E6A02D0022A7E
:107E40003AD036E0B8F80800002808BFC8F8247017
:107E50002AD0012804D0841EAC4216D28CB909E085
:107E6000781CA8F80C003044B0F5807F88BFA8F8D3
:107E70000CC019E04FF480724FF42A31BF4811F062
:107E800069FDBC49301909680F54601CA8420BD128
:107E9000BA48C0F8FC904FF42A30FAF75BFCB749B7
:107EA0004FF42A30FAF7BFFCB8F80800401CA8F8D5
:107EB00008000020BDE8F087FF220270C5B1B8F8C5
:107EC0000A20B318521CB3F5807F0FD2AC4C246843
:107ED0004C4518BF80F800C004D103F5283393F84F
:107EE00000380370AA4204BF01200870A8F80A20D5
:107EF0000120BDE8F08770B503F007009A4D049C9F
:107F00001646012804BF0020288115D013F0070F62
:107F100012D102F0DFFB78B128899649A0423CBF1C
:107F20000A681654401C80B22881A04204D122461F
:107F30000968042000F0ACFB002070BD70B50D4650
:107F4000044613F0070F04D003F00700022805D001
:107F500002E0104604F0F2F9002070BD04F0F1F9DF
:107F600020700120287070BD1FB513F0070F04D1D9
:107F7000012202A9162000F08BFB04B0002010BDE6
:107F800003F00701DFF8E0C10098012907D013F0E2
:107F9000070F04BF9CF80210012909D01FE001203F
:107FA0008CF802000020ACF80800CCF81C0014E0AB
:107FB000BCF80810814208D2DCF81C30491C42EAA7
:107FC0000322CCF81C20ACF8081089B2814206D1FB
:107FD00003208CF80200DCF81C00CCF82400002000
:107FE000704703F00701DFF880C10098012907D02E
:107FF00013F0070F04BF9CF80210022909D01FE0FC
:1080000002208CF802000020ACF80800CCF8200018
:1080100016E0BCF80810814208D2DCF82030491C78
:1080200042EA0322CCF82020ACF8081089B2814241
:1080300006D1BCF82000ACF80E0003208CF802003A
:108040000020704770B403F007020025464C012A57
:1080500002D0022A06D002E00220A070258170BC66
:1080600000207047A278022A1CD12289B4F80EC0E1
:1080700062450FD212F0030F04D1636A53F8046B08
:10808000C4E9086394F820300370206A000A206273
:10809000501C20812089604504D125810120087071
:1080A0000320A07070BC0120704770B503F007007A
:1080B00000252D4C0E46012806D013F0070F04BFF3
:1080C000A078022805D02BE00220A070258125622F
:1080D00026E02089E189884219D2216A090A41EA09
:1080E0000262401C2262208110F0030F0FD1606AEF
:1080F000B0F5303F28BF026006D2B0F5005F03D371
:1081000004222049FAF7F4FB606A001D60622089AE
:10811000E189884204D12581012030700320A070BC
:10812000002070BD30B403F007040025DFF838C02C
:10813000012C08BFACF8085046D013F0070F02D04E
:10814000022C44D040E0042A08BF4FF42C3039D030
:1081500024DC002A08BF4FF4005033D0012A08BFA6
:108160004FF42F302ED00FE0C84000207040002088
:1081700015400020ECD40100554E564DF459002016
:10818000FCA80200E8400020022A08BF4FF410308B
:1081900018D0032A08BFFE4814D010E0052A08BFF3
:1081A0004FF42A300ED0FB48102A00680AD0112A5A
:1081B00008BFF94806D0202A08BFB43002D0CCF856
:1081C0001C5001E0CCF81C0030BC00207047BCF80B
:1081D0000820042A07D2C2F10303DCF81C40DB00AC
:1081E00024FA03F30370501C80B2ACF80800042892
:1081F00024BF01200870012030BC704710B503F087
:108200000700012804D1002211460D2000F040FA99
:10821000002010BD2DE9F04703F00704DF4E089F52
:10822000904689460546012C04BF0020308119D0B4
:1082300013F0070F14D102F04DFA88B13089D849F4
:1082400002283CBF0A6802F80080401C80B23081DE
:10825000B84207D102220968062000F019FA01E0AD
:10826000022C02D00020BDE8F087328912B1012A29
:1082700004D009E0FCF780FF287005E0FCF77FFFE1
:108280002870012089F800003089401C30810120CD
:10829000BDE8F08770B503F00700C04D012803D09A
:1082A00013F0070F05D024E00020E8612862E87091
:1082B0001EE0BA492C8991F803C0C8690CEB020191
:1082C000CBB2022C03D242EA0020E86106E0B349B7
:1082D000042C096A04D242EA01202862EB7005E00E
:1082E000052C03D2624508BF01F050F82889401CD4
:1082F0002881002070BD10B503F007011046012948
:1083000005D013F0070F08BF00F080F904E0A3497F
:108310000020C861C8700881002010BD10B510464B
:1083200013F0070F08BF00F071F9002010BD70B501
:10833000072600244FF4103505EB0430FAF73FFA16
:10834000022808BF70BD601CC4B2B442F4D301203F
:1083500070BD30B403F007030024DFF840C2029A76
:10836000012B02D0022B0CD008E005208CF8020073
:10837000ACF808409CF805008CF8030030BC0020E5
:1083800070479CF80230052B14D1BCF8083093429A
:1083900005D29CF803500570581CACF80800BCF8D6
:1083A0000800904206D1ACF8084001200870032074
:1083B0008CF8020030BC012070472DE9F04779A00D
:1083C000DDF820C0006803F007050027734E744CE9
:1083D000012D03D013F0070F06D034E03781206859
:1083E0000770206847702EE03389634503D2256803
:1083F000EA545A1C32813289624524D137814FF0C8
:10840000010881F800802168C2B2097891421AD12E
:108410002168C0F307204978814214D10725002440
:108420004FF4103909EB0430FAF7C9F9022804D0E7
:10843000601CC4B2AC42F5D34046012806BF86F8A2
:108440000580377177710020BDE8F0872DE9F04194
:108450004FF0000C03F00700534E504C65460128C6
:1084600003D013F0070F0CD068E02570E580A561FC
:108470006570002046F82050401CC0B24028F9D357
:108480005CE0207805283CBF401C2070C0B2012869
:1084900008BF100222D0414902280B8A08BF981851
:1084A0001CD024BFE1888B4248D9404F01F0030023
:1084B00001F101083A54A7F128004FF41032806905
:1084C000984502EB002008BF002109D1491CC9B220
:1084D0000429FBD33449FAF7A6F926E020822DE0DF
:1084E000032232EA010120D17A5CCB009A40491C78
:1084F000C9B242EA0C0C0429F6D3617801F03F02BC
:10850000491CC9B246F822C0617040290DD12649E4
:10851000FAF789F96570A069401CA061002046F84F
:108520002050401CC0B24028F9D3E088401C80B2E3
:10853000E080218A884204BF012020710020BDE82C
:10854000F08110B50446002003F032FF002000F057
:1085500065FF21460222BDE81040062000F09AB8CF
:108560002DE9F0411E46174688460546F9F7F0F812
:10857000F9F714F8040018BFF9F719FA012D41466C
:1085800023D00120F8F7FDFE3146012010E0000065
:1085900000AF0200844100200C830020C84000206E
:1085A000ECD4010055AC0000F4590020F04000204C
:1085B000F8F71FFD3846F8F7A2FC002C08BFBDE80D
:1085C000F081BDE8F041F9F7F5B90020F8F7D9FEE0
:1085D00031460020F8F70DFD3846F8F790FCECE73F
:1085E0002DE9F0411F4616460D4601280CBF002418
:1085F00001242046F8F70EFF28802046F8F7EAFC11
:108600003880F8F793FC3080BDE8F08110B5114C4C
:1086100021462389CA78D1F81CC01118C9B2022B8F
:1086200003D240EA0C20E06107E0B3F5817F06D277
:10863000094A12681A4402F8020CE17006E008BF09
:10864000904203D10549604600F0C2FE2089401CDB
:10865000208110BDC8400020ECD40100F459002056
:10866000FE48002202704270827002714271C27034
:10867000DFF8ECC3114601EB410300200CEB430390
:108680001A54401C0628FBD3491C0829F3D3704711
:1086900011F0A8BB2DE9F04115460E460746FAF742
:1086A0009EFC00F008040820FAF794FC2A463146A4
:1086B000384611F097FB05462046FAF787FC284616
:1086C000BDE8F081E54880787047E448407870471D
:1086D000E2490020487070472DE9F84F0024FBF76D
:1086E000EEF8DE4FB878002800F0D381E9464FF06D
:1086F000FF38FAF774FC00F0080A0820FAF76AFC61
:10870000F8780025F0B17879D54900EB4002401C9B
:10871000C0B201EB42017871082828BF7D71F8785A
:10872000401EF87091F801800E780020B8F1000F1B
:1087300006DD0A18927809F80020401C8045F8DC14
:108740000D704D705046FAF741FCB8F1000FC0F2C1
:108750009281F0B20024172880F05081DFE800F009
:1087600083230F19260C32FC3783696F74B4FBFA2C
:10877000F9F8F787969BA000FCF7A6FD13E09DF89B
:1087800000100120FCF70AFD01207870044600F07B
:1087900035B99DF8000002F087F901210320FCF7AC
:1087A000FDFC01207870012400F028B9BDF800001C
:1087B00040BA03F0C9FD02210320FCF7EFFC0120C1
:1087C0007870F0E79DF801109DF800004CE04FF044
:1087D000010987F80190387848BBF9F7A5F830B35C
:1087E0009DF8008087F8009018F0040F18BFFDF77F
:1087F000A9FE18F0020F05D0FF210F20FCF721FF82
:1088000048F0010818F0010F10D0FCF7B5FC022861
:1088100002D103F0E7FD48B1FCF7AEFC052802D118
:1088200000F011FE10B10020FBF714FC3D707D70CC
:10883000E4E09DF80000401E01F056FDB3E79DF80E
:10884000000003F001FEAEE79DF8000000287DD097
:10885000FCF792FC022818BF012403F0CCFD01466E
:108860000220FCF79BFCC9E0FCF798FC9BE79DF815
:108870000000002818BF012003F09AFD9DF80000B9
:10888000002818BF012000F0C9FDB7E09DF80000E6
:1088900003F07FFD87E79DF8000003F0EEFD82E71F
:1088A0009DF8000020B1012872D0022805D0A5E073
:1088B0004FF42F30F9F74EFFA0E001F04EFF0021FA
:1088C0000420FCF76BFC6EE7FAF789FB00F0080860
:1088D0000820FAF77FFBF878002808BFBD704046F3
:1088E000FAF774FB4FF00009C84672B6FAF75BFE60
:1088F00048B1FAF732FF8146FAF70FFFFAF733FF74
:108900008046FAF71AFFF8F723FFF8F747FE834689
:10891000F8F7B6FFFAF707FC5FEA000A18BFFAF7A4
:10892000E6FB4FF49350FAF75EFB62B64D480560E4
:108930004D480168D1F8CC10006841F4BE0141F007
:108940002041C0F8C81011F064F906E032E050E0B0
:1089500049E042E03BE030E01BE0BBF1000F72B6C3
:1089600003D0F8F7F5FEF8F7F0FFFAF71CFE48B170
:10897000B9F1000F18BFFAF71CFEB8F1000F18BFCD
:10898000FAF763FEBAF1000F18BFFAF772FB62B68E
:1089900034E09DF80000012804BF042105203FF4C5
:1089A00063AF022806D0032807BF0021042002215C
:1089B000084659E70021032056E79DF80300009A76
:1089C0001E2160F31F62012003F0DFF916E0BDF8FD
:1089D000000040BA08F0E4FC10E0BDF8000040BA26
:1089E00008F0F3FC0AE0BDF8000040BA08F013FDFF
:1089F00004E0BDF8000040BA08F001FDB4BBE94650
:108A00004FF0FF38FAF7EBFA00F0080A0820FAF7FF
:108A1000E1FAF878F0B17879114900EB4002401C96
:108A2000C0B201EB42017871082828BF7D71F87847
:108A3000401EF87091F801800E780020B8F1000F08
:108A400006DD0A18927809F80020401C8045F8DC01
:108A50000D704D705046FAF7B9FA08E0F440002066
:108A6000F45A002044400020D4D4010003E0B8F1BF
:108A7000000FBFF66EAEFAF7B2FA00F00806082053
:108A8000FAF7A8FAF978002908BFBD703046FAF75E
:108A90009DFAFCF771FB022802D101F0E6FD20B936
:108AA000002C04BF0020BDE8F88F0120BDE8F88F3E
:108AB00002460020022928BF704752B1012A18BF80
:108AC000704701EB810000EBC100F84901EB001099
:108AD0007047C1EBC100F64900EB800001EB40108C
:108AE000704770B5FAF77BFA00F008060820FAF72D
:108AF00071FAF04C00256078302806D24FF40C61F2
:108B0000EB4810F02CFFA570E570A079302806D254
:108B10004FF4D071E54810F022FFE5712572304620
:108B2000BDE87040FAF752BA00FB01F2B2F50C7FD3
:108B30009CBFE04AC2E9030170470028DD4AD268C1
:108B400018BF0260DB480029006918BF0860504365
:108B50007047D848012101710078D54980F00100A3
:108B6000C0EBC00000EB800001EB40107047D14823
:108B70008278002132B1C27822B9027882F00102F3
:108B80000270817001717047CA491E284A78487086
:108B900008BF002003D01F2808BF012000D10870A3
:108BA00010467047C3480078C14980F00100C0EB0F
:108BB000C00000EB800001EB40107047F0B4BD4EE8
:108BC00096F800C0BA4CCCEBCC0CF5680CEB8C0CD6
:108BD00004EB4C1C03FB05F40CEB440C8D4234BF3E
:108BE0002C460C463669F31A934238BF1A460026C3
:108BF000002A9CBFF0BC70470023002C06D930F837
:108C000013702CF813705B1C9C42F8D8761C0CEB8C
:108C1000450C00EB41009642EED3F0BC70472DE9C5
:108C2000F041A44F14468C4601467A7806981D46BA
:108C30008A4218BFBDE8F0810121F970012802D0F5
:108C4000022825D02AE038789949C0EBC000FE6898
:108C500000EB800001EB4011A64234BF32462246B1
:108C60003869A84238BF05460023002D16D90020D8
:108C7000002A06D91CF8007021F81070401C8242AE
:108C8000F8D85B1C01EB4601A444AB42EFD305E0EE
:108C900000232A4621466046FFF790FFBDE8F041D9
:108CA00000F0A7BA002808BF70478249824B4A7873
:108CB00082491B78002A097818BF022A05D0042AA5
:108CC00018BF092A01D0012278E77D4A1278012ACB
:108CD00084BF7C4A1378012200F0A5BA2DE9F04F39
:108CE000744983B00122CA70774A49781778724A6A
:108CF000232992F800A024BF03B0BDE8F08FDFE87D
:108D000001F01223122312232323231223232323CC
:108D1000B6B6232B2B2BB6B6B6B6B6B6B6B6B623BA
:108D2000B6B6B6AAAA0066490978012904D96749E6
:108D30000F78644991F800A000287DD000235246A6
:108D4000394600F070FA8DE0002875D000235246B5
:108D50003946FFF733FF85E0F8F7FAFCF8F71EFC19
:108D60000090002818BFF8F722FE55480078012827
:108D700084BF544890F800A0F8F7DEFD10F0040F0F
:108D800018BF0AF1010A52484A4C006800F58040B9
:108D900001906078A0F1110920784549C0EBC0002E
:108DA00000EB800001EB4015E068B84238BF074691
:108DB0002069504538BF8246F8F74FFE83460020B1
:108DC000F9F709FA0026BAF1000F37DD0024002F69
:108DD0002BDD0199C6EBC60001EBC0081BF90400AE
:108DE0001C2824BF002025F814001BD200EBD071F2
:108DF0004910C00758F82110C00E21FA00F081B2C6
:108E00004FF0FF30B9F1000F1ED0B9F1010F08BFCC
:108E1000C8B205D0B9F1020F04BF0846F9F7E1F96D
:108E200025F81400641CBC42D8DB2248761C564549
:108E3000C06805EB400500E014E0C7DB009800289F
:108E400018BFF8F7B7FD0DE011F4805FC1F3032000
:108E500018BF4042E4E728B100230AF10202394674
:108E6000FFF7ACFE03B0BDE8F04F00F0C2B903B0AD
:108E7000BDE8F08F0F4801214172407980F0010078
:108E800000EB800101EBC000084901EB00107047C6
:108E90000848C279002132B1027A22B9427982F0BF
:108EA00001024271C171417270470000E463002009
:108EB000245B0020FC4000208F40002095400020D3
:108EC00090400020924000208E40002091400020E1
:108ED000E8D40100F6491E288A79887108BF00206D
:108EE00003D01F2808BF012000D1487110467047E9
:108EF000EF48407980F0010000EB800101EBC000F9
:108F0000EC4901EB001070472DE9F04FEA4985B0BC
:108F1000012291F80080E94991F80090E4490A7231
:108F20008979E44C11291CBF1229132939D008B3BF
:108F3000DF49497901EB810202EBC10104EB011227
:108F40000021B9F1000F06D930F8113022F81130A4
:108F5000491C8945F8D80021B8F1000F0AD909EB5E
:108F6000010302EB410C30F81330491CACF86830B7
:108F70008845F4D8FAF733F800F008050820FAF726
:108F800029F8CB4C607A002818BF012100F0B98085
:108F9000E1712846FAF71AF80020207205B0BDE802
:108FA000F08FF8F7D5FBF8F7F9FA0190002818BF11
:108FB000F8F7FDFCBE488179A1F11106817A009194
:108FC000407900EB800101EBC00004EB0015F7F7DE
:108FD000E8FDBB494FF0110B0028096801F58041FD
:108FE00001F5F56701F5E76104BF8A46012004D069
:108FF000BA4658460F464FF0010BF9F7ECF8F8F770
:109000002AFD00240390B9F1000F2FD90098C0EB7E
:10901000C000C0000290039800570828B4BF143065
:1090200008381C2824BF002025F814001BD200EBB0
:10903000D0720299521001EB8201C00751F80A1058
:10904000C00E21FA00F081B24FF0FF30002E4AD05E
:10905000012E08BFC8B204D0022E04BF0846F9F79B
:10906000C0F825F81400641C4C45D4D35846F9F7D1
:10907000B2F8F8F7F2FC00248246B8F1000F2CD9C0
:109080000098A346C0EBC0004FEAC0091AF90400DB
:109090001C2824BF05EB4400A0F868B01AD200EBEE
:1090A000D071491009EB8101C007C959C00E21FADE
:1090B00000F081B24FF0FF30E6B1012E08BFC8B218
:1090C00004D0022E04BF0846F9F78BF805EB4401E3
:1090D000A1F86800641C4445D8D30198002818BF43
:1090E000F8F768FC46E711F4805FC1F3032018BF6E
:1090F0004042B6E711F4805FC1F3032018BF40423D
:10910000E4E7607980F001006071002140E770B50C
:109110000D4667490122CA706A4A497816786A4A38
:10912000212914781EBF2229232970BD002818BFC9
:10913000002D11D0002322463146FFF73FFD631C6E
:10914000012221462846FFF739FD05EB4400A31C08
:1091500001223146FFF732FDBDE8704000F049B80A
:1091600070B5534D0446687890B9A06868B1574906
:109170000978012994BF544955490B785549012272
:10918000097800F050F8687810B96068FFF7A6FD1C
:109190006878112804BF0020FFF7A0FD6878122826
:1091A00004BF0020FFF79AFD6878132804BF002051
:1091B000FFF794FDE06810B1A97921B105E02069BD
:1091C00018B1A97909B9FFF79FFEA879112804BF42
:1091D0000020FFF799FEA879122804BF0020FFF7AE
:1091E00093FEA879132818BF70BD0020BDE8704019
:1091F0008AE670B5F9F7F3FE00F008060820F9F7E3
:10920000E9FE2B4C20790025002801BF207880F052
:1092100001002070A5701CBF0120A0703046F9F736
:10922000D5FEE57070BD2DE9F047994616460D460E
:109230000446F8F717FC5FEA000C1DD01C490878BB
:10924000254AC0EBC000D1F80C8000EB800002EB97
:10925000401009FB08F200EB4200454594BF2F4641
:1092600047460969A1EB0901B14238BF0E4600210A
:10927000002E08D8BDE8F0874B46324629462046E6
:10928000BDE8F0479AE40023002F08D91CF9032019
:1092900034F8122020F813205B1C9F42F6D8491C9A
:1092A00000EB480004EB4504B142ECD3BDE8F08785
:1092B000FC400020E4630020934000209440002004
:1092C000E8D401008E4000208F4000209040002014
:1092D0009240002095400020245B0020284900286F
:1092E00014BF00200120087070472548007800282E
:1092F0000CBF0120002070472148017871B121493D
:109300000A6852690B6842F001025A610A68126BDE
:109310001D4B096822F440521A430A630021416040
:109320008160C160016141617047E5E700B5017886
:10933000C27983B0114341F040018DF800104178AB
:109340008DF80110418809098DF8021081880909FA
:109350008DF80310817801F00F02017962F31F117B
:109360008DF8041081798DF80510017A8DF80610BA
:10937000407A8DF80700684610F053FE03B000BD38
:1093800010410020CCD4010000205FA070B50E4633
:109390000446FBF7F1FE042811D1A4F510708028D3
:1093A0000DD2A019A0F24120802808D22502002465
:1093B000002E04D92846F9F7CDF9012801D0002064
:1093C00070BD641C05F58075B442F3D3012070BDF7
:1093D00070B50D460446FBF7CFFE04280AD1A4F56C
:1093E0001070802806D220022946F9F71CFA0128BD
:1093F00008BF70BD002070BD10B5074CFFF76CF9B9
:10940000012808BF10BD206801F049FA002818BFE4
:10941000FBF7EBFEF2E70000844100208E4A0028B3
:10942000516814BF41F0010021F001005060704705
:10943000894B59680A0E120721F07F4142EA006009
:1094400008435860704784484068C0F30360704721
:1094500081484068000F70477F48006970477E4927
:109460000120086170477C490020086170472DE9A0
:10947000F04F7A4F87B03868B0F90E11B0F90C018F
:1094800000F0BAFC0DF008FD3868D0F8F800C0F321
:109490000340FAF71AFDFBF76FFE052839D1DFF814
:1094A000C091DFF8C0B16C4D4FF000084FF47A7AEC
:1094B0006868C0F303643868A100D0F8F800C5F804
:1094C0000880C84000F00F0621460520C5F80C8032
:1094D00002F0DCFC21460520F6F7FCFE002C7DD0D6
:1094E000022C1DD0042C7AD068680A2C4FEA106137
:1094F00020F07F404FEA017118BF41F0007108432E
:109500006860FFF7E9F8012803D0FBF735FE05286E
:10951000CED0FAF7F3FC07B0BDE8F04F0DF0BEBCBB
:109520000F213046FBF7F8FE0028EAD000F002FEDB
:1095300000F0F6FDFAF78AFC06460020F7F7DFFC9C
:109540004948F8F772F80120F8F764F8F9F76EFD6A
:109550004648F9F719FEF9F7FEFDF9F72BFE3968D1
:10956000B1F80621504300F5FA70B0FBFAF082B270
:109570006A8091F80801287050B1F9F71BFE39682C
:10958000B1F80411484300F5FA70B0FBFAF082B26A
:109590001046F9F793FDD9F8001035488861F8F7BF
:1095A000D7F8F8F7EAF9287838B1401E10F0FF0034
:1095B000287004BF6888F9F781FD6868C0F3036408
:1095C000FFF78AF8012806D06868C0F30360A0425C
:1095D00008BF002E1DD0D9F8000001E034E037E0CC
:1095E000C0F818B0F9F783FDF9F7C1FD0020F9F7CD
:1095F000CBFDF9F728FDF8F7ABF8F7F7D1FF00201E
:10960000F8F713F800F08CFD00F0B5FDFBF7DAFF7A
:1096100077E76846F8F76AFB58B16846FFF7A0FDA0
:10962000684610F00CFE0646F8F796FBFBF7FEFDC9
:10963000C6E73868406E10F0704F02D0FBF7D5FDDA
:10964000BEE7FBF7FAFDBBE7304611F0ABFC58E78D
:10965000304602F0BAFF54E7284100208441002040
:10966000CCD4010000005FA013CF0100D5C20100DF
:1096700007005FA07047002808BF7047802201469E
:10968000014810F067B9704724660020F0B4FB4E23
:10969000DDE905C43668049DB66916F0010F04D0F3
:1096A0001F464B1BCD1BDBB2EDB216F0020F06D0EE
:1096B0006746A2EB040CD21B0CF0FF0CD4B216F0E0
:1096C000040F08D080F800C04A1B84704270C91A89
:1096D000C170F0BC70470370857080F801C0C47021
:1096E000F0BC70472DE9F043164601FB06F90D4624
:1096F000014685B01F464A46E14810F035F9E04C76
:1097000002F029FF4FF0000818B109F004F9012810
:109710001AD002F020FF18B109F0FDF8082842D055
:10972000B7F5805F1CBF0020B9F1000FDCBF05B0AA
:10973000BDE8F0832156794309132154401C81452B
:10974000F8DC05B0BDE8F08300210B46002ECEBF4B
:10975000DFF828C305B0BDE8F0830020002D1CDD34
:10976000DCF8002092F83E919945DCBF92F83F91D9
:109770004B450CDC92F83C918145DCBF92F83D21D1
:10978000904204DC62567A431213625401E004F8FA
:109790000180401C491CA842E2DB5B1CB342DCDBBD
:1097A00005B0BDE8F083AE428CBF701E681EC2B229
:1097B000B54234BF681E701EC1B20420CDE900025C
:1097C000002303A80292FFF761FF00210A46002E42
:1097D000DCBF05B0BDE8F0830020002D19DD9DF849
:1097E0000D309342DCBF9DF80F309A4209DC9DF8A2
:1097F0000C308342DEBF9DF80E30984204F80180A1
:1098000003DD63567B431B136354401C491CA84271
:10981000E5DB521CB242DFDB05B0BDE8F0832DE989
:10982000F0411C4615460E460746F9F729F9214630
:109830002846F9F7A6F90623914A31463846F9F742
:10984000F2FABDE8F041F9F72EB98E4AC2E90301F8
:1098500070472DE9FF4F8C4891B04FF00009067812
:109860008A4890F800A08548006890F8ABE0B0F90D
:10987000A810109190F8AA00CDF80090CDF814909F
:10988000CDF828900F900020CDF80490CDF80890E6
:10989000CDF80C90CDF81090CDF81890CDF81C9024
:1098A000CDF82090CDF82490CDF82C90CDF83090C4
:1098B000CDF8349001460746844602460E90BAF130
:1098C000000F54D94FF0000845464446002E34D9C5
:1098D00002FB064B129830F91B000028B4BFC0F100
:1098E000000B8346DE4524DAA8EB00080FFA88F85F
:1098F0000028ACBF8346C0F1000B5944A8BF844484
:1099000005DA05F10105C0F1000BEDB25F44DDF8A9
:109910004CB0BBF1010F0CD10028B8BF4042DDF8BC
:1099200040B0584505DA3DF812B00BF1010B2DF8A7
:1099300012B0601CC4B2B442CAD3B9F1000F07D14F
:10994000B8F1000F04DD0F98A842D8BF4FF001090D
:10995000B54208BF4FF002093DF91200B0EB5A0FB3
:10996000C4BF01200E90501CC2B25245AAD3454C30
:10997000E06A421A48BF0A1A454DA5FB0165EE0888
:109980000125964287BF1F9A157000221F9E98BF1F
:109990003270B9F1010F2CD0B9F1020F08D21A7848
:1099A000032A01BFC4E90B1C022015B0BDE8F08FEB
:1099B000B9F1020F25D0B9F1010F2AD0002808BF54
:1099C000C4E90B1C0FD01A78002A1CBF1E9A002A6B
:1099D00009D000EB400088423FBFC4E90B1C0320C4
:1099E00015B0BDE8F08F139878B30E9801282DD0EC
:1099F00035E0226B002A1CBFBCF1000FB2EB470F11
:109A0000CDD202201870C4E90B1C15B00320BDE8AC
:109A1000F08F1878022838BF1D70C4E90B1C187825
:109A200002280ED01E9830B1BCF1000F18BFBCEB5D
:109A3000470F06D901E0674503D215B00220BDE803
:109A4000F08F15B00320BDE8F08F08E018780028EB
:109A50001FBFC4E90B1C052015B0BDE8F08FC4E999
:109A60000B1C15B00020BDE8F08F064900200A7AD3
:109A700012F0060F18BF48697047000084410020AB
:109A8000DC6600203C4100208E4000208F400020FA
:109A9000CDCCCCCC0020FE49097A11F0060F18BFBE
:109AA000FC4870472DE9F00700248FB0002B9EBFC3
:109AB0000FB0BDE8F0077047561E4FF000086F4624
:109AC0004FF0000C002E16D904FB02C531F815909A
:109AD00001EB45056D88A9EB05052DB227F81C5053
:109AE0000E351C2D98BF27F81C800CF1010C1FFAB5
:109AF0008CFCB445E8D304FB02FC012A20F81C804E
:109B00004FF0010C13D904FB02C507EB4C0A00EB24
:109B100045093AF802AC39F8029C0CF1010CA9EBAA
:109B20000A091FFA8CFC20F815906245EBD804F165
:109B3000010C1FFA8CF49C42C2D30FB0BDE8F007B1
:109B400070472DE9F04FADF2246D03FB02FA4FF0A0
:109B5000000CE946BAF1000F84BF0026CE4D13D9A0
:109B600031F91C4004F10F071E2F98BF29F81C6023
:109B700004D935F81C70E41B29F81C400CF1010CC9
:109B80000FFA8CFCE245EBD84FF0000C002B59D9B2
:109B90000CFB02F44FF0000B39F9148008F11904A2
:109BA000322C3CD901252C46012A38D90CFB02461F
:109BB00039F9167007F10A0EBEF1140F14D907FB1C
:109BC00008FEBEF1000F0FDD09EB460E3EF902EC78
:109BD000A7EB0E071837302F06D831F916600F366D
:109BE0001E2E84BF6D1CEDB2641C24B2A242DDD8CF
:109BF000142D11D900244FF0010B002A1CD90CFBA5
:109C00000245641C31F8156039F8157024B2F61B52
:109C100020F81560A242F2D8BBF1000F0CD100244D
:109C2000002A09D90CFB0245641C31F8156024B2E6
:109C300020F81560A242F5D80CF1010C0FFA8CFC4B
:109C40006345A5D80021BAF1000F8EBF924A0DF2EC
:109C5000246DBDE8F08F30F8113022F81130491C26
:109C600009B28A45F7D80DF2246DBDE8F08F2DE9D1
:109C7000F04FDFF828C29DB00DF11008BCE8F000ED
:109C80008DE8F000BCE8F00088E8F000BCE8F000E7
:109C90000DF1200888E8F000DCE9004CCDE90C4C1F
:109CA0000026002B9CBF1DB0BDE8F08F0DF1380BD6
:109CB000A2F1010AEE464FF0000C65466746644685
:109CC000BAF1000F31D906FB024831F8189001EBC8
:109CD0004808B8F80280A9EB08080FFA88F82BF8B2
:109CE000148008F10F08B8F11E0F9CBF0CF1010C95
:109CF0001FFA8CFC0BD9AC4507D9BCF1000F04D07E
:109D00006546A4F1010C0CF0FF074FF0000C641C39
:109D1000A4B25445D7D3AC4507D9BCF1000F04D049
:109D20006546A4EB550C0CF0FF07052D23D906FB67
:109D3000027C31F91CC00CF10F041E2C1BD93EF81B
:109D40001740002AA4EB0C0C0FFA8CF54FF0000C16
:109D500011D906FB02C43EF81C8031F81470A8EB40
:109D600005080CF1010CA7EB08071FFA8CFC20F882
:109D700014706245EDD806F1010C1FFA8CF69E4274
:109D800099D31DB0BDE8F08F2DE9F0410746444856
:109D90003F4EDFF8188105784248B269047842489E
:109DA000A0FB02304308A3EB8300831805FB04F0FB
:109DB0004200C3EBC30008EBC0100FF0D5FDB06943
:109DC000421CB261002F08BFBDE8F081032A38BFF2
:109DD000BDE8F081F8F754FE21462846F8F7C8FEA2
:109DE00008F5E06308F5607230493846F8F7EFFE91
:109DF000BDE8F041F8F757BE2549488070472DE986
:109E0000F0412B4E8AB005462148CDE90056A6F117
:109E100070080C46CDF80880B0F9021003913F2974
:109E2000C8BF3F2005DC11F1400FB8BF6FF03F0005
:109E300000DA039000200490F8F722FE1948184F2A
:109E400001783878F8F794FE6846F8F72AFF08900A
:109E5000F8F729FEC4E90068BDF814002081BDF8B8
:109E600016006081BDF81800A081BDF81A00E081DD
:109E7000BDF81C002082BDF81E006082BDF81C00E9
:109E8000BDF81E103A7801FB020035F9100011E010
:109E90003C410020A46600209C680020F0D4010012
:109EA0008E4000208F400020ABAAAAAABC6E0020E2
:109EB000AC7900200AB0BDE8F0812DE9FF4FAE4F2C
:109EC000AE4E83B005002FD0F9F77EFDAC4A97F86F
:109ED00000C03178126800240223B2F91A7100EB35
:109EE0008C02A1F1020826461846B8F1020F77DD70
:109EF000ACF10109C7F10008A1EB030A0021BCF194
:109F0000000F7DD9494577D002EB410B32F8113073
:109F1000BBF802B0A3EB0B031BB24345B4BFA7428F
:109F20001C4669DA012673E002924FF0000930788E
:109F300097F800C04FF0FF364A4640F2E7384FF03E
:109F40000A0E4C4635464F46002837DDACF101037A
:109F5000801ACDE90003CEF1000A0020BCF1000F09
:109F600088BF0FFA87FB1AD931F91020424502DA6F
:109F7000904606B25D46019B98420CD001EB40032F
:109F80005B88D31A1BB25345B8BFCE4502DA52459F
:109F9000B8BF01249946401C80B26045E4D3781CC8
:109FA00087B2009801EB4C01B842D6DC012C05D1F8
:109FB000029858B102F0FAFA012807D07148012C32
:109FC0008680C58018BF00203CD10CE06D48B0F9F8
:109FD00004108E4206BFB0F9060085420024EDE76A
:109FE00016E00DE008E002F0E1FA012805BF06984E
:109FF00000280220012025E0491C89B2614581D357
:10A0000036B9401C80B202EB4C0282453FF776AF76
:10A01000022D18BFB5F1FF3F07D136B101252A4601
:10A020000521032001F0B1FE0BE0012D14BFB5F1B5
:10A03000FF3F002E05D100252A460521032001F00F
:10A04000A4FE68B207B0C0B2BDE8F08F4D48C06949
:10A0500070474C48006A70474B4870474B48704700
:10A06000B0F900300122012908DD30F912C09C4509
:10A07000B8BF6346521C12B28A42F6DB00220029A6
:10A08000D8BF704730F812C0ACEB030C20F812C0F8
:10A09000521C12B29142F5DC704770B4D4B2B0F9E0
:10A0A00000C001230646012C08DD30F91350654538
:10A0B000B8BFAC465B1C1BB2A342F6DB0023002CEE
:10A0C00009DD30F81350A5EB0C0520F813505B1C8C
:10A0D0001BB29C42F5DC00EB4202CBB2B2F900109D
:10A0E0000120012B08DD32F910C08C45B8BF614654
:10A0F000401C00B29842F6DB0020002BDCBF70BC95
:10A10000704732F810C0ACEB010C22F810C0401CB4
:10A1100000B28342F5DC70BC70471A48806A704711
:10A120001848002141628161704716480021416250
:10A1300081617047124810B50068124C008EA06013
:10A14000FBF71AF802280DD0052818BF10BDA0682B
:10A1500010F0060F1ABF20F0060040F0020010BDFC
:10A16000A06010BD02F03EF9002804BFA06820F0F6
:10A170000600F5D010BD70478E4000208F400020B3
:10A18000844100203C4100205C8200201C81002092
:10A19000704708283CBFFE49087070470020FC4902
:10A1A00088604860FB48006890F88100082838BF44
:10A1B000087070470020F64948607047F4480078FE
:10A1C000704770B5F34D0024286890F86C0010F0CB
:10A1D000020F0BD0FAF7D0FF022807D1EC4829680C
:10A1E000007801EB8000B0F8840084B2204670BD96
:10A1F00070B5E84D4FF48054286890F86C0010F06A
:10A20000020F0DD0FAF7B8FF022809D1E0482968FB
:10A21000007801EB8000D0F88400000CC0F3130438
:10A22000204670BDDA488078002818BF01207047AA
:10A230002DE9F041FAF7A0FF022803D102F0D2F88D
:10A24000022803D04FF48050BDE8F0814FF48055D0
:10A250002E4602F0F4F8DFF83C830446CC4FD8F8E1
:10A26000000090F86C1011F0010F0CD0B0F87600DF
:10A27000B9684042814206DC2CB10020641EB860FF
:10A28000204602F0E1F8D8F8001091F86C0010F0C8
:10A29000040F18BF002C0AD0B1F87C00621E904059
:10A2A000B1F87E20824238BF1046C0F31306D1F8C1
:10A2B000A40010F0020F1CBFB978002902D0000CD6
:10A2C000C0F31305B54298BF354602F044F940B1DA
:10A2D00008F021FB012804D14003B5F5005F38BF29
:10A2E00005462846BDE8F0812DE9F04FDFF8A4A22D
:10A2F00087B0DAF8001091F86C2012F0020F0DD040
:10A30000A34A91F88090DFF890B21778002809DB13
:10A31000484503D2B84218BF06463DD107B00020D9
:10A32000BDE8F08F3E464FF0FF38F7F739F9F7F701
:10A33000DFFF0025B9F1000F2ED9DAF80000002464
:10A3400000EB8500B0F8840081B22046F6F703FEEA
:10A35000F7F713FB6846F7F7C9FC00285FD00198B0
:10A3600078B101468D489BF8002000785043421E8A
:10A3700007D331F9020B0028B8BF40420444521EF3
:10A38000F7D2F7F7E9FCF7F70BF9A04584BF2E46A3
:10A39000A0466D1C4D45D0D3B74243D0082E3CBFDC
:10A3A0007B490E70DAF80000B0F8821039B300EB88
:10A3B000870200EB8600B2F88420B0F8840092B2E5
:10A3C00080B2801A484340F30F34F9F7FDFA744B1A
:10A3D0009BF80020002193F800C002FB0CF2002A39
:10A3E0000DD930F81120224420F811209BF80020CC
:10A3F00093F800C0491C02FB0CF28A42F1D84FF0DE
:10A40000806002F0CBF8DAF80000022100EB860051
:10A41000B0F8840082B2032001F0B7FC09E0FAF73B
:10A42000E4FE97E702F00BF803283CBF401C02F063
:10A430000BF8012007B0BDE8F08F5648544900687A
:10A44000B0F87600424288688242BCBF401E8860F5
:10A4500070472DE9F04F8FB093460E4604464FF0FB
:10A46000000A01F0ECFFDFF82C81494F0500D146CE
:10A4700010D1FFF7FAFAD8F80010B1F87810884236
:10A4800008D30120C7F8089001F0DEFF0FB00120CB
:10A49000BDE8F08F002E1FDDB8680028B8BFC7F8F0
:10A4A000089007DBD8F80010B1F874108842BCBFE0
:10A4B000401CB860D8F80000B968B0F87400884251
:10A4C00015DC032D13D2681CC7F8089001F0BCFFFF
:10A4D0000FB00120BDE8F08F09D1D8F80000B0F826
:10A4E00076004142B8688842C4BF401EB860B87860
:10A4F00050B1D8F8000090F8A40010F0040F1EBF6F
:10A5000000200FB0BDE8F08FD8F80000B0F972104D
:10A510008C420EDD796821447960B0F86E00884283
:10A5200010DC4FF0FF30C7F80490FFF7DDFE8246E5
:10A5300008E07868002805DD002CD4BF0121214601
:10A54000401A7860DFF85C9099F8000007283AD14B
:10A55000154859460078420068460FF005FAADF8F4
:10A560000040ADF80260ADF804503889ADF806003F
:10A57000B888ADF80800D8F80000B0F87210ADF84F
:10A580000A10B0F87410ADF80C10B0F86E100DE0B1
:10A5900070410020844100208E4000209240002025
:10A5A0008F400020FD40002095400020ADF80E10A7
:10A5B000B0F87600ADF8100099F80000072804BF45
:10A5C0006846FEF76FFB50460FB0BDE8F08F3E487F
:10A5D00010B50068D0F8A40010F4807F06D0C0F356
:10A5E0000330012101FA00F0F8F7FBF937490020A8
:10A5F0004870887010BD70B5344D0024A8780028CC
:10A6000014BF01260026687828B901F031FF002820
:10A6100008BF002100D001218E4224D00A1C18BF9F
:10A620000122AA7028480068D0F8A43013F0040F63
:10A630000ED021B1C3F30310082808D206E0002190
:10A64000A960696090F88100082800D22870012470
:10A6500013F0020F18BF0124002A18BF01220421A1
:10A66000032001F092FB204670BD174900200968C5
:10A67000D1F8A41011F4807F08BF7047DFF84CC0F8
:10A680009CF80120131C18BF012330B4104CC1F3F7
:10A6900003322468E46B012505FA02F2224011F42A
:10A6A000007F01D00AB102E00AB1002100E00121DF
:10A6B0008B4204BF30BC7047081C18BF01208CF8C7
:10A6C000010030BC97E70000844100207041002069
:10A6D000C4D401005F48007870475E48406800F5C8
:10A6E000407070475B48406800F58070704770B5F7
:10A6F000584C4FF41032584962601068884204BFC9
:10A700005068B0F5087F26D1D2F808C0BCF5D04F0C
:10A7100021D85249D06888420DD0002311461846EE
:10A72000B3EB9C0F07D251F8045B401C6B40B0EBBD
:10A730009C0FF8D37BB9012502F5807000F0AFF8CB
:10A7400048B1606800F5407000F0B8F800281EBFFE
:10A750002570012070BD002070BD3E4900200870AA
:10A760004FF41030F7F7F6BF3A48017841B140682E
:10A77000394A0168914202BF4168B1F5087F7047CC
:10A7800000207047334B5B6803F580731844F8F77B
:10A79000AFB8304B5B6803F540731844F8F7A8B8BE
:10A7A0002C484068006970472A4949680A69824212
:10A7B0009CBF00207047C0EBC00001EBC00000F55B
:10A7C00080607047234A526802EB80035B6A1A4438
:10A7D000234B53F82000FF3020F0FF0000FB012046
:10A7E0007047F0B41B4B00221D4E5C68174683185F
:10A7F00093F928C0BCF1000FB8BF41F822700DDBFF
:10A80000D3B204EB830556F823306D6AFF33254439
:10A8100023F0FF0303FB0C5341F82230521C102A93
:10A82000E5D3F0BC704794460029B8BF7047094A89
:10A83000526802EB80035B6A1344094A52F82020F5
:10A8400002F1FF0020F0FF0001FB00306146F8F745
:10A850004FB800007C41002054465053EFBEADDE9F
:10A8600028D5010010B5FFF742FFA8B1FFF735FF6B
:10A870000146D02216480FF06DF8FFF733FF154C54
:10A8800001464FF4C27220680FF064F82068406DF2
:10A89000BDE8104001F064BDFAF716FDE3E758B1DA
:10A8A0000D4A0168914207D1406820F00F00B0F5D1
:10A8B000087F04BF012070470020704730B1006856
:10A8C00020F00F00602804BF01207047002070476F
:10A8D0000C830020844100204150535210B572B6C1
:10A8E0000120F7F741FEF8F743FDF8F771FD4FF04F
:10A8F000FF30F8F76FFB664880234FF400520021C9
:10A9000052F821C040F821C0491CB1EB930FF7D396
:10A91000F8F772FBF8F78CFFF8F7B6FF0120F8F7AD
:10A9200088FFF7F7E3FE1E20F8F776FFF8F77CFDC7
:10A93000F8F766F8F8F72CFFF8F7D0FDF8F772FB98
:10A94000F8F7D1F8F6F73FFEFFF78CFFF8F7ECFACF
:10A95000F8F7A6FAFDF784FEFBF72EFFFEF7E5FCFD
:10A9600062B64C480CF04CF94B4C2068B0F90C0125
:10A970000CF090FAF5F795FCFFF70AFCF8F7BAFF30
:10A98000FAF757FE2068418A008AFEF7CDF8206862
:10A99000806EC0F34E0161F35F0001F0E9F9FEF74C
:10A9A00069FEFFF7C2FBFAF7ADFC206890F864007F
:10A9B00000F00F00F7F7EAFC206890F8200010F094
:10A9C000010F04BF0021032003D001F014FD014654
:10A9D0000220FAF7E3FB3148006800690C2100F01F
:10A9E0007002012001F0D1F9F5F752FCFFF7EFFDFD
:10A9F000002010BD2A4CFDF76FFE012806D0FAF7A3
:10AA0000BBFB032802D101F084FAC8B1002C05DC9D
:10AA100001F0F1FC01460220FAF7C0FB0126214DAE
:10AA2000FAF7AAFB0446FAF7AAFB01462046F5F717
:10AA300051FC062C29D2DFE804F02818072225153E
:10AA4000641E002CD7DCE3E7287840B9FBF735FD1E
:10AA500028B900221E21022001F097F92E7001F082
:10AA600047FFDDE7FEF703FDDAE7FBF751FCFAF7F6
:10AA700083FB012804BF0220FAF78DFBD0E701F029
:10AA800051FACDE7FEF7B8FCCAE7FAF715FCC7E7BD
:10AA9000008600200C83002084410020CCD40100DB
:10AAA000FF70020088410020FE490870704710B412
:10AAB0004FF42C30FC4A016891421CD14168B1F539
:10AAC000007F18D3836800228446B3F5056F88BFE2
:10AAD0004FF405630021B1EB930F24BF10BC704706
:10AAE0005CF82140491C2244B1EB930FF8D3002AB3
:10AAF00004BF10BC7047002010BC704770B54FF405
:10AB00002C310446E84D0868A84217D14868B0F5D2
:10AB1000007F13D38B6800228C46B3F5056F88BF86
:10AB20004FF405630020B0EB930F08D25CF820606F
:10AB3000401C3244B0EB930FF8D302B1002149B16D
:10AB40008A68B2F5056F88BF4FF4056220460EF0A3
:10AB500001FF1CE0FF224FF4056120460EF009FFC3
:10AB60004FF40070C4E900504FF40560A06000206D
:10AB7000E06084F8200084F8210084F8220084F842
:10AB8000230040F2FF71C4E90410A061E0610120DC
:10AB900070BD70B50021C160D0F808C00B460446F6
:10ABA000BCF5056F88BF4FF4056C0022B2EB9C0F1B
:10ABB00006D254F82250521C2B44B2EB9C0FF8D30F
:10ABC0005942C1604FF42C304FF405622146F7F72B
:10ABD0008FFE012818BF002070BD4FF4007170B4C3
:10ABE00002685160016801F1500291F821C091F8AA
:10ABF00020300CFB03F102EB41010022BCF1000FFD
:10AC000008D900EB4204521CB4F88A4021F8024BE8
:10AC10009445F6D80022002B08D900EB4204521CC0
:10AC2000B4F8CA4021F8024B9342F6D80022BCF196
:10AC3000000F07D900EB4204521CA48821F8024BF4
:10AC40009445F7D80022002B08D900EB4204521C8F
:10AC5000B4F8444021F8024B9342F6D8B0F886206D
:10AC600021F8022BB0F8882021F8022BB0F88420BC
:10AC700021F8022B00240022BCF1000F88BF00EB5A
:10AC8000841508D905EB4206521CB6F80A6121F872
:10AC9000026B9445F6D80022002B88BF00EB841588
:10ACA00008D905EB4206521CB6F8CA6121F8026BBE
:10ACB0009342F6D8641C032CDDD370BC70472DE999
:10ACC000F74F88B000250A992C462E460968049152
:10ACD00001F150030999002984BF7449D1F800801B
:10ACE0001CD90022002888BFB8F9CE700DD933F9DD
:10ACF000021B0029B4BFC1F1000C8C46BC45BCBF8F
:10AD00000D44641C521C8242F1D30999761C8E4278
:10AD1000E7D3002CC8BF95FBF4FA08DC490841438F
:10AD200001EB5002049901EB4201B1F950A000215E
:10AD300002910191049950310091002103910999E8
:10AD400000296CD95949009E069609684FF0000BFE
:10AD50004FF00109B1F9C0E0D1F8B4105F46C1F37A
:10AD60000741D846CDF814B00791002829D9B6F983
:10AD700000204FF0000C06999344634600280DD93B
:10AD8000B1F90040A51A48BF151B7545B8BF0CF1B5
:10AD9000010C01EB49015B1C8342F1D307998C45FF
:10ADA00003D305997F1C1144059108F1010806EBB6
:10ADB00049068045DBD3002FC4BF059991FBF7F10D
:10ADC00001DC9BFBF0F1039B0A9A09B202EB430200
:10ADD0009180364A1268B2F9BA30AAEB030399425D
:10ADE0000ADDB2F9B82052448A4205DD019A1144C5
:10ADF00001910299491C02910099099A01EB4001C5
:10AE000000910399491C039191429BD30299002917
:10AE100005DDDDE9011291FBF2F1019102E05146FD
:10AE2000CDF804A00A9AA2F886100021029103919D
:10AE30000499503100910021049100286FD91B49D9
:10AE4000009F069709684FF0000B099EB1F9BCE01E
:10AE5000D1F8B410D846090ED946CDF814B00791F0
:10AE6000002E32D9B7F900204FF0000C0699934418
:10AE70006346002E0DD9B1F90040A51A48BF151B35
:10AE80007545B8BF0CF1010C01EB40015B1CB342EE
:10AE9000F1D307998C4504D3059908F101081144B1
:10AEA000059105E08941002053454C46844100202E
:10AEB00009F1010907EB4007B145D3D3B8F1000F01
:10AEC000C4BF059991FBF8F101DC9BFBF6F1049BF3
:10AED0000A9A09B202EB4302A2F84410FE4A126831
:10AEE000B2F9BA30AAEB030399420ADDB2F9B820ED
:10AEF00052448A4205DD039A114403910299491C88
:10AF000002910099891C00910499491C0491814285
:10AF100095D302980028C4BF039991FBF0FA0A98D0
:10AF2000A0F888A001980A99504400B200EBD070B4
:10AF30004010A1F884000BB0BDE8F08F2DE9F74F69
:10AF400084B0E5490698DDE904430268054600201F
:10AF500000935063009B0968002B88BF01262AD903
:10AF600005EB4003B3F90430002BB4BFC3F1000C70
:10AF70009C460FFA8CFCB1F9CC70674510DCB5F932
:10AF800086C0BCF1000FB8BFCCF1000C002BB8BFDD
:10AF90005B42ACEB0303B1F9C6C01BB29C4506DAB9
:10AFA000536B06FA00FC43EA0C0CC2F834C0009B59
:10AFB000401C9842D4D391F8CA30002B7BD091F832
:10AFC000CB00834288BF18460023DDF800C0BCF1E7
:10AFD000000F84BF401C019073D94FF0010EDDF8C3
:10AFE00004C04FF000090120CA46BCF1010F4BD943
:10AFF00003FB0445B1F9CEC003950EFB0445029551
:10B0000003FB040602EB4605B5F95080B8F1000FCA
:10B01000B4BFC8F100054546AC4535DB0EFB040660
:10B0200002EB4605B5F95060002EB4BF75423546B7
:10B03000AC4529DB039D2F1A02EB4705B5F94E50AD
:10B04000002DB4BF6F422F46BC451DDB029F3F1A47
:10B0500002EB4707B7F94E70002FB4BFC7F1000BE2
:10B06000BB46E34510DCA6EB0808B1F9C8604645CD
:10B07000B8BF09F101097D1BB542C8BF0AF1010A39
:10B08000401C019DA842BBD3BAEB090048BFA9EB05
:10B090000A0091F8CAC0604507DB0120D2F834C02D
:10B0A00098404CEA000CC2F834C000985B1C834204
:10B0B00007D2002B00E004E018BFA3F1010E8ED1EF
:10B0C0008BE7069C049D4FF0000C20686346002D22
:10B0D000C0F830C088BF012714D904EB4306B6F985
:10B0E0004460002EB8BF764236B2B1F9CC80B0458C
:10B0F00005DD066B07FA03F846EA080606635B1CE3
:10B10000AB42EAD300236E1E1CBFB1464FF0010ACA
:10B1100027D004EB4305B5F94670B5F94460BD1B73
:10B1200048BFF51B2DB2B1F9C480A84516DAB4F9B1
:10B130008850B6EB050848BFA5EB06080FFA88F85B
:10B140007E1B48BFEE1B35B2A845056BAEBF0AFAA1
:10B1500003F65E1C0AFA06F6354305635B1C4B4595
:10B16000D7D3DDE9056500202B68002EC3F83CC06D
:10B1700088BF012714D905EB4004B1F9D880B4F990
:10B180000A41A04503DCB1F9DA80A04505DADC6BA1
:10B1900007FA00F844EA0804DC63401CB042EAD332
:10B1A000069D049E00202B68002EC3F838C088BF7F
:10B1B000012714D905EB4004B1F9D880B4F9CA418C
:10B1C000A04503DCB1F9DA80A04505DA9C6B07FAEB
:10B1D00000F844EA08049C63401CB042EAD3DDE96D
:10B1E000056500202B68002EC3F844C088BF0127E6
:10B1F00014D905EB4004B1F9DC80B4F94A41A0450B
:10B2000003DCB1F9DE80A04505DA5C6C07FA00F8D2
:10B2100044EA08045C64401CB042EAD3069D049EE4
:10B2200000202B68002EC3F840C088BF012714D926
:10B2300005EB4004B1F9DC80B4F90A42A04503DC17
:10B24000B1F9DE80A04505DA1C6C07FA00F844EA83
:10B2500008041C64401CB042EAD3DDE90574049E76
:10B2600020680023002FC0F84CC0C0F848C088BF39
:10B270004FF0010814D904EB4305B1F9E090B5F99A
:10B280008A51A94503DCB1F9E290A94505DAC56CFC
:10B2900008FA03F945EA0905C5645B1CBB42EAD319
:10B2A0000023002E88BF012714D904EB4305B1F910
:10B2B000E080B5F94A52A84503DCB1F9E280A8451F
:10B2C00005DA856C07FA03F845EA080585645B1C16
:10B2D000B342EAD302E0000084410020D2F8388073
:10B2E000106C30EA08031364916C43EA080021EA09
:10B2F00000049464116B44EA000021EA0005156320
:10B3000016D00021049E0846002E88BF01260FD9C2
:10B3100006FA00F73B4218BF491C401C049FB84284
:10B32000F6D3012904D148EA0300C2F840C0906373
:10B3300024B1D06C002808BFC2F848C0D2F83C80C5
:10B34000506C30EA08035364D16C43EA080021EAE8
:10B350000004D464516B44EA000021EA0009C2F8F9
:10B36000349016D00021059E0846002E88BF012685
:10B370000FD906FA00F73B4218BF491C401C059F35
:10B38000B842F6D3012904D148EA0300C2F844C008
:10B39000D06324B1906C002808BFC2F84CC01DB126
:10B3A000106940F010001061B9F1000F03D010696E
:10B3B00040F020001061906B18B1106940F040001F
:10B3C0001061D06B18B1106940F080001061106CF2
:10B3D00018B1106940F480701061506C18B1106998
:10B3E00040F400701061906C18B1106940F48060F6
:10B3F0001061D06C18B1106940F48060106107B022
:10B400000120BDE8F08F2DE9F04FB1B016460D4692
:10B410000446F6F7C5F8F5F7C4FB01004FF011003C
:10B420001DBF029001200390012108BFCDE9021049
:10B43000CDE91A54F6F70FFB00220DF1100B002D89
:10B4400009D98356082BB4BF1433083B0BF80230DC
:10B45000521CAA42F5D3F6F700FB0021002C07D9B5
:10B46000425C0BEB0103491C83F820208C42F7D887
:10B47000F6F762FA2D900120F6F766F9FE4800789B
:10B4800010F0200F4AD0F5F78CFBFC4944F2A8726B
:10B4900044F23873096800280A4419440CBFCDE906
:10B4A0000012CDE9002106F18A001C9040301D9069
:10B4B000FF210F20FAF7C5F8F6F772F80025E946E4
:10B4C0000DF1700A1AA850F8257002A850F825004E
:10B4D000F6F781FE0024002F88BF0BEB45181AD920
:10B4E00018F904001C2828BF00200DD259F8251097
:10B4F00000EBD072521051F82210C007C00E21FA92
:10B5000000F080B2F6F76DFE5AF8251021F814000D
:10B51000641CBC42E4D36D1C022DD3D3D648007802
:10B5200010F0010F00F0A181F5F73BFBD349002893
:10B53000096801F5C46201F584610CBFCDE91C12F4
:10B54000CDE91C210120F5F7F7FC30900120F5F73B
:10B5500090FF2E900298F5F73DFD28900398F5F79F
:10B5600039FD279024A8009022AB20AA1EA902989A
:10B57000F5F7DAFE25A8009023AB21AA1FA90398AE
:10B58000F5F7D2FE0298F5F745FF26900298F5F7F9
:10B5900041FFBB4D01902868B0F8E4100120F5F799
:10B5A000DAFC00210120F5F74FFF286890F8E6103B
:10B5B0000298F5F71EFD286890F8E6100398F5F755
:10B5C00018FD2868B0F8E8100298F5F7DAFE286848
:10B5D000B0F8E8100398F5F7D4FE0020F5F75BFF0C
:10B5E0002F902868B0F8EC10009190F8EB3090F8AC
:10B5F000EA2001210298F5F764FE2868B0F8EC1003
:10B60000009190F8EB3090F8EA2001210398F5F7CB
:10B6100058FE0020F5F73FFF14ACF6F7AEF9FDF742
:10B620005BF8012805D02046F6F760FB002800F003
:10B630002981F5F7B5FF179900221AAC002054F8BC
:10B6400022C0BCF1000F84BF02EB420306EB831360
:10B6500008D931F8027B03EB4008401CA8F80A71B6
:10B660008445F6D8521C022AE8D30298F4F7CCFF9E
:10B670002A900398F4F7C8FF29900298F5F72AFD5D
:10B680002C900398F5F726FD7D4D2B902868B0F897
:10B69000EE10009190F8EB3090F8EA20012102982A
:10B6A000F5F70FFE2868B0F8EE10009190F8EB3037
:10B6B00090F8EA2001210398F5F703FE0025002009
:10B6C000F5F7E9FE00210298F4F789FF00210398BD
:10B6D000F4F785FF0DF10808012158F82500F4F76B
:10B6E0007EFF1AA8002450F825701CA8002F50F8DF
:10B6F00025A032D904A800EB451905EB450006EB5F
:10B700008018002119F804B00846F5F7DDFE012085
:10B7100000FA0BF102A88B4650F82500F5F7CDFC96
:10B720006FEA0B010920F5F7CFFE0DF1500BF6F78C
:10B7300024F9FCF7D1FF012804D05846F6F7D6FAD1
:10B7400000287CD0F5F72CFFBAF8000008EB440184
:10B75000641CA1F84A01BC42D3D300210846F5F786
:10B76000B3FE6D1C022DAAD32A990298F4F737FF75
:10B7700029990398F4F733FF2C990298F5F79DFC6B
:10B780002B990398F5F799FC3D4C2068B0F8F01020
:10B79000009190F8EB3090F8EA2001210298F5F73B
:10B7A00090FD2068B0F8F010009190F8EB3090F820
:10B7B000EA2001210398F5F784FD0120F5F76BFEDF
:10B7C00014ACF6F7DAF8FCF787FF012804D020461E
:10B7D000F6F78CFA00285BD0F5F7E2FE1799002205
:10B7E0001AAC002054F822C0BCF1000F84BF02EB59
:10B7F000420306EB831308D931F8025B03EB4007E1
:10B80000401CA7F88A518445F6D8521C022AE8D376
:10B8100001203099F5F79FFB01202E99F5F714FED2
:10B8200028990298F5F7E5FB27990398F5F7E1FBCE
:10B8300024980090229B209A1E99029800E024E010
:10B84000F5F73FFD25980090239B219A1F990398B7
:10B85000F5F737FD26990298F5F793FD01990398BE
:10B86000F5F78FFD2F98F5F716FE2D98F5F76CFF7D
:10B8700031B0BDE8F08F000089410020E8D401001C
:10B8800084410020F9F7B1FCC9E6F9F7AEFC50E7B6
:10B89000F9F7ABFC97E72DE9F04FADF6F42DFF2259
:10B8A0004FF4056102A80EF064F8FF224FF42371F3
:10B8B0000DF658000EF05DF802A8CDF85808FFF715
:10B8C0001DF9FE4D4FF0000495F800A01AF0800F0E
:10B8D00073D0DDF858080DF6580290F820C090F8A3
:10B8E0002110503001FB0CF300EB43000023002932
:10B8F00008D902EB430730F8026B5B1CA7F88A609B
:10B900009942F6D80023BCF1000F08D902EB430797
:10B9100030F8026B5B1CA7F8CA609C45F6D8002380
:10B92000002907D902EB430730F8026B5B1CBE808D
:10B930009942F7D80023BCF1000F08D902EB430766
:10B9400030F8026B5B1CA7F844609C45F6D830F8D1
:10B95000023BA2F8863030F8023BA2F8883030F87B
:10B96000023BA2F8843000260023002988BF02EBA6
:10B97000861708D907EB430930F8028B5B1CA9F83E
:10B980000A819942F6D80023BCF1000F88BF02EB70
:10B99000861708D907EB430930F8028B5B1CA9F81E
:10B9A000CA819C45F6D8761C032EDDD36046FFF78E
:10B9B00086F94FF0010887E0FFE7C1480DF6580609
:10B9C0004FF00008006890F8B40000F00F0700F096
:10B9D000A6FA012809D00F213846F9F79DFC012865
:10B9E00008D0002000F098FA6EE000210846F5F734
:10B9F000BEFE02E0012000F08FFAB24890F80090FD
:10BA0000B1480778002F18BFB9F1000F5AD0DDF800
:10BA100058084FF4006180F8209080F8217080F879
:10BA2000224080F8234050300DF099FFF6F707FCD4
:10BA30001AF0210F04D0324639464846FFF7E3FC9E
:10BA40001AF0030F3CD0BA460196F5F775FF06468B
:10BA50000220F5F779FEFF210F20F9F7F2FDF5F747
:10BA60009FFD3046F5F770FEDDF85888002108F19B
:10BA70005000009053464A460846F6F7E8FA002080
:10BA8000F6F7A9FB00260AFB09FBBBF1000F0AD958
:10BA900008EB4607B7F85000F6F7A3FB761CA7F8AB
:10BAA0005000B345F4D8894800781D2804BF08F138
:10BAB0005000FDF713F951464846019AFFF7FFF889
:10BAC0004FF00108F5F7FBFE9DF828009DF82910BE
:10BAD000CDF8E40AB8F1000F19BF002800290DF6CF
:10BAE000F42DBDE8F08F0020069074480078CDF862
:10BAF000EC0A10F0020F00F0D3800020DDF8586847
:10BB000047F6FF7ADDF8E42A06F150086FEA0A09E1
:10BB1000009005460190002947D969480068CDF892
:10BB2000E80A05FB02F0012438F910304FF0000B51
:10BB30001F46BC46012A17D905FB024038F9100000
:10BB40006045C8BF84469842B8BF0346B0EB070EB5
:10BB500048BFA7EB000E0FFA8EF75F45C8BFBB4684
:10BB60000746641C9442E7D3CC45C8BFE146534521
:10BB7000B8BF9A46BCEB030048BFA3EB0C0000B271
:10BB8000DDF8E83AB3F9C030834205DBDDF8E80AB6
:10BB9000B0F9C200834505DD012000FA05F30198E4
:10BBA000184301906D1C8D42BBD30025002A45D956
:10BBB00043480068CDF8E80A38F9153001241F46DB
:10BBC000BC464FF0000B012917D904FB025038F98D
:10BBD00010006045C8BF84469842B8BF0346B0EB2A
:10BBE000070E48BFA7EB000E0FFA8EF75F45C8BFE0
:10BBF000BB460746641C8C42E7D3CC45C8BFE14630
:10BC00005345B8BF9A46BCEB030048BFA3EB0C00FA
:10BC100000B2DDF8E83AB3F9BC30834205DBDDF869
:10BC2000E80AB0F9BE00834505DD012000FA05F3FE
:10BC30000098184300906D1C9542BDD30198F062A6
:10BC400018B1306940F0080030610098B06218B156
:10BC5000306940F004003061A6F824A0A6F82690D0
:10BC6000BDF9DC28B9EB020048BFA2EB0900144A79
:10BC70001368B3F9B820904203DD306940F0020048
:10BC80003061BDF9DC28B2EB0A0048BFAAEB020024
:10BC9000B3F9BA20904203DD306940F00100306111
:10BCA000DDF8EC0A054C10F0010F05D00DF6580236
:10BCB000DDF8E40AFFF742F9207809E08941002025
:10BCC000844100208E4000208F400020FD40002055
:10BCD00010F0400F2FD10798401C079006980028BD
:10BCE00014BF0998089800F1010014BF099008904A
:10BCF0000DF65800FEF771FF0020024605900498EB
:10BD000002A98C46B0F5056F94BF03464FF4056356
:10BD10000020B0EB930F06D25CF82040401C224478
:10BD2000B0EB930FF8D35042C8604FF42C304FF46F
:10BD30000562F6F7DDFD0A208DF800009DF8180079
:10BD40008DF801009DF819008DF802009DF81A0089
:10BD50008DF803009DF81B008DF80400052269464C
:10BD6000012000F039F80DF6F42DBDE8F08F000049
:10BD70006549C2B2C0F307200A8048807047624814
:10BD80004188008861F31F207047DFF87CC10123E0
:10BD90008340BCF800C013EA0C0F08BF704700B521
:10BDA00083B000F03F008DF800008DF801108DF891
:10BDB0000220100A8DF80300100C8DF80400100EFC
:10BDC0008DF8050000208DF806008DF80700684604
:10BDD0000EF03CF803B000BDDFF82CC10123834016
:10BDE000BCF800C013EA0C0F08BF704710B582B052
:10BDF00000F03F008DF80000072A88BF07220020CE
:10BE00006B46002A09D911F800C01C18401C84F8A0
:10BE100001C09042F7D3072805D200211A18401C10
:10BE200051700728FAD318460EF010F802B010BD72
:10BE3000DFF8D4C001238340BCF802C013EA0C0F22
:10BE400008BF704710B582B000F03F0040F080009E
:10BE50008DF80000072A88BF072200206B46002AC1
:10BE600009D911F800C01C18401C84F801C0904288
:10BE7000F7D3072805D200211A18401C5170072853
:10BE8000FAD318460DF0E2FF02B010BD70B51E4D9A
:10BE900082B040EA0122AC880228234602D005285D
:10BEA00005D009E0002918BF022905D103E00029C7
:10BEB00018BF022900D11446A34204BF02B070BDCE
:10BEC0000126F7F777F9297844EA004011F0080FC6
:10BED00017D003218DF800108DF801608DF8020055
:10BEE000010A8DF80310010C8DF80410000E8DF876
:10BEF000050000208DF806008DF8070068460DF05B
:10BF0000A5FFAC8002B070BD8A410020FE490870D8
:10BF10007047FD4800787047FB4948707047FA4801
:10BF2000407870472DE9F04FF74891B000214170FB
:10BF3000FCF7D2FB012806D1F9F71EF903281CBF34
:10BF400011B0BDE8F08FF04C207810F0010F07D051
:10BF5000FFF7A1FC207820F001002070FCF7B8FB6F
:10BF6000207810F0020F00F0DF81E848E649006811
:10BF70004978B0F858000229C0F303200DD0E24CF4
:10BF8000A17801F00F01F9F7C7F901280CBF0220D1
:10BF90000020607005D000F0AEB900210846F5F72A
:10BFA000E6FBF5F7C9FCDFF860A30E909AF80200F3
:10BFB00010F0100F18BFF6F73FF9FF210F20F9F727
:10BFC00040FBD34800780490D24800780590D248CE
:10BFD00090F800B0D14800780D90059800281CBF5B
:10BFE0000498002813D0FEF7A5F8FEF799F8002072
:10BFF000F7F7CEFF0020F8F718F89AF8020010F0D3
:10C00000100F0CD00120F8F725F801200BE00D9857
:10C01000002818BFBBF1000FE5D100F06CB900207B
:10C02000F8F718F80020F8F715F80120F4F767FF83
:10C03000F5F78BFC1E20FCF7A7FD00210846FCF756
:10C0400037FD814601210020FCF732FDDDE90412B5
:10C050008046002001FB02F7002F84BFB0494A0C44
:10C0600006D929F8101028F81020401C8742F8D86B
:10C070001E20FCF72FFF00210120FCF719FD0546CB
:10C0800001210846FCF714FD04460D9900201BEB26
:10C0900001061CBFA2494A0C06D025F8101024F84E
:10C0A0001020401C8642F8D800200C9096488088CA
:10C0B00000287DD9701C40080F90FCF70DFB01286B
:10C0C00076D006A8F5F712FE002872D00798E8B3DC
:10C0D0008D48807810F0100F08D0DDF81CA0FDF717
:10C0E000B5FF51460FF054F8824614E000200023BB
:10C0F00000900190029003901A46194607980EF09E
:10C1000073F982468048807810F0200F03D0FDF745
:10C110009DFF824609E0F7F757FC059A00925246C8
:10C1200001461046049B0FF065F8BAF1000F1CBFE2
:10C130000020002F12D93AF9101039F910208A4244
:10C14000B8BF29F8101038F9102000E006E08A4244
:10C15000C8BF28F81010401C8742ECD80E9810F089
:10C16000010F1CBF0A98002831D06748807810F072
:10C17000200F09D000210A980EF0E6FBFDF76CFFB6
:10C180005FEA000A23D00BE0DDF828A0F7F7FDFBFB
:10C19000022200925246014610460F9B0FF02AF8E9
:10C1A0000020002E13D93AF9101035F9102001E0C3
:10C1B0001BE012E08A42B8BF25F8101034F91020B5
:10C1C0008A42C8BF24F81010401C8642EBD8F5F70D
:10C1D000C3FD0C98401C0C9002E0F9F706F80C988F
:10C1E000494989888842FFF468AFF5F7D9F9FDF726
:10C1F00097FFFDF7C0FF44490C988988884274D3A3
:10C200000E9810F0020F26D000224FF6FF73104652
:10C21000002F0ED939F9101038F910C0A1EB0C011C
:10C220009142C8BF0A469942B8BF0B46401C87429C
:10C23000F0D80B208DF80000100A8DF801008DF861
:10C240000220180A8DF803008DF804300522694693
:10C250000120FFF7C1FD0E9810F0010F45D000221C
:10C260004FF6FF731046002E0ED935F9101034F931
:10C2700010C0A1EB0C019142C8BF0A469942B8BF59
:10C280000B46401C8642F0D80020BBF1000F84BF53
:10C290000D9901EB0B0616D9A6EB000C05EB4C0132
:10C2A00004EB4C0C31F8027CABEB000105EB4108D0
:10C2B00004EB4101A8F866703CF802CC401CA1F8E0
:10C2C00066C08345E8D80D208DF80000100A8DF86F
:10C2D00001008DF80220180A8DF803008DF8043053
:10C2E000052269460120FFF777FD3020FCF74CFC62
:10C2F0003020FCF7EFFDF5F7E2FA0348017821F072
:10C30000020101700EE000009041002084410020F5
:10C310008E4000208F400020934000209440002059
:10C320000080FFFFFCF7D4F9F8F726FF03281CBFB5
:10C3300011B0BDE8F08FF8F758FFF9E504498870AF
:10C340007047034880787047014988807047000033
:10C3500090410020FB4908707047FA480078704708
:10C36000F84982B26FF30F00C1E904027047F54843
:10C3700080787047F34A0028516914BF41F00200E9
:10C3800021F0020050617047EE48007DC0F340008C
:10C390007047EC4AF02303EA0010516921F0F001E4
:10C3A000084350617047E748007DC0F303107047B1
:10C3B000E44A0028516914BF41F0010021F0010056
:10C3C00050617047DF48007D00F001007047DD4B91
:10C3D00019690A0E120721F07F4142EA0060084302
:10C3E00018617047D7480069C0F303607047D548AB
:10C3F0000069000F7047D4480068406DC0F30360C7
:10C400007047012101FA00F04FF47F0101EA004179
:10C41000CC480269114301617047012101FA00F023
:10C420004FF47F0101EA0041C648026922EA010196
:10C4300001617047C3480069C0F307407047C148B5
:10C44000008AC0F303307047BE4910B50246086940
:10C450004FF47043C0F3033420F4704003EA023316
:10C460001843086103210846FFF78FFC204610BDE2
:10C47000B448808AC0F38020704770B5B14E04463E
:10C48000C0F380007569C5F30021884210D0F7F72A
:10C4900036FD14F0040F05D006F03DFA012808BF60
:10C4A000002003D0A94890F86C00C00802F080FB7F
:10C4B00014F0010F14BF45F0400025F0400014F0C7
:10C4C000040F14BF40F4807020F4807014F0080F43
:10C4D00014BF40F4007020F4007014F0100F14BF6B
:10C4E00040F4806020F4806014F0200F14BF40F40A
:10C4F000006020F400607061BDE87040FEF77BB81A
:10C5000090484169002011F0400F18BF012011F040
:10C51000200F18BF40F0020011F4807F18BF40F0D8
:10C52000040011F4007F18BF40F0080011F4806F80
:10C5300018BF40F0100011F4006F18BF40F0200049
:10C5400070478048007DC0F3801070477D48007DB3
:10C55000C0F3401070477B48808AC0F300207047CA
:10C560007848808AC0F340207047FDF75BBE75486D
:10C57000808AC0F3C02070477248808AC0F30030C0
:10C58000704770484069C0F3003129B1C0F34010D2
:10C59000002804BF012070470020704769498A695C
:10C5A0001043886170476749C86170476548007FDC
:10C5B00000F0010070476348007FC0F340007047FF
:10C5C0006048007FC0F3800070472DE9F04387B0DA
:10C5D0000546F8F7D1FD0446F8F7D1FD594F8046DE
:10C5E000052C0CBF5A4E5B4E387DC0F3031218BFAA
:10C5F000B8F1050F05D1FFF7C4FF002818BF42F0BE
:10C60000020211462846F8F787FE002804BF07B04B
:10C61000BDE8F083FDF78EFDF7F718FC0546F6F749
:10C62000CCFD0020F4F76BFCF5F7A7F94FF00009FB
:10C63000FCF752F8012809D0F8F79EFDA04205D179
:10C64000F8F79DFD404508BF002D0AD0F4F7A8FF7C
:10C65000FDF791FDF8F7B6FFF6F7EBFD07B0BDE883
:10C66000F0836846F5F742FBC0B1052C0CD0B889C1
:10C67000401C81B2B981142906D90222322101203D
:10C68000FFF783FBA7F80C906846FCF769FD684646
:10C69000B047050008BFF5F770F9C9E7F8F79AFD4C
:10C6A000C6E7284AD080118170472DE9F04385B054
:10C6B000294A002104911578284A0B4616780091E2
:10C6C000019102910A46039104A90DF08DFEFDF738
:10C6D000BDFC81464FF000084A464746002E25D94A
:10C6E00032F9021B00234FF0010C012D11D932F950
:10C6F000024B611A09B220F8021B0029B8BF494257
:10C7000009B29942C8BF0B4621460CF1010CAC4559
:10C71000EDD320F8023B4345C8BF98467F1CB74283
:10C72000DED3B8F10F0FC4BF012004900C4800788D
:10C73000012804BF4846FCF7D1FA049805B0BDE8CB
:10C74000F083000098410020844100200C830020E9
:10C75000EFC10100CFCB01008E4000208F400020B0
:10C76000FD4000202DE9F84FDFF8F8B3044600261D
:10C77000BBF90690FC48FD490096007809783746D9
:10C780004518F8F7F9FCF7F71CF98246F7F7FDF8BA
:10C790009BF8041000EB4108F5480078032804BF1B
:10C7A0004046FCF7B1FBBAF1000F7DD09BF80400C6
:10C7B0000AEB400AEE480078022804BF5046FCF716
:10C7C000A3FB0020002D0CD93AF8101038F81020E7
:10C7D000114434F81020511A24F81010401C8542DE
:10C7E000F2D8DFF88C8398F80000062804BF2046B2
:10C7F000FCF78AFB0020691E1CBFBBF908C00B4672
:10C8000013D004EB400134F810204988891A09B28A
:10C8100024F810100029B4BF4A420A466245BCBF42
:10C820000E447F1C401C9842EBD3002FC8BF96FBE0
:10C83000F7F637B204EB450A2AF8027C98F80000B4
:10C84000072804BF2046FCF75FFB00263046691E20
:10C8500018BF0A460FD034F81010C91B09B224F8CB
:10C8600010100029B8BF494209B28E42B8BF0E4627
:10C87000401C9042EFD32AF8026CBBF81400C0F3BE
:10C88000002038B106F047F801282ED006F043F812
:10C8900008282AD006F0A1F8002818BF4FF00A098E
:10C8A0004E450ADD012000E011E0009098F80000FC
:10C8B000142804BF2046FCF727FB98F80000012845
:10C8C00004BF2046FCF720FB0098BDE8F88F00204D
:10C8D000002D86D934F8101038F81020891A24F861
:10C8E0001010401C8542F5D87BE74FF00509D7E7CB
:10C8F0002DE9F04F87B0FDF751FCDFF878B2DBF897
:10C900000000B0F93610B0F93400FDF775FAF7F70A
:10C91000F6FA042000F03DF9DFF8489280B199F86A
:10C920001400C0F3401010B9FFF72BFE40B9DBF83C
:10C930000000806DC0F303400F2818BFF7F7C5FA59
:10C94000052000F026F958B1FFF71BFE40B1DBF8D7
:10C950000000806DC0F303500F2818BFF7F7B5FA39
:10C96000FF2089F80300F8F707FC022804BFDFF86E
:10C9700008A24FF000087DD1D9F81000C0F303647D
:10C98000DBF80000A100806DC9F82080C84000F0ED
:10C990000F05C9F8248021460220C9F82880FFF736
:10C9A00075FA062C4DD2DFE804F0690303036D6DC0
:10C9B000D9F81000C0F3036499F81400022CC0F3F6
:10C9C000031212D011462846F8F7A6FC002838D0EA
:10C9D00002210846F3F77EFCFDF7ACFBFDF7A0FB58
:10C9E000F7F734FA050009D029E0FFF7CAFD00285F
:10C9F00014BF42F0020222F00202E3E799F80000BD
:10CA000000281CBF0001F4F720FAF4F79EFF89F814
:10CA100001805A4E5A4FFBF75FFE01280BD0F8F702
:10CA2000ABFB022807D1D9F81000C0F30360A04285
:10CA300008BF002D06D0FDF773FBFDF79CFBF8F750
:10CA4000C1FD5DE06846F5F751F9A0B16846FCF715
:10CA500087FB68460EF0E3F80546307838B1DAF81F
:10CA6000000080683860DAF80000C0F80080F5F750
:10CA700073F9D0E74DE0F8F7B8FBCCE728460EF0A5
:10CA800091FA3DE0F8F778FB0446F8F778FB0746A3
:10CA9000052C0CBF3B4E3C4E99F81400C0F303121A
:10CAA00018BF052F05D1FFF76CFD002818BF42F015
:10CAB000020211462846F8F72FFC08B3FDF73AFBAF
:10CAC000F7F7C4F90546F6F778FB0020F4F717FAF4
:10CAD000F4F753FFFBF700FE012809D0F8F74CFBF1
:10CAE000A04205D1F8F74BFBB84208BF002D19D082
:10CAF000F4F756FDFDF73FFBF8F764FDF6F799FBF9
:10CB0000FBF7EAFD012804D0F8F736FB02283FF4D2
:10CB100033AF0AF091F8F7F7F1F907B0BDE8F04F3D
:10CB2000FDF73CBB6846F5F7E1F8D0B1052C0ED017
:10CB3000B9F80C00401C80B2A9F80C00142806D9E2
:10CB4000022232210120FFF720F9A9F80C80684663
:10CB5000FCF706FB6846B047050008BFF4F70DFF79
:10CB6000B8E713E098410020944000209340002053
:10CB70000241002084410020B0D401001540002073
:10CB800070400020EFC10100CFCB0100F8F722FB7D
:10CB9000A0E70D4A0228117D1269C1F30311C2F307
:10CBA000074205D0012808BF11F0020F0AD002E0A9
:10CBB00011F0040F06D0012101FA00F0104018BF57
:10CBC000012070470020704798410020384A30B457
:10CBD000146894F86CC01CF0040F1ABF012222EAFA
:10CBE0000C050CF00105B0F90030B1F900201DB1C1
:10CBF000E58AAA1A521E12B21CF0020F03D0A48AB0
:10CC0000E31A5B1E1BB21CF0040F19BF02800B80DD
:10CC100003800A8030BC70474FF6FF71A0F8A8105F
:10CC2000A0F8AA10A0F8AC10A0F8AE1070472DE93B
:10CC3000F0470E46824605F03FFE074605F032FEFD
:10CC400000F13E09002E18BF002588BF4FF6FF787F
:10CC50000FD098BFBDE8F087C5EBC50007EB4014C7
:10CC600094F8D600012804BF94F88C00002811D154
:10CC700003E0BDE8F04701F0F1BEA4F8A880A4F8F5
:10CC8000AA80A4F8AC80A4F8AE802246494650465B
:10CC900003F00EFA94F8DD00022812BF03282046A4
:10CCA00001F032FD681CC5B2B542D5D3BDE8F087AE
:10CCB0007042002000230028B4BF424202460029EF
:10CCC000B4BFC1F1000C8C4642B9BCF1000F05D0D5
:10CCD0000029ACBF4FF487705A2070474FEA0C4CC4
:10CCE000BCFBF2FC30B4FF4C002254F822506545E6
:10CCF0001ED804EB82056D68AC4519D202EB4202E6
:10CD000013B200FB01F2002ABCBF5A4213B2002842
:10CD1000B8BFC3F1B40008DB0029BBBF584200B262
:10CD2000C3F5B47030BCB8BF704700B230BC7047B8
:10CD300004EB82056D68654598BF5A23521C12B2F8
:10CD40001D2AD2DBDDE72DE9F001E7491025402659
:10CD50008024E64A09684FF0200C670010B30128D0
:10CD600050D002281CBFBDE8F0017047488A32232A
:10CD700000FB03F84B8BB8FBF3F808FB08F8C2F88C
:10CD8000148000EB001808EB4010B0FBF3F04043B8
:10CD90009061486F000F062823D2DFE800F0221EC2
:10CDA00022272B2F488A00EB80034FEA83084B8B06
:10CDB000C000B8FBF3F8B0FBF3F008FB08F8404301
:10CDC000C2E90580B1F87400C0F30330062808D228
:10CDD000DFE800F00703070C10149580BDE8F001B0
:10CDE0007047A2F804C0BDE8F00170479680BDE826
:10CDF000F00170479480BDE8F00170479780BDE86E
:10CE0000F0017047488A498BC0EB00135B00B3FB0D
:10CE1000F1F35B43536100EB4003C3EB4010B0FB05
:10CE2000F1F0404390619480BDE8F0017047AE4856
:10CE300000B5006890F87C10428A01FB02F3418B38
:10CE4000B3FBF1FCA94BC3F80CC090F87D00504334
:10CE5000B0FBF1F0186102EB82008000B0FBF1F052
:10CE60004043D8610020FFF76EFFA1484FF6FF71E5
:10CE70000180418000BD2DE9F04F8DB09846DDE97D
:10CE800016760D46044605F00DFD079005F02AFDC7
:10CE90000C900020009095484FF4A051B0F804A0E9
:10CEA0000B970191D0E905B004908F4801684B8A37
:10CEB0004A8B9800B0FBF2F040430A90642058433C
:10CEC000B0FBF2F04043089003EB8300B0FBF2F0BC
:10CED0004043099094F891C086481CF800700A30CD
:10CEE00047B1012F0AD0032F04BF1CF8000003280C
:10CEF0004ED007E01CF8000020B904E01CF8000048
:10CF000001282DD00120DFF8F09194F8DD20A9F15F
:10CF10000A07A7F10A0C022A1CBF94F8B320012AC1
:10CF200065D094F89130754A02EBC30252F8083C80
:10CF3000039352F8042C02922A8806926A8805927A
:10CF400094F8C420002A74D094F89220C2EBC20353
:10CF50000C9A02EB431292F8C420002A6BD095E0A1
:10CF6000DDF81CC001209CF80CC0BCF1000FCAD039
:10CF700003EBC30C0CEB031CBCFBF2FC03EB430305
:10CF8000DB00B3FBF2F252430CFB0CFB0492BAE75A
:10CF9000079F01203F7B002FB5D003EBC30707EBB2
:10CFA0000317B7FBF2F703EB4303DB00B3FBF2F22B
:10CFB000524307FB07FB0492D845A4D3504F07EB1D
:10CFC0004C0232F8023CB3F5807F9CD9A3F5807304
:10CFD0009BB222F8023C94F89120B3F5807F07EBD6
:10CFE00042023CBF4FF4807322F8023C8BE72A8850
:10CFF00003926A88029294F89130002203F80C2080
:10D0000094F89130DA5594F8913003F8092094F8A7
:10D0100091E03B4A019B02EB4E0222F8023C94F85D
:10D020009120012A88D1314A0023137053709370E4
:10D0300082E70EE0FFE794F89130314A02EB4302B9
:10D0400032F8023CB34221D922F8026C94F8C42091
:10D05000E2B9089A904594F8DD2012D3022A10D044
:10D06000089A904512D394F891E0254B94F8C42087
:10D0700003EB4E0333F802ECB64588BF23F8026C8D
:10D0800006E04FF4A0630222019301E094F8C4206B
:10D090000A9B984538BF0222144B9B78002B01BF96
:10D0A00094F89130012B94F8C430032B0AD1DFF8A7
:10D0B0003CE001238EF80230114B1B88B34284BF41
:10D0C0000F4B1E80D84529D3022A18BF002825D02F
:10D0D00094F891300020D85594F8913003F8090065
:10D0E00010E0000028D8010070420020C441002058
:10D0F000E44100203587002017870020B4860020F7
:10D100002287002094F8910010F80C30642B3CBF6B
:10D110005B1C00F80C30032000901AE0049B98453B
:10D1200001D2022A03D110B1022A21D011E094F8D1
:10D130009130002003F80C0094F8913003F80900B6
:10D1400094F89100C35D642B3CBF5B1CC355022067
:10D15000009094F891B0DFF8E8E50EEB4B031BF874
:10D16000077033F8020CBFB1B04237D34AD946E05A
:10D1700094F891304FF0000003F80C0094F89130CF
:10D18000D85594F8910010F80930642B3CBF5B1C13
:10D1900000F809300120DBE71BF80CC0BCF1000FE0
:10D1A00023D0864216D2A0EB060CA0EB6C0080B216
:10D1B00023F8020C94F89130000A0EEB43034FF66B
:10D1C000FF7C23F8020C94F891300CEA00200EEB5F
:10D1D000430307E0DDF82CC0604501D2504401E074
:10D1E00010D90CE023F8020C0CE01BF809C0BCF1CC
:10D1F000010F07D9DDF804C06045EFD302D9A0EBD9
:10D200000A00EFE794F891700EEB4700012F30F819
:10D21000020C04D1DFF82CC5009B8CF800300028EC
:10D2200008BF002160D0022A1CBF099A90455CD833
:10D23000079A000A92F83020022A1BD30E8B069A16
:10D24000DDF80CA006FB02F30A8AB1F81A80B3FBE2
:10D25000F2FC06FB0AF6B6FBF2F6B1F81290059B5B
:10D26000029A08FB03F308FB02F2B3FBF9F3B2FBEB
:10D27000F9F21AE08A8A069B0E8A02FB03F3B3FBDB
:10D28000F6FCDDF80CA0B1F8169002FB0AF2B2FB36
:10D29000F6F6B1F81280059B029A09FB03F309FB2D
:10D2A00002F2B3FBF8F3B2FBF8F2A0F1010808FBBD
:10D2B00006C608FB0232B6FBF0FCB2FBF0F2088AAD
:10D2C00000FB0CF007D30B8BB0FBF3F04B8A498BC0
:10D2D00003FB02F206E08B8AB0FBF3F04B8AC98AAB
:10D2E00003FB02F2B2FBF1F130E0B1F814C0069A90
:10D2F0000B8A0CFB02F2B2FBF3FACA8A059E498A3A
:10D3000002FB06F6B6FBF1FB039E4FEA10100CFB86
:10D3100006F6B6FBF3F8029E02FB06F6B6FBF1F941
:10D32000A0F1100606FB08F806FB09F606EB0B1643
:10D33000B6FBF0F608EB0A18B8FBF0F803FB08F0B0
:10D3400001FB06F1B0FBFCF0B1FBF2F1FE4A02EB8F
:10D35000C70343F8080C94F8913002EBC30242F87B
:10D36000041CA880E9800DB0BDE8F08F2DE9F84FCE
:10D37000F649F74B01444FF0000E01F801EC03446D
:10D38000012103F8011CF349744601EB401100919F
:10D39000F149724601EB401B01F5A07101EB401908
:10D3A000009800210BEB041809EB041700EB04169E
:10D3B000002008EBC10307EBC10C06EBC10503EB32
:10D3C000800A4AF8202C0CEB800A4AF8202C05EB46
:10D3D000800A401C00B24AF8202C0228EFDB481CCF
:10D3E00001B20229E4DB601C04B2022CD8DBDB486A
:10D3F000DB4E0021D0F800C0A6F110070BEB0E1891
:10D4000009EB0E1A002006EBC10908EBC1050AEB77
:10D41000C10407EBC103814207D1BCF87A2043F86D
:10D420002020BCF8782049F8202053F8202005EB74
:10D43000800B02EB820252004BF8202C04EB800B95
:10D44000401C00B24BF8202C0228E4DB481C01B23F
:10D450000229D7DBBDE8F88F10B490F891C0C14C19
:10D4600000230CF8043090F891C00A340CF8043012
:10D47000BA4B90F891C01B6893F87430C3F3031350
:10D480001B02153404EB4C0C2CF8023C90F891C0B4
:10D49000A4F16E0303EBCC0C4CF8081C90F891102F
:10D4A00003EBC10141F8042C90F8910010BC5DE73A
:10D4B00010B5044605F016FA014694F8DD0002287E
:10D4C00004BFB4F8AC00B4F8AE1009D094F89200E0
:10D4D000C0EBC00001EB4011B1F8AC00B1F8AE10E8
:10D4E00094F8C420022A04BFA4F8AC00A4F8AE103B
:10D4F00010BD2DE9F041044605F0F4F994F8DD0083
:10D50000994E022835D09548B4F8AE50B4F8AC1016
:10D510000068038B028AB0F81AC0478A05FB0CF535
:10D5200095FBF7F05943B6F9005091FBF2F16B43CC
:10D5300093FBF2F3B6F9022002FB0CF292FBF7F236
:10D54000B1EB030C48BFA3EB010CBCF10A0F16DAD8
:10D55000811A48BF111A0A2911DAA5F57F40FF3850
:10D560000DD03088A4F8AC007088A4F8AE00BDE8F7
:10D57000F081B4F8AC003080B4F8AE0002E04FF0B7
:10D58000FF3030807080BDE8F0812DE9F041044625
:10D5900005F0A8F901466B48DFF8D0C100690CF12D
:10D5A0000B0700FB00F694F8DD00022842D094F847
:10D5B0009200C0EBC00001EB4010B0F8AC10B0F826
:10D5C000AE00B4F8AC30B4F8AE205D1A05FB05F837
:10D5D000151A05FB0585B5420ADA94F8915015F83D
:10D5E0000C50012D04BFA4F8AC10A4F8AE0013D069
:10D5F00094F8915007EB850636F8048CA3EB0808E5
:10D600004144A4F8AC1036F8021C511A0844A4F89E
:10D61000AE00002005F80C0094F8910007EB8000A4
:10D6200020F8043C94F8910007EB800020F8022CCD
:10D63000BDE8F08194F89120B4F8AC1007EB8202B9
:10D64000B4F8AE0022F8041C94F8912007EB820293
:10D6500022F8020C94F89130012203F80C20B0E774
:10D660002DE9F04F90F891C08FB04FF480630029FE
:10D670000CBF394C3E4C04EB4C14364D029205EB7A
:10D680004C1705F5A5756544203C15F8015C07EBC2
:10D69000051606EBC10858F8206C921B039290F80F
:10D6A000DD20022A1CBF90F8B30001287ED058F874
:10D6B0001C8C04EB051206EB0809CDF83890D2F863
:10D6C0000490D6689568106809EB0602DFF8A4900C
:10D6D00028441044D9F800A035445044D9F804A097
:10D6E000DFF87CB05244D9F808A0D9F80C90554422
:10D6F0004E44DDF808A0DDF83890AAEB0909CDF812
:10D700002090DDF80C90A9EB0809CDF82C90DBF8FF
:10D7100000908144CDF82890DBF8049009EB020AD0
:10D72000DBF80890DBF80CB0A9440BEB060EDDF833
:10D7300028B00BFB0EFB0AFB19BB9BFBF3FB1BE0AA
:10D7400022870020C4410020B4860020548C002091
:10D750005E8C0020148B00209488002070420020F2
:10D760002442002003870020E84100207F8600201B
:10D77000D489002014420020BBF1000F08BF4FF0F5
:10D78000010B4FEA8E2E4FEA8A2A9AFBFBFA4FEAE8
:10D79000892999FBFBF99EFBFBFECAF1000ACDF833
:10D7A00034A0C9F10009DDF828A000E077E04FEAD5
:10D7B0008A2A9AFBFBFB00FB0EFA02FB09AA9AFBE2
:10D7C000F3FACDF828A0DDF834A000FB0AFA02FB3A
:10D7D0000BAA9AFBF3FACDF824A005FB0EFA06FB80
:10D7E00009A999FBF3F9DDF834A0CDF8309005FBD9
:10D7F0000AF906FB0B9999FBF3FBDDF828A0DDF88D
:10D8000020900AFB09FEDDF824A0DDF82C900AFB2D
:10D8100009EEDDF820A0DDF830909EFBF3FE09FB59
:10D820000AFADDF82C900BFB09A999FBF3F9DDF856
:10D8300038A0C844F244CDE900A8DDF828A0CBF513
:10D84000806ECAF5806808FB00FBDDF824A0DDF8D7
:10D850003090CAF1000AC9F100090AFB05BB08FBB8
:10D8600002F809FB00F00AFB06880EFB05009BFB93
:10D87000F3FB98FBF3F890FBF3F0CDF810B0CDE993
:10D88000058009FB02F00EFB060090FBF3F0079009
:10D89000FF480022E84604AE00EB0C0315E0FC4A0A
:10D8A00000206244039012F8012C02AB07EB021235
:10D8B00002EBC10253F8204002EB8005401C00B28D
:10D8C00045F8204C0228F5DB20E013F8015C58F8FD
:10D8D000220007EB051505EBC10505EB820545F8B0
:10D8E000200C002006EBC20513F801AC55F820907F
:10D8F00004EB0A1A0AEBC20A4AF82090401C00B254
:10D900000228F1DB501C02B2022ADEDBE048604450
:10D9100010F8010C07EB001000EBC10050F8200CD0
:10D920000FB0BDE8F08F0288438862F30F01808852
:10D9300063F31F419A4284BF63F30F0162F31F41F7
:10D940000A0C824288BF60F31F4188B20A0C9042E1
:10D9500084BF62F30F0160F31F41080C704770B57C
:10D960000146154691F8DD60CA4B91F8911090F888
:10D9700091202C88688801EB4101A3F1780C0CEB15
:10D98000810C022E19D03CF80A1C2CF8081C3CF81B
:10D990000C1C2CF80A1C2CF80C4C3CF8041C2CF821
:10D9A000021C3CF8061C2CF8041C99182CF8060CD8
:10D9B00011F8011C012911D019E02CF8084C2CF8A1
:10D9C0000A4C2CF80C4C2CF8020C2CF8040C1A44C1
:10D9D0002CF8060C012102F8011C08E0ACF10C0047
:10D9E000FFF7A1FF0446ACF10600FFF79CFFAC80F7
:10D9F000E88070BD30B4002488B0A44601EB00116B
:10DA000001EB4C0030F8100C04440CF101001FFA3B
:10DA100080FCBCF1080FF3D3E4081C600023184617
:10DA20006D4601EB400C3CF810CCACEB040C0CFB4D
:10DA30000CFC45F820C0401C80B263440828F0D399
:10DA4000D80831F80A3C31F8101C591A49431160C2
:10DA500008B030BC7047904A0021024402F8011C13
:10DA60008E4A024402F8011C8D4A024402F8011C4D
:10DA70008C4A02EB800242F8041C8B4A02EB8002C3
:10DA800042F8041C894A02EB800242F8041C884ACE
:10DA900002EB800242F8041C864A02EB400020F8A8
:10DAA000021C418070472DE9FF4FE1B053B20022C4
:10DAB0005792814A1F461268B2F812C0528BCCEBC3
:10DAC0000C1CBCFBF2F25092754ADFF8D0C1024444
:10DAD00012F8016C0CF10202844402441CF8015C4F
:10DAE00012F8014C00EB800C01EB0C1C002E7DD0D9
:10DAF0000CEB450131F8505C5495B1F8501053913E
:10DB000012F8011C143949B20029BCBF283149B2AE
:10DB10000CEB410131F8502C5292B1F850101E22FA
:10DB200051910CEB4401052A31F8504C5994B1F84D
:10DB30005010589140F2E7815A49EE4601EB8001BE
:10DB400051F8044C58495E9401EB8000012150F8D3
:10DB5000040C5B90844268DD649800885A90501EE3
:10DB600058BF744612D40CEB430544F8201004EB64
:10DB700080065B1E35F8505C5BB2C6F8A050002BE7
:10DB8000B8BF2723401E00B20028ECDA00210C4663
:10DB9000B846501E58BF754616D40CEB480355F8CE
:10DBA0002060B3F850307343A8F1010659184FFABA
:10DBB00086F844EBE374B8F1000FB8BF4FF02708C4
:10DBC000401E00B20028E8DA00252E46501E58BF3D
:10DBD000F1465CD40CEB470309EB8008B3F85030F6
:10DBE000D8F8A0807F1E03FB08F300E00BE05D196E
:10DBF0007FB246EBE376002FB8BF2727401E00B266
:10DC00000028E7DA7DE0611CCAB23CF8501C549150
:10DC1000BCF85010539125F00101614431F8505C7B
:10DC20005295B1F8501051917BE76E9800885A9048
:10DC3000501E58BF744612D40CEB430544F8201014
:10DC400004EB80065B1EB5F850505BB2C6F8A050DE
:10DC5000002BB8BF2723401E00B20028ECDA0021B9
:10DC60000C46B946501E58BF75462ED40CEB4903DE
:10DC700055F8206033F8503C7343A9F10106591858
:10DC80004FFA86F944EBE374B9F1000F16E038E07F
:10DC9000548C0020E08C0020CC410020CA410020A0
:10DCA000CE410020044200200C420020EC41002024
:10DCB000F4410020FC41002070420020B8BF4FF02A
:10DCC0002709401E00B20028D0DA00252E46501E3B
:10DCD00058BFF14615D40CEB470309EB800833F825
:10DCE000503CD8F8A0807F1E03FB08F35D197FB27B
:10DCF00046EBE376002FB8BF2727401E00B200286E
:10DD0000E9DA0027B8463846002AC8BFF4460ADDDB
:10DD10005CF8203000F101005B43DF1948EBE37849
:10DD200000B28242F4DC0023CDE955331846002AC4
:10DD3000C8BFF44615DD0CEB80095CF82030D9F83B
:10DD4000A09003FB09F3DDE955A94FEAE37B13EB50
:10DD500009034BEB0A09401CCDE9559300B28242FE
:10DD6000E9DC4FF0000AD1465046002AC8BFF3460E
:10DD700010DD0BEB80035BF820C0D3F8A03000F17E
:10DD8000010003FB0CF313EB0A0A49EBE37900B241
:10DD90008242EEDC4FF0000CE3466046002A0EDDC6
:10DDA0006B4603EB800300F10100D3F8A03000B212
:10DDB0005B4313EB0C0C4BEBE37B8242F0DCA7FBE9
:10DDC0000C32CDE95CCB08FB0C2207FB0B2CDDE908
:10DDD0005520A0FB0ABECDE95F2002FB0AE200FB52
:10DDE0000922B3EB0B006CEB0202CDE95520104386
:10DDF00004BF4FF0000B594632D0DDE95C03A0FBB5
:10DE0000012C5C9103FB01C100FB0411DDE95F30D3
:10DE1000A0FB05CB03FB05B300FB0633B2EB0C0004
:10DE200061EB0301DDE955320BF0A8FD8346A7FB4A
:10DE3000050108FB051107FB06125C99AAFB013CD2
:10DE400009FB01C10AFB0411C01A62EB01010904BC
:10DE5000DDE9553241EA104100040BF08FFD014627
:10DE60005A9848431BEB204048BF00205B9B5E9ABA
:10DE70009A4224DD549A539B4A430BEB2242D31A15
:10DE800044BF539B9B1A509A93423CD2529A51439F
:10DE9000519A0BEB21418A1A44BF519A521A509958
:10DEA0008A4230D25899091A44BF5899411A509A57
:10DEB000914228D26E9908800120579023E0539A0E
:10DEC000549B4A430BEB2242D31A44BF549B9B1AE8
:10DED000509A934217D2519A5143529A0BEB2141D7
:10DEE0008A1A44BF529A521A50998A420BD25999AF
:10DEF000091A44BF5999411A509A914203D2649920
:10DF0000088001205790579865B0BDE8F08F2DE943
:10DF1000FF4F8DB09A468B46054604F0C3FC009037
:10DF200090F8300002282CBF03200A20049095F8B6
:10DF30009140022C94BF4FF001094FF0000995F871
:10DF4000760001281CBFFE48C06908D0019095F8F2
:10DF5000DD00FC4B4FF0000802283AD109E0FA48F6
:10DF600064220068418A408B5143B1FBF0F040438A
:10DF7000ECE71819B9F1000F00F8018CF3482044C0
:10DF800000F8018C80F80980F148204400F8018CE9
:10DF900080F80980EF4800EB440020F8028CA0F8DC
:10DFA0001280ED488BF8C480204485F8C48000F8C6
:10DFB000018CEA48204400F8018CE948204400F82C
:10DFC000018CE848204400F8018C1CBF2046FFF774
:10DFD00042FD0F981919B9F1000F0288E248039128
:10DFE00000EB0410079011F8011C029100EB4100B6
:10DFF00020F8102CBAF80010DC4AA0F8901076D067
:10E00000A2F122002044A2F120010590214410F841
:10E01000010C01F8010CA2F11E012144069111F836
:10E02000011C01B3411CC9B2282926D3D04904EBF5
:10E03000840301EB031101EB400331F850EC33F89A
:10E0400050CCAEEB0C0C02EB840E4EF804CCB3F8C3
:10E050005030B1F85010CB1A02F1080101EB8401E5
:10E0600041F8043C24E002EB840141F8048CC149EE
:10E0700001EB840141F8048C1AE0BD4B04EB840CE5
:10E0800003EB0C1303EB410131F8503C31F852CC57
:10E09000A3EB0C0302EB840C4CF8043CB1F85030B9
:10E0A000B1F84E105B1AB34901EB840141F8043C0E
:10E0B0000F9904EB840C27280B88AD4901EB0C1158
:10E0C00001EB400121F8503CBAF80030A1F8503083
:10E0D00003D1069B012103F8011C401C0599C0B225
:10E0E000282801F8010C24BF059800F8018C95F848
:10E0F000DD00022800F08081002006900590029843
:10E100000799C01D00F007000F9B01EB400030F89D
:10E11000101C1B88B0F89000591ABAF80030181A71
:10E12000B9F1000F34D0944B234413F801CC934B36
:10E13000BCF1000F03F1080648D003EB840C002962
:10E140005CF8047CACBF0B464B421F4406EB8403D7
:10E150004CF8047C53F804EC0028B4BF4642064651
:10E16000764402EB840243F8046C52F8042C002A33
:10E17000B8BF5242BA1A4CF8042C7E4A02EB840211
:10E1800052F8042C002AB8BF5242B21A43F8042CA9
:10E190006D4A1268138B5943138A91FBF3F6518B26
:10E1A0004843518AB9F1000F90FBF1F704D072484F
:10E1B000204410F8010C00B3002E3CDD65484FF000
:10E1C000020100EB440020F8028C4CE003EB8402D7
:10E1D000002952F804CCB4BF4B420B46634442F8CA
:10E1E000043C06EB8402002852F804CCB4BF43423E
:10E1F0000346634442F8043CCAE76148002E00EB42
:10E20000440030F8022CB4BF714231468A4205DA2C
:10E21000002EACBF3146714220F8021C4288002F0C
:10E22000B4BF794239468A42C6DA002FACBF3946BC
:10E2300079424180C0E706DA4648012100EB4400FC
:10E2400020F8028C0FE04248204410F8011C41489D
:10E2500000EB440030F8022C642A04D2521C20F84F
:10E26000022C01200690002F07DD3A4A4FF00400EF
:10E2700002EB4402A2F8128015E007DA354A4FF0AB
:10E28000030002EB4402A2F812800CE0314A30484D
:10E2900002EB44022044538A407A642B03D25B1C75
:10E2A0005382012205922A4A224412F8013C1BB3F0
:10E2B0008B4222D1274B03EB440333F8023C3C2B27
:10E2C000224B234496BF13F801CC03F8018CBCF118
:10E2D000640F2BD2DDF818E0BEF1000F26D10CF14F
:10E2E000010C0CF0FF0C03F801CCBCF10A0F1DD39C
:10E2F000194B234403F8018C18E0144B234413F802
:10E3000001CCBCF1050FDFF850C0A44436BF1CF8A7
:10E3100001EC0CF8018CBEF1640F05D2052EA4BFF0
:10E320000EF1010E0CF801EC03F8018C537A4BB39B
:10E33000834245D1074B03EB44035B8A3C2B22E02D
:10E34000C44100202A8E002070420020488E002008
:10E35000348E00205C8E0020848E00208E8E002063
:10E36000988E00208A880020EA8C0020EC41002052
:10E370004A870020F4410020CE41002004420020C2
:10E38000FC41002035E0FE4B234496BF93F809C0C2
:10E3900083F80980BCF1640F2BD2DDF814E0BEF1E4
:10E3A000000F26D10CF1010C0CF0FF0C83F809C012
:10E3B000BCF10A0F1DD3F34B234403F8018C18E082
:10E3C000EF4B234493F809C0BCF1050FDFF8B4C349
:10E3D000A44436BF1CF801EC0CF8018CBEF1640FAC
:10E3E00005D2052FA4BF0EF1010E0CF801EC83F845
:10E3F000098002F8011C507202980399401CC0B2B7
:10E4000001F8010C08280AD3039800F8018C9BF846
:10E41000C400002804BF01208BF8C40006E09BF86C
:10E42000C400002808BF85F8C48053D00AAB08AAEE
:10E43000D5492046FFF7DEFA83460BAB09AAD3493C
:10E440002046FFF7D7FA01998B4598BF88420CD92F
:10E45000032085F8C400CE48CE492044214400F86A
:10E46000018C012001F8010C14E0C548204410F88B
:10E47000011C08299CBF407A082810D9032085F880
:10E48000C400C3480121204400F8018CC148204445
:10E4900000F8011C95F8C400032839D01AE0BC48E4
:10E4A000204410F8011CC8293CBF491C00F8011C7D
:10E4B000B849214411F8011C012908D110F8011CA8
:10E4C000049881429CBF032085F8C40020D9022013
:10E4D00085F8C400B048204400F8018CA9482044C5
:10E4E00000F8018CAD4802212044019000F8011C85
:10E4F000AB48B9F1000F00EB040B0BF8011C04BF93
:10E5000011B0BDE8F08F95F8C400032810D012E0D8
:10E51000A148204410F8010C032805D29948204452
:10E5200010F8010C0328DDD3009902200873D9E705
:10E5300004F0F4F928B12046FFF78DFA11B0BDE8D8
:10E54000F08F9848204410F8010C01280ED00028C4
:10E550001CBF11B0BDE8F08F9348204410F8010CA7
:10E56000401C07283CBF11B0BDE8F08F282ED8BF53
:10E57000282F09DC8D4800EB440030F8021C2829C4
:10E580009CBF408828280FD90098007B002804BF32
:10E5900011B0BDE8F08F0320019901F8010C0BF8D0
:10E5A000010C11B0BDE8F08F7F48CDF800A02044E9
:10E5B0007F4910F8012C20460F9BFFF774FA0128C1
:10E5C00007D0019800F8018C0BF8018C11B0BDE860
:10E5D000F08F0199012001F8010C0BF8010C11B02A
:10E5E000BDE8F08FB0F8A830B1F8A8C0B3EB0C02CA
:10E5F00048BFACEB0302B0F8AA30B1F8AA10581A21
:10E6000048BFC81A02FB02F100FB0010704770B54A
:10E610000D46044604F046F994F8DD00654E0228E4
:10E620001DBF94F8B3000128012DB4F8AC000FBF52
:10E63000B4F8AE2094F8910006EBC00151E9020253
:10E6400032213125B4F8ACC0B4F8AE3005FB00C0BF
:10E65000B0FBF1F005FB0232B2FBF1F194F891202E
:10E6600006EBC20242F8080C94F8912006EBC202B5
:10E6700042F8041CA4F8AC00A4F8AE1070BD2DE95B
:10E68000F0074D4A0F88B0F800801268DFF82CA11F
:10E69000B2F81890158AB2F81AC0568A07FB0CF423
:10E6A00094FBF6F208FB09F393FBF5F314B2BAF806
:10E6B00000201BB202FB09F999FBF5F5BAF80290AC
:10E6C0002DB209FB0CFC9CFBF6FC0FFA8CFC5E1BCC
:10E6D00048BFEE1A0A2E10DAB4EB0C0348BFACEBBD
:10E6E00004030A2B09DAA2F57F43FF3B1FBF028018
:10E6F000A1F80090BDE8F0077047AAF80080AAF8DA
:10E700000270BDE8F00770472DE9F04F87B004466E
:10E7100000F09EF9834600F09EF9824604F0E2F88C
:10E72000059004F0BFF8DFF890908046007B94F8E5
:10E730009150D9F80010002864D0086FC0F3C0428F
:10E740000192C0F34042C0F3804004920090486FB1
:10E75000C0F303410F021149294411F8011C022999
:10E760000EBF4FF44076C0F3035006020220FEF7BE
:10E77000EAFA1148006890F8700010F0010F1FE0ED
:10E78000488E00208E8E0020EA8C00208A8D00208A
:10E79000988E00208A880020848E002036870020F2
:10E7A00040870020CE410020CC410020FC410020C9
:10E7B0004A870020A48E002070420020E4410020FF
:10E7C00000F02B8194F89200B4F8A810ADF808106E
:10E7D000B4F8AA10ADF80A10C0EBC001059802AA5F
:10E7E00000EB411949462046FFF7B9F80198002887
:10E7F00041D0BDF80C00ADF80800BDF80E00ADF832
:10E800000A003DE091F87000C0F3C0020192C0F32D
:10E810004002C0F380000492009098F81A0001288A
:10E8200015D004F07BF838B104F075F8012815D044
:10E8300004F071F8082811D0D9F8000090F874009D
:10E8400001070F0DC0F30310060200208FE7B1F897
:10E850007400C0F3032007023E46F6E7D9F8000033
:10E86000B0F8740001070F0DC0F30320000200F59B
:10E87000807601207BE76E490020294401F8010CD5
:10E8800094F8DD00022819BF94F8B3000128284647
:10E89000FEF76CFDBDF8082000212046FEF7E0FEE3
:10E8A0000190BDF80A2001212046FEF7D9FE01990A
:10E8B0000029B8BF00210028B8BF0020DFF874C1CC
:10E8C000DCF80020B2F91030A3F1010E8E45B8BF7C
:10E8D0007146B2F91220531E8342B8BF184689B25E
:10E8E00082B25548554BADF80C10ADF80E202844B7
:10E8F0002B4410F801CC13F801EC00F801EC03F8FC
:10E9000001CC009800281CBFADF80810ADF80A2013
:10E910000DF10E0303AA49462046FFF7F8FAB4F8B2
:10E92000A820B9F8A800111A48BF811AB4F8AA2083
:10E93000B9F8AA30D01A48BF981A494300FB00130F
:10E9400098F80C00A8B93E48284410F8010C01289A
:10E9500007D070B93B48284410F8010C401C282807
:10E9600007D9BDF80C00ADF80800BDF80E00ADF8F1
:10E970000A00CDE9007698F8302002A92046FEF77B
:10E980007AFA049838B1BDF80C00ADF80800BDF86B
:10E990000E00ADF80A00BDF80800BDF80A10584591
:10E9A000B8BF58465145B8BF5146224D2A68B2F902
:10E9B0001030A3EB0B03A3F1010C8445B8BF6046F4
:10E9C000B2F91220A2EB0A02531E8B42B8BF1946BD
:10E9D000A4F8AC00A4F8AE1003F0A0FF012804BF17
:10E9E00094F8DB00012807D1B4F8A800A4F8AC0023
:10E9F000B4F8AA00A4F8AE00286890F8700010F0EF
:10EA0000100F04BF07B0BDE8F08F98F83010204613
:10EA1000FEF7BBFD07B0BDE8F08FB4F8A800A4F87E
:10EA2000AC00B4F8AA00A4F8AE0007B0BDE8F08FBF
:10EA3000E08C002070420020548C00205E8C00206E
:10EA4000CE410020CC410020FE487047FE48704770
:10EA5000FE4800787047FD4840787047FB480E211B
:10EA60008180C180E02101814181704703460020FF
:10EA700002460029D8BF704753F822C0521C604498
:10EA80009142F9DC70472DE9F05F0E46054603F030
:10EA900039FF044603F032FF310291FBF0FC2902FA
:10EAA00091FBF4F3DFF8A4E3E74D5E12BEF80490A7
:10EAB000BEF8068000214FEA6C2705F1E00A002C21
:10EAC0000BDD01FB03F206EB222245F821204AF878
:10EAD0002120491C09B28C42F3DCDA4E002106F1F8
:10EAE000E00B00280BDD01FB0CF207EB222246F8BD
:10EAF00021204BF82120491C09B28842F3DC0CFB91
:10EB000009FC03FB08F34FEA6C315A135F13CEF88C
:10EB10000C102B684FEA6C3C9B1A2B6005EB8403AE
:10EB200053F8045C154443F8045C33685B1A3360A3
:10EB300006EB800353F8045C0D4443F8045C9EF834
:10EB40000330002BDAF8003017D09B1ACAF80030D7
:10EB50000AEB84030BEB800053F804CC624443F8C7
:10EB6000042CDBF80020521ACBF8002050F8042CBB
:10EB7000114440F8041CBDE8F09F9A1ACAF800201E
:10EB80000AEB84020BEB800052F8043C3B4442F851
:10EB9000043CDBF80020511ACBF8001050F8041C9C
:10EBA0006144E6E7A948C078012818BF00207047F3
:10EBB0002DE9F041DFF898820446A44DD8F8000012
:10EBC000468A078A0E20142C1CD2A4F10F010529B5
:10EBD00018D3491D052903D21420A880E88013E02A
:10EBE000611F052903D21620A880E8800CE0052CBF
:10EBF00008D203F093FE002814BF18201220A8802A
:10EC0000E88001E0A880E88000210CB3D8F800007B
:10EC1000428A408BC2EB0212B2FBF0F0A870E9709E
:10EC2000A9884FF6FF7000EA01112981E98800EAFE
:10EC300001106881D8F80000418A408B6143B1FB24
:10EC4000F0F02870687039463046BDE8F0411AE7A8
:10EC5000A9700120E870E3E710B57D484FF6FF7416
:10EC6000026892F86C30508AB2F81AC0DB0843434D
:10EC7000B3FBFCF3118A754A137053700E23938013
:10EC8000D380E02313815381C0EB0013B3FBFCF36B
:10EC900093700023D370FFF7F6FE6E49002001EB5E
:10ECA000800221F82040401C80B254800A28F6D30C
:10ECB00010BD2DE9F04FB3B00D460446CC22664995
:10ECC00068460AF047FE6248B5F902200068012A4A
:10ECD00090F807C090F80680478A068A687800FB9B
:10ECE0000CF109B2D8BF01222B78DFF870E1EB46B6
:10ECF00083B1ACF101094B45194417D104EB410133
:10ED000031F9021C0129D8BF0121C902494291FBF6
:10ED1000F2F140E004EB4101B1F902100129D8BF42
:10ED20000121C90291FBF2F109B235E004EB41097E
:10ED300039F9021C0129D8BF0121B9F90290B9F1B2
:10ED4000010FD8BF4FF001094FF0640A01FB0AF12F
:10ED500009FB0AF901EB620109EB620991FBF2F18F
:10ED600099FBF2F93BF911103BF91990494508BF9D
:10ED7000002111D001EB090A1AF5004FB8BFF24685
:10ED800004DBBAF5004FA8BF47F6FF7AA1EB0901F3
:10ED9000C90291FBFAF109B2A0B1A8F101094845F5
:10EDA000A0F1010909FB0CF90FFA89F9994415D171
:10EDB00034F91940012CD8BF0124E402644294FBC9
:10EDC000F2F255E003EB0C0934F91940012CD8BFDD
:10EDD0000124E40294FBF2F212B24AE034F91990F1
:10EDE000B9F1010FD8BF4FF0010900F1010A0AFB88
:10EDF0000CFA0FFA8AFA9A4434F91AA0BAF1010F00
:10EE0000D8BF4FF0010A642409FB04F404EB620448
:10EE100094FBF2F44FF064090AFB09F909EB62096B
:10EE200099FBF2F23BF914403BF91220944208BFDF
:10EE300000221ED004EB020919F5004F14DBB9F5CE
:10EE4000004F0DE0F48E0020648F0020344200203B
:10EE500070420020B4900020A0D801000080FFFF85
:10EE6000B4BFCE4647F6FF7EA21AD20292FBFEF254
:10EE700012B21B04000403EB011100EB021201F5B6
:10EE8000004002F5004190FBFCF091FBF8F170436B
:10EE900001FB07F100144FEA21414CBF002202465A
:10EEA000B242C8BF304602DC0028B8BF00200029AB
:10EEB000B4BF00220A46BA42C8BF394602DC002964
:10EEC000B8BF0021A5F8A800A5F8AA1033B0BDE886
:10EED000F08F2DE9FF4FFFB00E4691467021684636
:10EEE0000AF03DFD70211CA80AF039FD702138A8F8
:10EEF0000AF035FD702154A80AF031FD03F0F2FC50
:10EF0000044603F0CFFC7B9003F0E0FC00F13E08E8
:10EF1000739003F0FBFC789003F0F0FC054603F0DF
:10EF2000F1FC0746FE480068418A7091008A7190A2
:10EF300003F0F4FC012812D103F0EDFC01280ED1FE
:10EF4000DFF8E0A31820AAF80400DDE97001FFF75C
:10EF50009AFDF548DAF80C20016B11440163F3487F
:10EF60007A907038799099F8000099F8011099F822
:10EF7000913001FB050099F89210305CC1EBC101A2
:10EF800004EB4112EA4900F03F0001EB830C3CF82E
:10EF9000041C7291A1F57F43FF3B1DBF3CF8021C8E
:10EFA000A1F57F43B3F1FF0393880CBFD188729B17
:10EFB000B9F80440749404F1050ADE4CA4FB0ABAC3
:10EFC000CAF3CF0ACDF8F0A1B9F806A00AF1050BF3
:10EFD000A4FB0BEBCBF3CF0BCDF8DCB103F1050BAE
:10EFE000A4FB0BEB01F1050EA4FB0EE4C4F3CF046C
:10EFF0007694749C4CF6CD4E04FB0EF4E40C7594A0
:10F000000AFB0EF4E40C7D9403FB0EF4E40C749400
:10F01000DDF8F0A1CBF3CF0B01FB0EF44FEAD44E99
:10F02000DA4504BFDDE9764AA24506D0DDE9744A37
:10F03000A24504BF7D9C74450FD17B9C94F8304061
:10F04000022C0AD3DDF8CCA19AF830A0A24504BF67
:10F0500099F89040022C00F0C9804FF6FF712CF80F
:10F06000041CB34A99F8913002EB830222F8021C87
:10F0700099F80AA099F80B10729199F80C4099F838
:10F080000D10729AE9460DF1700E8A4228D802FBE3
:10F0900005F31FFA83FB5346A2451DD8DDF8FCC1DA
:10F0A0000BEB03083CF918C016F8088008F03F087D
:10F0B00080450DD1DDF8E081C44509DB59F8238096
:10F0C000E04449F823805EF82280C4444EF822C010
:10F0D0005B1C9BB2A342E1D9521C92B28A42D6D9A0
:10F0E00000214A460846002D40F3E48052F82030C3
:10F0F000401C1944A842F9DB002940F3DB800021C1
:10F1000072460846002F40F3D58052F82030401C4C
:10F1100019448742F9DC002940F3CC800020002DFF
:10F1200088BF38A90BD9799A59F8203052F8202095
:10F130005A4341F82020401C80B28542F3D8002079
:10F14000002F88BF54A90BD97A9A5EF8203052F864
:10F1500020205A4341F82020401C80B28742F3D837
:10F16000002138AA0846002D05DD52F82030401C49
:10F1700019448542F9DC00224B461046002D05DD7E
:10F1800053F820C0401C62448542F9DC91FBF2FC3C
:10F19000002154AA0846002F05DD52F82030401CFB
:10F1A00019448742F9DC002273461046002F05DD22
:10F1B00053F82040401C22448742F9DC91FBF2F0D6
:10F1C000BCF1000FB8BF4FF0000C0028B8BF002002
:10F1D0007199491E8C45C4BF7199A1F1010C7099B8
:10F1E000491E8842C4BF7098401E66E0DDF8C8B171
:10F1F0004F4C4FF6FF7AD34504BF3CF802BCD345D1
:10F2000007D12CF8043C99F8913004EB830323F8E0
:10F21000021C917A99F80A30994238BF89F80A108D
:10F22000D17A99F80B30994238BF89F80B10117BCD
:10F2300099F80C30994288BF89F80C10517B99F8E5
:10F240000D30994288BF89F80D1099F80AA099F8F5
:10F250000BB0CDF8C8B11378527899F80D1002FBB5
:10F26000053299F80C4018F802208B4502F03F094E
:10F270003FF607AF0BFB05F292B273925246A245DE
:10F2800011D8739B134418F803C00CF03F0ECE4501
:10F2900005D12CF03F0C4CEA000C06F803C0521CC0
:10F2A00092B2A242EDD90BF101021FFA82FB8B450B
:10F2B000E0D9E6E64FF0000C60468299A1F800C064
:10F2C0008C9908800DF5037DBDE8F08F2DE9F34F93
:10F2D000F9B00546CC22184968460AF03BFBCC221F
:10F2E000164933A80AF036FB002076906D9040F264
:10F2F0008B107890002077907A98027841780848AF
:10F30000D0F800C09CF807309CF806007490BCF858
:10F3100012006E90BCF810007090749810E000001D
:10F320007042002034420020D48F002044900020FE
:10F33000B4900020CDCCCCCC6CD9010038DA0100DF
:10F340004FEA40086E98B0FBF8F970984FEA43080E
:10F35000B0FBF8F84FF6FF7000EA490A00EA4800EF
:10F360007190002075907A98CDF8BCA19CF807B0F8
:10F3700090F800A04078002A00FB0BA00FFA80FA5A
:10F380007CD0581E904278DD01206C90501E01FB0D
:10F3900003000FFA80FB501C01FB030000B235F99B
:10F3A0001AE035F91BA035F910006EF31F445045E3
:10F3B000C4BF60F30F046AF30F0605DC60F30F06A9
:10F3C00001206AF30F04769020B20028BCBF002011
:10F3D00060F30F0430B20028BCBF002060F30F06BA
:10F3E0000FFA84FB0EEB0B004FEA0E3ABAFBF0FA71
:10F3F000CDF8CCA14FEA0B3ABAFBF0F0DDF8CCA186
:10F400007290AAEB000041F6333B75900FFA86FA32
:10F4100000FB0BF00AFB00F0B0FBFEF0DDF8CCA126
:10F42000000B0AFB00F0CDF89CA100F50060DDF8B0
:10F43000D8A1000BBAF1000FDDF8C8A114BFCDF8B8
:10F4400098A1CDF8A0A145D0689000208246729086
:10F450006C98012808BF00206BD002287DD0DDE920
:10F4600066A0A0EB0A0ABAF5406F9ABF0120EB46EE
:10F4700008F1020072D9C5E000E02DE002206C9096
:10F48000012001FB030000B235F91AA035F9100084
:10F490006AF31F4460F30F06BAF1000FBCBF4FF0D0
:10F4A000000A6AF31F440028BCBF002060F30F0667
:10F4B0004FEA244A0FFA86FB0AEB0B004FEA0A3A9E
:10F4C000BAFBF0FACDF89CA14FEA0B3ABAFBF0F088
:10F4D000689000206690B8E703206C90501E01FBF6
:10F4E000030000B235F91AA035F910006AF31F4481
:10F4F00060F30F04BAF1000FBCBF4FF0000A6AF3CB
:10F500001F440028BCBF002060F30F044FEA244AC8
:10F510000FFA84FB0AEB0B004FEA0A3ABAFBF0FA47
:10F52000CDF89CA14FEA0B3ABAFBF0F066900020B0
:10F530008AE70DF5CC7BDDF8C8E15BF820B0DE444E
:10F54000CDF8C8E102EB000EAEF1010E401C0BFB42
:10F550000EAAC0B20328ECD301E011E03AE0DDE9E5
:10F56000700BA0EB0B0000FB0AFA7298BAFBF0F0EC
:10F570000001A3F1010AB0FBFAF000EB081047E02C
:10F58000DDE9670AA0EB0A0ABAF5406F8EBF08F101
:10F5900001000120EB4617D83BF810E0F24502D2FB
:10F5A000A0F1010A03E0401CC0B26628F4D34FEA80
:10F5B000083000F5805000FB0AF8DFF818A800209A
:10F5C000D346E8FB0AB0400CDDF8C481A8EB00008C
:10F5D000401C1DE03BF810E0F24502D2A0F1010A08
:10F5E00003E0401CC0B26628F4D34FEA083000F5AF
:10F5F000005000FB0AF8DFF8DCA70020D346E8FB48
:10F600000AB0400CDDE9708AA8EB0A084044801E6D
:10F61000DDF8B081B8F1010F41D1DDF8D48141F2BC
:10F62000545A08FB0AF84FEA183ABAF5805F88BFC7
:10F630004FF4805A4FF00108EB463BF818E0F245D2
:10F6400006D20DF1CC0A0AEB480838F802AC06E005
:10F6500008F1010808F0FF08B8F1660FEDD30FFAC2
:10F6600084F836B218EB060417D04FEA0838B8FB16
:10F67000F4F83603B6FBF4F4A8EB040404FB0AF434
:10F68000E40A544588BF544604EB4404769EC4F310
:10F69000D714002E0CBF2044001B083000094FF087
:10F6A0000008002975D0749C641E8C4270DD01FB3B
:10F6B0000324A1F1010808FB032801F1010A24B287
:10F6C0000AFB03230FFA88F80FFA83FA35F914407E
:10F6D0002B4635F9188035F91A50012664F31F437B
:10F6E000A845A3BF68F30F0365F30F07012565F372
:10F6F0000F03BCBF68F30F0700256D951DB2002DE9
:10F70000BCBF002565F30F033DB2002DBCBF002533
:10F7100065F30F070FFA83F804EB08054FEA043A84
:10F72000BAFBF5FA4FEA0838B8FBF5F5AAEB05087D
:10F7300041F6333E0FFA87FB08FB0EFE0BFB0EFB78
:10F74000BBFBF4F4240B0AFB04F4CDF8A8A104F5E8
:10F750000064DDF8B4A1240BBAF1000F14BF699561
:10F760006B9540D06B940025AA46012E08BF00245B
:10F7700069D0022E7DD0DDE96954651BB5F5406F77
:10F780009ABF0124EA4609F1020473D9B8E000E007
:10F790002BE001FB032424B24FF0010A0AFB032AE9
:10F7A00035F914402B4635F91A50022664F31F43ED
:10F7B00065F30F07002CBCBF002464F31F43002D2A
:10F7C000BCBF002464F30F071D140FFA87FA05EB82
:10F7D0000A042D03B5FBF4F56A954FEA0A35B5FB2B
:10F7E000F4F46B9400246994BDE701FB0324A1F1B8
:10F7F000010A24B20AFB03230FFA83FA35F91440F5
:10F800002B4635F91AA0032664F31F436AF30F034E
:10F81000002CBCBF002464F31F43BAF1000FBCBF2F
:10F82000002464F30F031D140FFA83FA05EB0A0496
:10F830002D03B5FBF4F56A954FEA0A35B5FBF4F4F0
:10F84000699400248EE70DF5D27B01EB040E5BF882
:10F8500024B0AEF1010E641C0BFB0EAAE4B25D44B1
:10F86000032CF0D3DDE96E4BA4EB0B0404FB0AF48C
:10F8700001E00AE02EE0B4FBF5F42501749C641E5F
:10F88000B5FBF4F404EB091440E0DDE96A45651BBF
:10F89000B5F5406F8EBF09F101040124EA4615D881
:10F8A0003AF814B05D4501D2651E03E0641CE4B271
:10F8B000662CF5D34FEA093404F58054DFF814952B
:10F8C0006543CA460024E5FB09A4640C6F9D2C1B0C
:10F8D000641C1BE03AF814B05D4501D2651E03E0DC
:10F8E000641CE4B2662CF5D34FEA093404F50054E5
:10F8F000DFF8E0946543CA460024E5FB09A4640CE4
:10F90000DDE96E59A5EB09052C44A41E012E37D163
:10F9100041F2545508FB05F52E0BB6F5805F88BF04
:10F920004FF480560125E84638F815904E4505D22B
:10F9300033AE06EB450535F8026C03E06D1CEDB205
:10F94000662DF1D31DB23FB2EB1908BF04F10803D5
:10F9500015D02D03B5FBF3F53F03B7FBF3F3EB1A1B
:10F960007343DB0AB34288BF334603EB43036D9D09
:10F97000C3F3D713002D0CBF2344E31A08331C092B
:10F98000114306D178998C4201D3814201D90121DA
:10F9900077919CF86E109CF86D50CB0901F07F02B6
:10F9A0004FEAD51C05F07F0113D0002B18BF10447F
:10F9B000BCF1000F12D0BCF1000F18BF0C447A99B3
:10F9C000A1F8A8007A98A0F8AA4077987BB0BDE883
:10F9D000F08F904234BF0020801AE9E78C4234BF98
:10F9E0000024641AEBE72DE9F04716460F4604465B
:10F9F00002F078FF8146F848857894F86E00012877
:10FA000004D194F8DD00012818BF002502F076FF2C
:10FA1000804602F077FF0246F04894F890A04FF03D
:10FA2000000C0168BAF1010F488A0B8A94F8921011
:10FA3000C1EBC10109EB41114FF0010934D091F83C
:10FA40007510012908BF84F87590617800291CBFE2
:10FA5000521E914208DA217800291CBFA8F1010248
:10FA6000914201DA84F875C0002DD8BFBDE8F08757
:10FA7000BD420BDC591B491E8F42D8BFB54205DC85
:10FA8000401B401EB042A8BFBDE8F08794F8750047
:10FA9000012818BFBDE8F08784F8DA9084F8D6C052
:10FAA00084F8DDC0BDE8F087617800291CBF521ED4
:10FAB000914206D0217800291CBFA8F10102914291
:10FAC000D0D184F875C0AF4209DB591B491EB94239
:10FAD000A8BFAE4203DB411B491E8E42C4DD84F841
:10FAE0007590C1E72DE9F84F1D4616460C46834632
:10FAF00002F0F8FE014694F89200C0EBC00001EB62
:10FB00004012B6480021BBF1010F03D0BBF1080F32
:10FB100029D046E003684FF0C20C40F2DE4E5F8A07
:10FB2000188B07FB0CF8B3F81AC01B8AB8FBFCF85B
:10FB300040F2045A07FB0EF703FB0AFAB7FBFCFC82
:10FB4000BAFBF0FAB1FBF0F91FFA8CF74FF4946CA2
:10FB500003FB0CF3B3FBF0F080B21FFA88F81FFA36
:10FB60008AFA00901DE000685A2340F6A61AB0F801
:10FB700012C0078B0CFB03F8438B008AB1FBF7F92B
:10FB800000FB0AF0B0FBF7F01FFA80FA40F2465093
:10FB90000CFB00F0B8FBF3F8B0FBF3F01FFA88F8A9
:10FBA00087B24E4534BF48463046A4F8A8005645B3
:10FBB0008CBF50463046A4F8A800454534BF4046A7
:10FBC0002846A4F8AA00BD428CBF38462846A4F8AF
:10FBD000AA000120BBF1080F15D0BBF1010F18BF1F
:10FBE000BDE8F88F4E4522BF009AB242454503D387
:10FBF000BD4298BFBDE8F88F94F8DD20022A18BFF7
:10FC0000BDE8F88F1CE04E4528BFB24504D34545FA
:10FC100024BFAF42BDE8F88F94F8DD30022B0FD03F
:10FC200084F8DB0092F8DB20012A18BFBDE8F88FCA
:10FC300084F8DA0084F8D61084F8DD10BDE8F88F77
:10FC400084F8DA0084F8D61084F8DD1084F8DB102C
:10FC5000BDE8F88F2DE9F74F86B0144602F022FE7A
:10FC6000064602F033FE814602F03CFE01465B4848
:10FC70000068428A0492008A039094F89200C0EBD4
:10FC8000C00001EB401502F03DFEDFF84C8105900D
:10FC90000DF1040B98F80300D8B10020FEF788FF9F
:10FCA000DDE9060102AB2246CDF800B0FFF711F9FD
:10FCB000BDF80800A4F8A800BDF80400A4F8AA0044
:10FCC00002F029FE012872D002F025FE08286ED02D
:10FCD000BBE096F83E04002720B121460698FFF7C6
:10FCE000F5FA0746B8F80800B8F80410B0EB011FA1
:10FCF0000DD298F8031051B9401C80B2A8F8080042
:10FD00000009A8F80400DDE90310FEF7BCFEB8F80E
:10FD10000A00B8F80610B0EB011F0DD298F80310D6
:10FD200051B9401C80B2A8F80A000009A8F80600E2
:10FD3000DDE90310FEF7A7FE96F83E044FF0000A37
:10FD400098B999F83E0401280FD994F8DD000328EA
:10FD50000BD1A8F808A0A8F80AA0A8F804A0A8F851
:10FD600006A0DDE90310FEF78EFEDDE9060102AB19
:10FD70002246CDF800B0FFF7ACF896F83E0458B133
:10FD8000012815D099F83E14012902BF022894F8E1
:10FD9000900002282FD042E084F86EA0BDF8080041
:10FDA000A4F8A800BDF80400A4F8AA0037E040E0D9
:10FDB000012F15D0B4F8A81040F24920B1F5167FF4
:10FDC00028BFA4F8A800B4F8AA10B1F5167F26D36E
:10FDD00023E000004F09F2943442002070420020DA
:10FDE00084F86EA086F83EA4BDF80800A4F8A80028
:10FDF000BDF8040011E0012F09D0B4F8A800B0F557
:10FE0000167F9CBFB4F8AA00B0F5167F07D9B5F8E5
:10FE1000A800A4F8A800B5F8A800A4F8AA000E202D
:10FE2000A8F80400A8F80600DDE90310FEF72BFE91
:10FE300046E702F073FD40B102F06DFDBDF80430FD
:10FE4000BDF808202146FFF74DFE95F8B3000328C2
:10FE500007BF2878002809B0BDE8F08F687800282F
:10FE600004BF09B0BDE8F08F0599491E8842A4BFC0
:10FE700009B0BDE8F08F94F8B30001281CBF09B0A9
:10FE8000BDE8F08FB5F8A800A4F8A800B5F8AA005E
:10FE9000A4F8AA0009B0BDE8F08F2DE9F05F044690
:10FEA00002F020FD8649DFF81CB2D1F800909BF8E3
:10FEB00000C0B9F81260B9F81A107200B2FBF1F282
:10FEC00002EB0C031FFA83F89BF801309BF803B098
:10FED0001A4497B264227243B2FBF1F594F892107F
:10FEE000B9F810A0C1EBC10100EB4112B4F8A800B1
:10FEF000B4F8AA10BBF1000F19D0604538BF6046B6
:10FF0000994238BF1946AAEB0C02A2F1010C8445B4
:10FF1000B8BF604680B2F21A531E8B42B8BF194672
:10FF200089B2A4F8A800A4F8AA10BDE8F09F94F83C
:10FF300090B0BBF1010F2AD194F801B0BBF1000FD2
:10FF400010D099F806E0AEF1010EF3451CBF94F80D
:10FF500000B0BBF1000F05D099F80790A9F1010995
:10FF6000CB450AD194F891E0DFF85CB14FF0050978
:10FF70000BEB4E0B2BF8029C09E094F891E0DFF8B4
:10FF800048914FF0000B09EB4E0929F802BC40459F
:10FF90001ED294F8DD00032819D194F891904A48B4
:10FFA00000EB490B3BF8020C052810D2B2F8AA90DE
:10FFB0004046B1EB0909B2F8AE1048BFC9F10009DB
:10FFC000A94584BF4FF005092BF8029C00E060466C
:10FFD000B9421ED294F8DD10032919D194F89190FA
:10FFE000394901EB490B3BF8021C052910D2B2F844
:10FFF000A8903946B0EB0909B2F8AC0048BFC9F186
:020000021000EC
:100000000009A94584BF4FF005092BF8029C00E0C8
:100010001946AAEB0808A8F10108804522DA94F8ED
:10002000DD0003281AD194F89190274800EB490984
:1000300039F8020C052811D2B2F8AAC01FFA88F0CC
:10004000B1EB0C0CB2F8AE1048BFCCF1000CAC45D3
:1000500084BF4FF0050C29F802CC03E0AAEB0C009A
:10006000401E80B2A6EB070CACF101078F42BFF631
:1000700058AF94F8DD10032916D194F891C01249B5
:1000800001EB4C0C3CF8021C05290DD2B2F8A8304B
:10009000B9B2C31AB2F8AC0048BF5B42AB4284BFEE
:1000A00005222CF8022C3CE7F11A491E89B238E7E8
:1000B00010B51446FFF7CEFD2046BDE81040ECE633
:1000C0007042002034420020DC90002070B51446BD
:1000D0000D46064602F012FC8446D5E90520296942
:1000E000002904BF002319460AD002EB82029200C5
:1000F0004900B2FBF1F300EB80008000B0FBF1F1AE
:100100002380FF486180A0FB0332A0FB0110D208CE
:10011000C00800FB0C2036F81000A08070BD2DE94F
:10012000F0410446DDE90606089F0D4600281CBF85
:10013000002081F8210002D00020BDE8F08128686D
:1001400020606868C4F80A001068606090882081A8
:100150007C22194604F1140009F0FCFBA868C4F8DD
:100160000E002869A061A889A082A88BA4F870005D
:1001700095F8200084F8D70095F8220084F8D8007C
:10018000012084F8D60084F8D9703078401CC0B2C1
:1001900030700A2828BF0120CED3BDE8F0812DE9B8
:1001A000FF5F1F461646054602F07CFBB0F90200D1
:1001B0004FEAE00A02F0B7FB504502DD02F0B3FB64
:1001C000824600229346904691463046BE4221DC4C
:1001D000B0420CBF0146411ECBB2B8420CBF014633
:1001E000411C01F0FF0C08F101011FFA81F835F9FB
:1001F000101051450ADD49B135F913309942A4BFB9
:1002000035F91C30994201DB82B203E0401C00B298
:100210008742DDDA3C46B74220DB0CBF2046601E39
:10022000C1B2BC420CBF2046601CC3B209F1010040
:100230001FFA80F935F9140050450BDD50B135F93E
:1002400011108842A4BF35F91310884202DB1FFA4F
:1002500084FB03E0601E04B2B442DEDA93450DD0A5
:100260004FEA48022946019809F07EFB01984FEABF
:10027000490205EB4B0100EB480004E0B81B4000CD
:10028000821C2946019809F06FFB08EB090004B0B5
:1002900080B2BDE8F09F2DE9F0479CB084462498D9
:1002A0008A464FF00008017840784446CDF8008037
:1002B000CDF80480CDF80880CDF80C80CDF8108002
:1002C000CDF81480CDF81880CDF81C80CDF82080B2
:1002D000CDF82480CDF82880CDF82C80CDF8308062
:1002E0004FEA8109CDF83480CDF83880109411940C
:1002F00014941F468600129413941594169419941E
:10030000179418941A944B46224669466046CDF8D5
:100310003C801B94FFF743FF0546334622460EA957
:100320005046FFF73CFF0446002109F102008542D8
:1003300014DC0020002DC8BFE9460FDD09EB4002A8
:1003400039F91030B2F902C0BCEB030248BFA3EB8D
:100350000C021144401C00B2A842EFDBA6EB0800DF
:100360000022801CA042A4BF0020002CC8BF0DF1B9
:1003700038080FDD08EB400338F910C0B3F902600C
:10038000B6EB0C0348BFACEB06031A44401C00B2AA
:10039000A042EFDB88009100B0FBF5F0B1FBF4F177
:1003A0000844400838841CB0BDE8F08770477047A7
:1003B00070470028DCBF002070474FF480714FEA7F
:1003C000002C00200B129CFBF3F30A46991801EB5A
:1003D000D1714910531A48BF8B1A802B02DB401C85
:1003E0006428EFD3081270472DE9FF4F85B01F46F0
:1003F00016460D46002402F081FA0190B6F900E09D
:10040000B6F902000290287903906A79E87995F8A4
:1004100006A0A446654666460090824229DC039801
:10042000504521DC029902EB8203C1EB430303FB3D
:1004300003FB019902FB0108059931F918100A29FB
:100440000EDD00EB8008CEEB480808FB08F903FB43
:1004500008F809FB01CC0BFB015508FB01660C44B5
:10046000401C00B25045E4DD501C02B200988242AC
:10047000D5DDDFF8908088FB0C104111A1EBE07115
:1004800088FB05204211A2EBE07288FB0630431185
:10049000A3EBE0734CB1080211021A0290FBF4F0D6
:1004A00091FBF4F192FBF4F202E0002001460246D7
:1004B00000FB01F302FB12320844C0F1000C1412DD
:1004C000A0000CFB0CF1C0EB212000124100002920
:1004D000D8BF002019DD0D024FF4807000210312F7
:1004E00095FBF3F30246981800EBD0704010131AF6
:1004F00048BF831A802B02DB491C6429EFD303E039
:10050000CDCCCCCC1F85EB510012000200EBD0709B
:10051000DCEB60010CEB6000C0F100027C6148BFC5
:100520004942F960002AB8BF524201EB8100400005
:1005300088FB0030C310A3EBE0703A61FF28C8BF0E
:10054000FF2049115211FF2988BFFF21FF2A88BFD0
:10055000FF22002912BF002A01210A46002808BFF5
:10056000012087F8750087F8761087F8772009B0A2
:10057000BDE8F08F2DE9F04117460C46064602F023
:10058000BDF9054602F0BEF9014623786078002BDC
:10059000CCBF5A1E0022A5F1010C6345B4BF5C1C00
:1005A00064460028CCBF431E0023A1F1010C604526
:1005B000B4BF401C60464FF0000C83420FDC114674
:1005C000A24208DC03FB0518491C36F9188009B261
:1005D000C444A142F6DD591C0BB28342EFDDC7F8DB
:1005E0001CC0BDE8F08170B5044602F087F90546ED
:1005F00002F088F92178024600291CBF681E81425A
:1006000006D0607800281FBF511E8842002070BDB0
:10061000012070BD70B50D46044602F06FF9064624
:1006200002F070F9227801230146002A1CBF701ED7
:10063000824206D0607800281EBF491E88420020F2
:1006400000D11846002818BF85F86230002070BD20
:100650002DE9F007A0F1020ADDE90A54DDE9089668
:10066000079F4FF0000804EB400C8A45B2BFA3F887
:1006700000803CF804ACA3F800A0431E8B42B2BF3C
:10068000A7F800803CF8021C398034F81010A9F853
:100690000010411C91428EBFA6F80080BCF80210E9
:1006A0003180801C90428EBFA5F80080BCF8040009
:1006B0002880BDE8F00770472DE9F0018A1ADDE9CE
:1006C0000847DDE90565DDF81CC0994202BF20F846
:1006D00032C0BDE8F0017047AB1BACEB0501A4EBE9
:1006E0000C05CB1A2EB2711A01EB41013C1B4900DB
:1006F0000FB203EB4303A11B5B0001EB41011DB2F1
:1007000049000BB2794205EB8101C3EB031421448C
:100710008C00002CC8BF891104DC890049420912F1
:10072000494209B24C4203EB84031DB24B1B002B20
:1007300003DD2B2463431B1205E06FF02A0463439F
:100740001B125B421BB26C1001EB45012B25694368
:10075000A6EB21210DB29E0000215F0106EB0416DD
:1007600007EB84174FF06C0803FB08F304EBC40499
:1007700003EB041305EB450406EB851607EBC517E1
:1007800003EB841306EB0C2607EB0C2703EB0C237F
:1007900046F30F2647F30F2743F30F2400EBC20362
:1007A00020F832C05E80491C9F8089B2DC80042919
:1007B000F4D3BDE8F00170472DE9FF4F03F10108C4
:1007C00085B01E46154681461146424532BF002778
:1007D00009B0BDE8F08FB246881EA842B2BF3B46C2
:1007E00009EB410030F9043C4A1EAA42B2BF3A4626
:1007F00009EB410030F9022C39F911C04C1C544569
:100800008EBF384609EB4100B0F9020001F1020B3E
:10081000B3458EBFBA4609EB410ABAF904A0CDF838
:1008200008C0CDE90032CDE9030A33462A460698CE
:10083000FFF742FFA1B24145CDD309B0BDE8F08F2B
:1008400030B48278037890F803C04478D21AACEBC5
:10085000040C0B70D2B20CF0FF0483784FF0000C44
:100860008B70052A26D209E023B38D7883F001032B
:100870006D1E8D70521ED2B2052AF5D242784A7092
:10088000C078C870052C3CBF30BC7047BCF1000F6D
:1008900001BF4878401C48704FF0010C1FBFC8785A
:1008A000401EC8708CF0010C601EC4B2052CEDD245
:1008B00030BC70470B785B1C0B700123DAE72DE925
:1008C000FF4FF5B01C46DDE98295074602F01AF8A5
:1008D000064602F013F8804670A909F10400FFF7FC
:1008E000AFFF9DF8C001002818BF401EC0B28DF8B0
:1008F000C0019DF8C211A8F1010291420CBF11463E
:10090000491CCAB28DF8C2219DF8C111002918BF37
:10091000491E8DF8C1119DF8C311731E99420CBF79
:100920001946491C8DF8C311101A20709DF8C30197
:100930009DF8C111E946401A607028789DF8C011F1
:100940009DF8C141401AC6B2A878B5F90450001B01
:1009500000F0FF089DF8C301A04224BF4FF0000A39
:10096000DFF884B639D3CDF888A1CDF88CA1CDF8C5
:1009700090A1CDF894A1CDF898A1CDF89CA1CDF887
:10098000A0A1CDF8A4A1CDF8A8A1CDF8ACA1CDF837
:10099000B0A1CDF8B4A1CDF8B8A1CDF8BCA1DBF8D9
:1009A00000009DF8C2319DF8C021C07962A9604362
:1009B00007EB4000FFF700FF9DF8C1013822201A25
:1009C000C0EBC00009EBC00062A908F0CDFF601CBD
:1009D000C4B29DF8C301A042C5D2B700C8EBC80895
:1009E000FCB209EBC8013822769808F0BDFF6FF021
:1009F000020000EB86003A1D824218DD9DF8C0110E
:100A00009DF8C231591A00EB880339F913309D4221
:100A100009DA002807DBB0EB810F04DCC4B204EB79
:100A2000880339F91350401C00B28242EBDC9DF878
:100A3000C3119DF8C1210020891A58BF71AA0BD497
:100A4000C0EBC00304EB830339F8133022F81030F5
:100A5000401CC0B28142F3DACBB2002271A8779970
:100A6000FFF7AAFE79B0BDE8F08F2DE9F05F1446DC
:100A70000E46054601F016FFDFF86CA500F13E07B3
:100A80002078DAF80020617894F805C0D27901FB6B
:100A90000200385C00F03F08E079401C60458CBFE4
:100AA0004FF00009BDE8F09F2379A079401C9842DF
:100AB00021D9DAF8001007EB030BC87900FB0CF220
:100AC0000CFB003012F80B2002F03F02424518BF29
:100AD00025F8109009D136F91020B1F90C108A428E
:100AE000CCBF25F8102025F81090581CC3B2A0796F
:100AF000401C9842DDD80CF1010000F0FF0CE079B9
:100B0000401C6045D0D8BDE8F09F2DE9FF4F87B06D
:100B10000E461598446801F0F1FE059001F0F2FED2
:100B200000210291079A00910191039104911160B3
:100B300031800746220E4FF00009C4F307200599C3
:100B4000C846EA460692824224BF04F0FF0EC4F370
:100B5000074B3DD3F446E34535D3059A00FB02C36A
:100B6000149A32F913400A2C0EDB3288521C328060
:100B7000B84238BF0746404588BF80468C4538BFDD
:100B80006146CC4588BFE14600233AF91320A242D2
:100B90000FDA0822082B09D20AEB420535F8025C6D
:100BA0002AF81250521ED2B29342F5D32AF81240BC
:100BB00003E05A1CD3B2092BE7D30CF1010202F077
:100BC000FF0CDC45C9D9401C069AC0B29042C1D97D
:100BD000A9EB01000999401C08700A99A8EB0700CD
:100BE000401C0870002007993AF91020401C096841
:100BF000C0B20A44079909280A60F4D30BB0BDE8D3
:100C0000F08F2DE9FF4FF9480D468DB0D0E9001265
:100C10001A9CCDE90012D0E90212CDE90212D0E906
:100C20000412CDE90412D0E90610CDE9061001F056
:100C300039FE3E30089001F061FE064601F062FE8A
:100C4000B5F902700B9729780A916978099100210A
:100C50004FEA072C8A46884689460B460A46A0F189
:100C6000010EA6F1010BCDF830C0002024F81100D0
:100C70003DF812C00A9860440FFA80FC02A830F8D0
:100C800012500998284405B205FB06C000B2002D99
:100C9000A8BFAE452DDBBCF1000FA8BFE34528DBA4
:100CA000DDF834C03CF910C024F811C0BCF1000FCD
:100CB00006DC4FF0010C24F811C0BCF1000F05D088
:100CC00034F91150DDF830C0BCFBF5FCE24408F10A
:100CD000010C0CF0FF0834F911C0CC45C8BFE14647
:100CE000089D285C00281CBF581CC3B20CEB0700F1
:100CF00007B2481CC1B2501CC2B2042AB5D30022AC
:100D0000002024F8110004A830F812C00A986044AA
:100D10000DF1180C00B23CF81250DDF824C0AC44C0
:100D20000FFA8CFC0CFB06052DB2BCF1000FA8BF1E
:100D3000E64513DB0028A8BF83450FDB0D9830F98B
:100D4000150024F811000028DCBF012024F8110050
:100D50000898405D00281CBF581CC3B2481CC1B293
:100D6000501CC2B2042ACBD31098B8F1000F037004
:100D70000B98484401B214BFBAFBF8F000200029D8
:100D80001ABF3A02B2FBF1F200221202002814BF8D
:100D9000B2FBF0F20022000A0F9BA3F84A100F9951
:100DA00008650F98A0F848700F98426511B0BDE82B
:100DB000F08F2DE9FF4F05468B4881B00F46006844
:100DC00014464FF00008B0F92CB0B0F92E10009185
:100DD00090F8BFA0B5F9026001F090FD814601F0E6
:100DE00091FD0346B34524DDB4F900000028C4BFDB
:100DF000B4F90210002903DD0844304400B210E0C9
:100E0000B4F904100029C1BFB4F90620002A8818DB
:100E1000304405DC6288314410440844E1880844C9
:100E200000B20099884204DAA88B504538BF4FF0D1
:100E300001083046002234F812100844511C0AB24E
:100E400000B2042AF7DB002287F86320B8F1000F14
:100E500022D00499491C90FBF1F081B2687810B35C
:100E60005B1E984204BF95F800C0BCF1000F07D08C
:100E7000984222D195F800C0A9F10109CC451CD1B6
:100E8000032087F86300002034F91030B6EB430FDD
:100E90001DDA87F863201EE0A98900291CBF90FB9A
:100EA000F1F081B217E095F800C0BCF1000F1CBF53
:100EB000A9F1010AD445D3D1E2E7002818BF98422E
:100EC00009DA2878002808BF012004D1D9E7401C9E
:100ED00000B20428D8DBA7F8581005B04046BDE89A
:100EE000F08F2DE9FF4F85B00C4606460025DDF852
:100EF000489001F003FD039001F004FD029096F884
:100F000000807778B68901F00EFDB4F90020B4F9BD
:100F1000021001911144B4F90430B4F90620009292
:100F200040101A449142CCBF11B209B2B4F908C0C2
:100F3000B4F90EA0B4F90A30B4F90C200CEB0A0B8A
:100F400003EB020EF345CCBF0FFA8BFB0FFA8EFBBF
:100F50003FB9DDF804E08645C4BF00F1010EA4F8F6
:100F600000E0DDF808E0AEF1010E774505D1B4F9F7
:100F700000708742C4BF471C6780B8F1000F04D1DE
:100F8000009F8742C4BF471CA780039F7F1EB845B0
:100F900005D1B4F904708742C4BF471CE780B4F997
:100FA00004708742C4BFB4F90680804520DD8445C3
:100FB000BEBF8342B4F90030834206DB8245BEBF28
:100FC0008242B4F90220824200DA0125052E24D2A1
:100FD0000798401CB04220D1594526DCB9F1010FD9
:100FE00023D9089808BB24E07042002004DB0100EC
:100FF000B4F900808045C4BFB4F902808045E5DDC6
:101000008445BCBF82428742DFDB8342BEBF82454C
:10101000B4F906208242D8DBD8E7594500DD25B176
:10102000B9F1010F01D9089818B109B00020BDE845
:10103000F08F09B00120BDE8F08F2DE9F04186B0B6
:1010400014460F468046002501F02CFC064602A8F7
:10105000009001AB224639464046FFF7D2FDB07EF4
:10106000002804BF96F83400002807D19DF804300A
:1010700002AA21463846FFF79CFE0546002084F868
:101080005A5084F85F0006B0BDE8F08170B515468F
:101090000C4601F007FC014600208A7E002A06BFAC
:1010A000097B002970BDA1891E2981BF95F87610A2
:1010B0004B29E18B072906D895F87610642986BF5D
:1010C000E18B062970BD012070BD2DE9F74FACB052
:1010D0009246074601F0F0FB299001F0E3FB2390D4
:1010E00000208DF8880006460546BAF1000FC8BFFB
:1010F0004FF0010B40F3E3802D9805EBC50100EBA9
:10110000810494F82100012840F0D4807C2101A8BA
:1011100008F025FC00202090219001A84FF0000944
:10112000289001F0BFFB804624A800902AAB2146FE
:101130003846289AFFF765FD98F81A00002804BF82
:1011400098F83400002807D19DF8A83024AA20463A
:101150002899FFF72EFE814600208DF85E908DF8CD
:10116000630001F0CBFB0346D4E90401A269002827
:1011700004BF002108460AD001EB8101890040002C
:10118000B1FBF0F102EB82029200B2FBF0F0ADF89D
:1011900080104E4AADF88200A2FB01C1A2FB0020E4
:1011A000C908C00800FB031101AB37F81100ADF806
:1011B000840020AA21463846FFF716F901F072FB99
:1011C000817E4FF00009002904BF007B002811D167
:1011D000A0891E2881BF9DF87A004B28E08B072844
:1011E00006D89DF87A00642884BFE08B062801D9D0
:1011F0004FF00109B9F1000F1CBF239880F836B0F9
:1012000001F07CFB804601F07DFB01462078002840
:101210001CBFA8F10102904206D0607800281EBFD2
:10122000491E8842002000D15846002818BF8DF87A
:1012300066B09DF888007C22C0EBC001299800EBC5
:1012400041182068C8F800006068C8F80A002098B3
:10125000C8F80400BDF88400A8F8080001A908F146
:10126000140008F077FBA068C8F80E002069C8F8E1
:101270001800A089A8F81400A08BA8F8700094F8B2
:10128000200088F8D70094F8220088F8D80088F861
:10129000D6B088F8D9909DF88800401CC0B28DF86F
:1012A00088000A282CBF0120002040B9A089B04244
:1012B00088BF0646681C05B25545FFF61DAF23984A
:1012C00086809DF888002FB0BDE8F08FCDCCCCCCC7
:1012D000F0B5ADF23C4D0F46064601F0E3FA044688
:1012E00001F0F4FA05464FF48761684608F037FBD1
:1012F000A07E012805D195F830203146384606F009
:1013000076FF01F06AFB00281CBF384607F0F6FBA9
:101310006A463946304603F0DAFD84F82E0002466C
:1013200069463046FFF7D1FE0546A07E012803D16D
:101330002946304607F0DDFB01F054FB002806BFCC
:10134000002084F844040A2D04D22946304601F0D6
:101350003BF9054684F82F500DF23C4DF0BD0000DE
:10136000FE484CF6CD430268FD48B2F8C6108181B4
:101370005943C90C0181B2F8C410C1815943C90C49
:1013800041812321018207214182F6498161322175
:1013900081827047F24800897047F1488089704720
:1013A000EF496428088184BF6420088180B200EB83
:1013B00080004FF6FF7202EA400088817047E848DB
:1013C00040897047E648C0897047E549B0F5C87F55
:1013D000488184BF4FF4C870488180B200EB800020
:1013E0004FF6FF7202EA4000C8817047DC48008A6D
:1013F0007047DB4908827047D948408A7047D8490E
:10140000B0F5C87F488284BF4FF4C87048827047E7
:10141000D348808A7047D249B0F5967F888284BFCE
:101420004FF49670888280B24043642250438861B2
:101430007047CB488069704770B501F033FA01F00E
:1014400045FA044690F84104C54E002538B994F891
:10145000420418B92021C44808F095FAB58094F8E0
:101460004204002808BFF58070BD10B501F01AFADB
:1014700001F044FAF323002100288CBFBA4A10BDC2
:1014800012F801C00CEA030C02F801C0491CC9B2F1
:101490008842F5D810BD70B5054601F003FA01F099
:1014A0002DFA012D08BFFE2402D0022D08BFFD2415
:1014B000002100288CBFAC4A70BD535C23405354BC
:1014C000491CC9B28842F8D870BD70B514460D46A3
:1014D000064601F0E7F901F0EFF90023012E02D0F2
:1014E000022E08D00EE0042C08BF01230AD0052CE0
:1014F00008BF042306E0042C08BF022302D0052CF9
:1015000008BF0823C5EBC50100EB4111887A0A7BAF
:1015100082422CBF944A70BD12F800C04CEA030C02
:1015200002F800C0401C91F80CC0C0B28445F3D250
:1015300070BD2DE9F04116460D46074601F0B2F99F
:1015400001F0BAF901F0DEF9804601F0D7F9014661
:1015500082482C46B5420068B0F90E30824810D857
:1015600037F914209A4208DD025D0C2C42F0040287
:10157000025524BF42F010020255621CD4B2B4429C
:10158000EED9A8F1010251438AB2B54228BFBDE8A5
:10159000F081511937F91110994208DD415D0C2D88
:1015A00041F00801415524BF41F020014155691C1B
:1015B000CDB2B542EDD3BDE8F08110B501F09EF992
:1015C000002100288CBF684B10BD5A5C12F0100F30
:1015D0001CBF22F010025A54D2B212F0200F1CBFCE
:1015E00022F020025A54D2B212F0040F1CBF42F073
:1015F00010025A54D2B212F0080F1CBF42F020025F
:101600005A54491CC9B28142DFD310BD2DE9F05FA5
:1016100090468946834601F045F9044601F04CF9AD
:10162000064601F05FF994F82F5001F06BF902467D
:101630004A48006890F8CDA00020014604460746BD
:10164000002D88BF921E33D9C4EBC40306EB4313AD
:1016500083F8C97083F8CB7093F88CC0BCF1000F8D
:1016600001BF93F8D6C0BCF1010F93F872C0BCF172
:10167000000F19D193F801C0BCF1010F98BF4FF0D2
:10168000010C04D99445A8BF4FF0020C0CDB83F881
:10169000C9C0BCF1010F04BF401CC0B204D0BCF1F2
:1016A000020F04BF491CC9B2631CDCB2AC42CBD3ED
:1016B0002E4A4FF00004137852781844114410F069
:1016C000FF00C9B218BF00290AD00844824507D8D4
:1016D0000124424649465846FFF72BFF20484780E1
:1016E0002046BDE8F09F2DE9F04101F0DBF804460B
:1016F00001F0E2F8054601F0F5F81848184994F8A9
:101700002F400068B1F80CC00022408A002C86BF30
:10171000A0EB0C060627BDE8F081C2EBC20005EB8A
:10172000401191F88C00002804BF91F8DD000228D8
:101730000FD1B1F8AE3063459CBF81F8C87001206D
:1017400005D9B342A4BF81F8C870022001DB81F83B
:10175000C900501CC2B2A242DFD309E0704200208F
:101760004442002090D00300FA9000204A4200201A
:10177000BDE8F0812DE9F04116460C46054601F022
:1017800091F801F0BFF8804601F0B8F8FE49B44284
:101790000968B1F90E3088BFBDE8F081A8F10107F2
:1017A000A8F1020CDFF8E48335F9142001199A42FC
:1017B000BCBF35F91110994205DA18F8041021F070
:1017C000040108F8041007FB004189B20CFB004239
:1017D00035F9111092B29942BCBF35F912109942F5
:1017E00005DA18F8041021F0080108F80410611C4B
:1017F000CCB2B442D8D9BDE8F0812DE9F04F85B024
:1018000001F050F8044601F057F8019001F06AF831
:10181000DD490090DE4809684FF0000BD0F81890C1
:1018200091F8CE2003928789C589488A94F82F8041
:10183000C11B401B89B286B25C460291B8F1000F11
:1018400040F2D6800198C4EBC40100EB411292F83B
:101850009200C0EBC001009800EB411392F88C009D
:10186000002870D192F8C80006286CD04FF0000C08
:1018700082F8C8C092F8DD00022818BF032804D0FF
:1018800092F8D60001286ED0ADE082F8C9C0B2F857
:10189000AE00A84282BF8642022082F8C80008D863
:1018A00092F89000022802BF93F8C800022882F83C
:1018B000C80092F8DD00032804BF92F890100229B6
:1018C00005D193F8C810012908BF01207AD092F8F9
:1018D000C810022918BF012935D002280CD092F86F
:1018E0009000022804BF93F8CA00002804D0B2F880
:1018F000AE00A84206D918E0B2F8AE00B84203D94B
:10190000A84201D8012005E00299814217D98642F8
:1019100015D8022082F8C90092F8DD10022913D0F0
:1019200092F89010022903D009E08642F1D906E02E
:1019300093F8CA1041B193F8C810032914D082F863
:10194000C8C082F8CAC04EE0B2F8AC00A2F8CC0021
:10195000B2F8AE00A2F8CE00032082F8C800012041
:1019600082F8CA003FE036E0B2F8AC10B3F8CCA081
:10197000B3F8CEE0A1EB0A0CB2F8AE100CFB0CFCF5
:10198000A1EB0E0101FB01C149451EDCA2F8CCA070
:10199000B3F8CE10A2F8CE1093F8CA10491CC9B201
:1019A00082F8CA10039B994238BF03200AD304214E
:1019B00082F8C8100A462146FFF787FD4FF0010B59
:1019C00011E0FFE782F8C8000DE0012082F8C800AE
:1019D00082F8720007E0B3F8CC00A2F8CC00B3F8AC
:1019E000CE00A2F8CE00601CC4B24445FFF42AAF7A
:1019F00005B05846BDE8F08F2DE9F05F6448002738
:101A00003C46B0F810A0408A0FFA80F900F04AFF77
:101A1000054600F051FF95F82F60002580464FF0F5
:101A2000040B002E57D9C5EBC50008EB401090F809
:101A30008C1000294BD190F8C810042918BF062932
:101A400045D090F8DD10022902D0032909D03EE0EC
:101A500090F8C910002904BF681C60F3070404D182
:101A600035E090F8C910002931D0017C827BC37B1E
:101A7000891ACAB2417CC91AC9B28A428EBF1346BA
:101A80000B461146828A524506D2591A4945A4BFCF
:101A9000B0F90210A02909DD80F8C8B090F8C9009B
:101AA00004222946FFF711FD012710E090F8CA1023
:101AB00001290CD190F8C900012804BF681C60F30B
:101AC0000F2404D0022804BF681C60F31744681C6C
:101AD000C5B2B542A7D30025002E2FD904F0FF0AC6
:101AE000C4F30729C4F30744C5EBC50008EB401055
:101AF00090F88C10F1B990F8C810042918BF062985
:101B000018D090F8DD10022918BF032912D190F8DF
:101B1000CA1001290ED9BAF1000F18BF514610D0D2
:101B200041B180F8C8B090F8C90004222946FFF7F7
:101B3000CCFC0127681CC5B2B542D5D33846BDE8F8
:101B4000F09FB9F1000F05D090F8C910012908BF26
:101B50004946E5D0002CEDD090F8C910022908BF05
:101B60002146DDD0E6E72DE9F05F9A4691460E4624
:101B700007460A9D00F0C2FE804600F0C3FE834681
:101B80000148006806E0000070420020FA90002042
:101B90004442002090F8CC00022354464FF0010C40
:101BA000AA4598BFA8F1010215D803FB084139F9ED
:101BB000111081420BDB07F804C0002C1CBF39193F
:101BC00001F801CC9442BCBF391981F801C0611CF5
:101BD000CCB2AC42E9D9ABF10301CAB2AA4594BF79
:101BE000A8F10103BDE8F09F02FB08A189B239F911
:101BF000111081420EDB06F80AC0BAF1000F1CBFBB
:101C000006EB0A0101F801CC9A45BCBF06EB0A01BC
